:020000040800F2
:1040000000500020917D0008657C0008697C000854
:104010006D7C0008717C0008757C000800000000C1
:104020000000000000000000000000007D7C00088F
:10403000797C000800000000817C00085DA8000871
:10404000857C0008897C00088D7C0008917C000834
:10405000957C0008997C00089D7C0008A17C0008E4
:1040600000000000A57C0008A97C000800000000FA
:104070000000000000000000000000000000000040
:104080000000000000000000C97C0008CD7C000892
:10409000DD7C0008ED7C0008097D000899450008DA
:1040A000197D0008094C0008814900080000000043
:1040B0001547000841460008E94600081D7D000834
:1040C000FDC30008257D000879C400082D7D000887
:1040D000317D0008357D00088545000871450008E0
:1040E000417D0008457D0008497D00080000000072
:1040F00000000000000000000000000000000000C0
:0C41000000000000000000005FF800005C
:10410C0030BF704720BF704740BF7047BFF36F8F01
:10411C007047BFF34F8F7047BFF35F8F704701DF5E
:10412C007047EFF31480704780F31488BFF36F8FE0
:10413C007047EFF30980704780F309887047EFF3FD
:10414C000880704780F30888704772B6704762B673
:10415C00704771B6704761B6704780F3118870472D
:10416C00EFF31280704740BA704700BA70470000F6
:10417C00054A0649064B1160064A1360064A13604D
:10418C00064A1360704700BFB80400206194000811
:10419C001993000894040020640300208C04002070
:1041AC00064A074B1A60074A074B1A60074A084B26
:1041BC001A60084A084B1A60704700BF39BC0008E7
:1041CC006403002045BE0008B804002039BE000876
:1041DC008C04002035BC000894040020044B054AD4
:1041EC001360054A1360054A1360054A1360704753
:1041FC00199300086403002094040020B8040020E4
:10420C008C040020704700BF704700BF30B597B0DA
:10421C0003F0A4FA03F0C2FA0AF092FF694B0024EF
:10422C004FF480301C700AF0ABFF0BF00FF9012833
:10423C0032D10F300BF042FE02200BF027FE20464D
:10424C000AF0EEFF20460AF0FFFF4FF480600AF000
:10425C00F1FF5D4B5D4A1B68934202D14FF4403035
:10426C0004E05B4A934205D14FF480304FF4E011E7
:10427C000AF0B2FF01200AF0BBFF39200BF0D0F896
:10428C000028FAD002200AF0B9FF0AF0C1FF082872
:10429C00FBD14C4B01221A70012001460BF076F831
:1042AC004FF000604FF480410BF0D2F94FF44070A6
:1042BC000BF030F9474B1B78552B0ED1464B1B7826
:1042CC00532B0AD1454B1B78422B06D1FFF750FFDD
:1042DC00434B01221A70013A05E0FFF761FF404B96
:1042EC0000221A7001323F4B3F4C1A7005F038FB1C
:1042FC0005F070FB07F0CEFF03F0FCFE06F08AFA27
:10430C0020463A4905F012FE05F03EFB384B1B786F
:10431C00012B05D1207804F0ADFDE07804F0BAFC57
:10432C002F4B1B78012B25D1324C0DF1100C25464F
:10433C000FCDACE80F00AE46BEE80F00ACE80F00A6
:10434C009EE80F0030340DF1400E8CE80F000FCCBE
:10435C00AEE80F0094E8030004AD02248EE80300DD
:10436C0022460195042010AD2349002302950094A8
:10437C0005F034F91B4B1B78012B05D11A4B1A692C
:10438C005879996807F05EFD00F02AFB01F0B4F94A
:10439C0003F0D0F940F2167006F0ACFE40F2127049
:1043AC0006F006FF03F030FB03F09CFA012002F04C
:1043BC00CBFE00F0E3FF03F0BFF906F0D1FE00F0F6
:1043CC0001FFF1E7A4040020580000200024F400B1
:1043DC0000127A00FC3F0008FD3F0008FE3F000879
:1043EC00140000204D000020BC040020D00300204D
:1043FC004A0000200013010800080140014B186816
:10440C00704700BF9C010020014B5868704700BFEB
:10441C009C010020014B1868704700BF1809002050
:10442C00014B9868704700BF9C01002008B5024BF7
:10443C0018680CF039FF08BD54090020014BD868EE
:10444C00704700BF9C010020014B1868704700BFEB
:10445C0070090020014B1868704700BF2409002028
:10446C00014B1868704700BF2C090020034B93F8D0
:10447C00422022EA000283F842207047D003002039
:10448C00034B93F8423018420CBF002001207047B8
:10449C00D0030020034B93F8512040EA020283F82A
:1044AC0051207047D0030020034B93F8512022EA8F
:1044BC00000283F851207047D0030020034B93F87F
:1044CC00513018420CBF002001207047D00300204F
:1044DC00014B1868704700BF40090020014B186859
:1044EC00704700BF04090020014B5868704700BF9B
:1044FC0004090020014B1868704700BF58090020C0
:10450C00014B5868704700BF5809002008B50120BE
:10451C00FFF7D4FF48B1054B00220420DA60FFF707
:10452C00CDFF10B10120FFF7BFFF08BD9C0100209B
:10453C0008B507F02FF808BD08B506F08FFE08BDCA
:10454C0008B54FF4803005F0DFF908BD08B5044B11
:10455C0093F860301BB94FF4003005F0D5F908BD65
:10456C00D003002008B5034B1B78012B01D104F0BC
:10457C00C9FB08BD4B00002008B5034B1B78012B71
:10458C0001D104F01BFC08BD2902002008B54FF432
:10459C0080700BF005FD70B14FF480700BF00EFDC8
:1045AC00054B1B78012B03D0044B1B78012B02D13C
:1045BC00034B01221A7408BD48000020270200207A
:1045CC009C01002008B50220FFF75AFF38B1044BBC
:1045DC00B3F8400007F010F80220FFF747FF08BDC2
:1045EC00D003002010B50120FFF74AFFD8B107F027
:1045FC0011F80D4991F82530CA6B5B08B2FBF3F347
:10460C00B0FBF3F202FB1303084AA1F84030147814
:10461C0034B9074B403118680222403005F064FB76
:10462C000120FFF723FF10BDD00300202E02002035
:10463C000400002008B5044B1978012903D1034B61
:10464C0018680AF021FA08BD480000204400002038
:10465C0038B51E4C022120680AF010FA012828D126
:10466C00022120680AF010FA002003F0E3F9184C3C
:10467C0005460146607C06F0B9FD164B657493F84F
:10468C00213080B2062B00D09BB9114B01B2DA68F5
:10469C008A18DA6068B10F4B93F861304BB10E4B4E
:1046AC009A6812F0200F02D020225A6101E02022D9
:1046BC001A61064C012120680AF0E0F90128014634
:1046CC0002D120680AF0E0F938BD00BF3C000020A0
:1046DC009C010020D00300200010014008B5074BBE
:1046EC001978012903D1064B18680AF0CDF9054B4E
:1046FC001B78012B01D1FFF7ABFF08BD270200206F
:10470C00440000204000002008B5074B197801290F
:10471C0003D1064B18680AF0B7F9054B1B78012B2F
:10472C0001D1FFF795FF08BD2602002044000020B0
:10473C0025020020B0F5007F10B5044610D003DC34
:10474C00B0F5807F37D121E0B0F5806F03D0B0F5A4
:10475C00006F30D10DE005F0CFF84FF4807019E008
:10476C0005F0CAF84FF4807005F0CEF84FF4806075
:10477C0014E005F0C1F84FF4807005F0C5F84FF463
:10478C00806005F0C1F84FF400700BE005F0B4F850
:10479C004FF4806005F0B8F84FF4007005F0B4F8F1
:1047AC004FF4006005F0B0F84FF4804005F0ACF821
:1047BC00024BA3F86240024B1C6010BDD0030020DA
:1047CC002809002010B504464FF4803005F0A4F8F9
:1047DC00012808D0044B4FF400601C60FFF7AAFFBF
:1047EC00024B00221A6010BD300900205409002031
:1047FC0038B505464FF4803005F08EF801281CD0F2
:10480C000E4B4FF480601C680D4B9D60FFF792FFC0
:10481C004FF4804005F078F8B4F5007F04D1094BD3
:10482C001A68094B1A6008E0B4F5006F05D1074B04
:10483C0018680CF01FFB044B186038BD28090020C9
:10484C009C01002054090020EC08002024090020C1
:10485C0008B5034BDB68C018FFF7CAFF08BD00BFE3
:10486C009C01002008B54FF48070FFF763FF08BD72
:10487C0038B52C4B93F82130082B52D8DFE803F0D5
:10488C00055151515151052F4B00274A0128D3682E
:10489C00254D08BF536101286A69244C6B6102D114
:1048AC00AB6923603DE01F499B1A886991F825C0CC
:1048BC001F494FF0140E0EFB00FE59434FEA5C0CDF
:1048CC00062303FB0CFC91FBFEF1206891FBFCF131
:1048DC00282208F0CBF820602368AB6121E0012886
:1048EC00114B124C02D1DB69236010E011490D4AC7
:1048FC000D680F48916905FB00FC14204843D16BEF
:10490C009CFBF0F292FBF1F222602268DA61094B17
:10491C0000221A6005E0084B18680CF0C5FC034B2C
:10492C00186038BDD00300209C0100202409002011
:10493C00804F12006C0900205409002010B5044669
:10494C004FF4804004F0E0FF034B0120DC609C60DE
:10495C00FFF78EFF10BD00BF9C01002008B5034877
:10496C0004F07CF9024804F079F908BD0409002030
:10497C004009002008B5024820210AF095F808BD2E
:10498C00002C014038B505464FF4803004F0C4FFCC
:10499C0001281AD00D4B4FF400701C680C4B1D6095
:1049AC00FFF7C8FEB4F5006F05D10A4B18680CF080
:1049BC0061FA094B1860094B9B6813F4004F04D142
:1049CC0004F0C4FF08B902F051FF38BD28090020DB
:1049DC007009002024090020540900200010014017
:1049EC0010B502F05BFF012003F034FA404804F0EC
:1049FC0035F9404C404804F031F9404804F02EF9A8
:104A0C0094F8210006F0E0F994F82130062B0ED131
:104A1C004FF4004004F070FF802004F075FF01207B
:104A2C0006F094FC94F82500400806F055FC314C37
:104A3C0094F82130072B23D14FF4004004F064FF8D
:104A4C00802004F061FF94F82A30012B02D1002061
:104A5C0006F07CFC274CE06B94F82C1006F050FE12
:104A6C0094F82510E06B490806F05EFD06F06CFD2D
:104A7C00234B00221A7403F0B3FC012006F06AFDEC
:104A8C001C4C94F82130082B11D14FF4004004F049
:104A9C003BFF002006F05AFCE06B94F82C1006F05B
:104AAC002FFE94F82510E06B490806F03DFD114CE3
:104ABC0094F8213073B94FF4004004F01DFF8020AE
:104ACC0004F022FF012006F041FC94F82500400878
:104ADC0006F002FC0B4C4FF400732361012003F031
:104AEC00BFF94FF48043236102F0C0FE10BD00BF3C
:104AFC0004090020D003002058090020F0080020F1
:104B0C009C0100200010014038B5094C094D94F867
:104B1C00202095F821309A4208D0FFF761FF012040
:104B2C00FFF7A6FE95F8213084F8203038BD00BF81
:104B3C009C010020D00300200A4938B5CC68002322
:104B4C008C600949094D0B60094900220A602A60F2
:104B5C00084A094D01202B601360FFF789FEFFF70F
:104B6C003FFF38BD9C010020700900205409002033
:104B7C00EC080020180900203009002038B51A4B29
:104B8C001B78012B02D106F00BFD03E0174B1868C4
:104B9C0009F06CFF164B0422D96B91FBF2F2904298
:104BAC000ADA4FF0030C0CFB02FC124B5B6A6345F8
:104BBC0002DDCB1A1B180DE003235343984206DD8C
:104BCC000C4B5B6A934202DAC31A5B1A02E0094B84
:104BDC005B6AC31A074A0849D4680D68E41AEB1AD1
:104BEC000B605062D46038BD2E02002044000020BF
:104BFC00D00300209C0100206C0900202DE9F04519
:104C0C009F4B93B01B889F4C13F0100F40F0A28267
:104C1C00A36A18460133A36204F06EFD216B9A4B14
:104C2C00E26A013193F821302163984901324FF443
:104C3C000050072B0861E26208D1954B1B78012BC1
:104C4C0001D106F0C3FC0120FFF798FF8E4B93F8BF
:104C5C002130082B05D18E4B1B78012B01D106F08E
:104C6C00B5FC894D1422AB69864C5343226B9A4296
:104C7C00C0F09B80002318462363FFF7F9FD636B9C
:104C8C004FF480600133636304F046FE00282DD09E
:104C9C00A168804BE268284603F086FF7E4B1860C3
:104CAC0004F06EFD58B104F0E7FD022807D1A268AC
:104CBC00E3680E920F930EAB0FCB04F083FD714A99
:104CCC00714B9068D168DA68411A0029B8BF494223
:104CDC0091420BDC714A9B681268002AB8BF5242A1
:104CEC009A4203DC4FF4804004F006FE664C94F8C4
:104CFC002030012B25D14FF4806004F00DFE68B1FB
:104D0C00604A6749D3689568634A204612680095E3
:104D1C0003F0CCFA0CF0AEF8624B18604FF4007054
:104D2C0004F0FAFDC0B15F4C20680CF0BDFA5A4B90
:104D3C0001461A68544803F083FA0CF09BF8206083
:104D4C000AE0554B216818680A46494207F06EFE86
:104D5C000CF090F8534B18604FF4007004F0DCFD2D
:104D6C0020B900F5806004F0D7FDF0B14D4D4B4CEF
:104D7C0028680CF099FA266801464B4B324642489B
:104D8C0003F0C2FE494B186004F0FAFC68B104F061
:104D9C0073FD012809D128680CF086FA23680E905F
:104DAC000F930EAB0FCB04F00DFD364E364BF16A64
:104DBC00DA699142C0F0A281B76B1A8D0137B763E3
:104DCC000027F7623E260AAC0096394D06F5D276DE
:104DDC00C8214B23204601964FF40266029603F03D
:104DEC00D5F894E8070085E807004FF4806004F0DC
:104DFC0093FD01280CD04FF4007004F08DFD0128B8
:104E0C0006D04FF4006004F087FD012840F0F480D8
:104E1C001D4F97F82140002C54D0204B244AD3F836
:104E2C0000801D4B6D4607CAD3F800C085E807000B
:104E3C0038461B4F134C1D4E05971A4F04F13C0E70
:104E4C00194B1C491C4ACDF810E0CDF81CC0069734
:104E5C00CDF82080039603F009FBB4F93C30B4F98B
:104E6C003E10DFF85CA03468C918144BDAF8000067
:104E7C0010221C6007F0FAFDCAF80000ACE000BF7D
:104E8C00002C01409C010020D003002000100140A8
:104E9C002E02002040090020700900202409002067
:104EAC00EC080020540900200409002030090020DF
:104EBC003409002058090020F008002018090020AF
:104ECC002C090020012192480BF0E8FC05F0B0FD04
:104EDC00012806D003D3022805D020460CE08D4DC6
:104EEC0002E08D4D00E08D4D286802F083FF0446F2
:104EFC00286802F06FFF201A894B4FF4F174198D5A
:104F0C004B223E2300944FF40264019402F07AFF8A
:104F1C00844B854E93F840300446012B08BF444225
:104F2C0021461022306807F0A1FD804D07462A6803
:104F3C0023467F497A48376003F056FE7D4A794B09
:104F4C001268002858642A6002DD002283F8402091
:104F5C00744B5A6C002A02DA012283F8402001209B
:104F6C0002F068FD6E4B054693F8243013B980F0BF
:104F7C000705EDB26B4F70487E6C002EB8BF7642C1
:104F8C00B6B2314609F01AFD6B48314609F018FDEE
:104F9C003146694809F016FD294697F84020012052
:104FAC0005F0EAFE6448202109F0C4FA04F0E8FB9D
:104FBC0090B104F061FC03280ED105F039FD642397
:104FCC0043436FF0630278330E930F941192109257
:104FDC000EAB0FCB04F0F6FB04F0D2FB60B104F087
:104FEC004BFC48B9514B1A684F4B0E921B680F93F0
:104FFC000EAB0FCB04F0E6FB4B4B1A68484B002A68
:10500C005B68B8BF52429A4205DD012004F074FC83
:10501C0002F084FC04E0012004F076FC02F086FC33
:10502C00414B3F49186806F007F84FF4003004F084
:10503C0073FC012808D1414803F010FE404803F0EE
:10504C000DFE0020FFF7BEFB02F078FF3D4BDB7935
:10505C000BB102F0D7FC324B93F8222012F0010F67
:10506C0022D0394A1268002A1EDD93F8233013F03F
:10507C00010F03D0002002F071FC40B9284B93F8CB
:10508C00230010F001000FD102F068FC60B902207F
:10509C00FFF714FA10B1234B0022DA600020FFF75F
:1050AC0071FC2A4B00221A601D4B93F8222012F03F
:1050BC00020F23D0244A1268002A1FDA93F82330F7
:1050CC0013F0020F03D0012002F048FC48B9144B36
:1050DC0093F8233013F0020F10D1012002F03EFCA4
:1050EC0060B90220FFF7EAF910B10E4B0022DA602A
:1050FC000020FFF747FC154B00221A60084B93F871
:10510C002130002B34D1124B4FF400525A612FE056
:10511C000024014020020020180000201C00002068
:10512C00D00300209C0100202C090020180900202D
:10513C005809002030090020002C014004090020EF
:10514C0040090020BC040020240900205409002040
:10515C0000100140A36C18460133A36404F0D2FA8A
:10516C00074B4FF40052074801215A610BF096FB94
:10517C000548012109F088FC13B0BDE8F08500BF9B
:10518C000010014000240140002C014008B502F041
:10519C007DFBA0B904F0DAFB88B900F5005004F0EF
:1051AC00BBFB60B900F5807004F0B6FB38B9044B5A
:1051BC004FF461729A861A879A8702F057FB08BDE2
:1051CC00002C014010B505F01FFB204CE36CC31AFA
:1051DC00002BB8BF5B42B3F57A7F36DD1C4B9B6866
:1051EC0013F4006F2AD102F051FB60B1012004F0DE
:1051FC0083FB402004F080FB94F850300A2B02D83B
:10520C00013384F850304FF4807004F085FB20B9E2
:10521C00FFF7B8FB0F4B00221A6002F037FB80B18E
:10522C000A4B93F850300A2B0BD8094B4FF4806281
:10523C001A6140205A6104F067FB02E0002384F8F5
:10524C00503005F0E1FA014BD86410BD9C010020F0
:10525C00001001405409002010B505F0D5FA194C86
:10526C00636DC31A002BB8BF5B42642B28DD164B51
:10527C00186802F0AFFD154B206093F82B30012B12
:10528C000AD103F55A63984206DD02F0F7FA0420BE
:10529C0004F032FBFFF7E6FA0A4B1B68B3F57A7F92
:1052AC0002DC022004F028FB064B1B68B3F57A7F66
:1052BC0002DD022004F028FB05F0A6FA014B58652C
:1052CC0010BD00BF9C01002028000020D00300204E
:1052DC0010B505F099FA264CA36DC31A002BB8BF74
:1052EC005B42B3F57A7F42DD224B186802F072FD07
:1052FC006060082004F010FBB8B9636840F6B32274
:10530C00934209DD083004F0F7FA02F0EDFA02F0EE
:10531C00B5FAFFF7A7FA26E0B3F5156F0ADC0820FB
:10532C0004F0F2FA02F0E6FA09E0626840F60B23A8
:10533C009A4218DC082004F0E7FA02F0E1FA0E4B6E
:10534C009B6813F4004F0ED104F000FB58B900F524
:10535C00005004F0E1FA30B900F5807004F0DCFA8A
:10536C0008B902F083FA05F04FFA014B986510BDAD
:10537C009C0100202C0000200010014070B505F0AD
:10538C0043FA4F4C0646E36DC31A002BB8BF5B4281
:10539C00B3F57A7F0DDB206E04F096F90025A06B37
:1053AC00256604F097F9606BA56304F099F9E6653E
:1053BC006563444A424B1168434A186E12690029CE
:1053CC00B8BF49420130002AB8BF52429142186618
:1053DC0003DC102004F090FA02E0102004F094FAA0
:1053EC00374CFFF791FBFFF737FFFFF771FF237C7B
:1053FC0063B1354B93F82130072B07D1FFF7F2F847
:10540C00FFF7E0F8FFF782F80023237405F04EFE57
:10541C002D4D6B6D984225D905F0F6F9284C636E2D
:10542C00C31A002BB8BF5B42B3F57A7F1ADB05F0C9
:10543C00FBFD4FF4003004F05FFA95F860305BB977
:10544C00224B29461868012201F8602F603004F0C5
:10545C004BFC05F0D9F9A06605F03AFE05F0D4F93D
:10546C00174B586605F0D0F9154B17499A6E8B6D92
:10547C00821A002AB8BF52429A420BD391F860208C
:10548C00012A07D1114B1868002301F8603F6030E6
:10549C0004F02AFC0C4B93F86030012B03D14FF431
:1054AC00003004F029FA04F071F938B1084B18688F
:1054BC00044B1968024BDA6804F0F0F970BD00BFB8
:1054CC009C01002024090020D003002004000020AF
:1054DC002C09002008B5054A0346022093FBF0F086
:1054EC0080B282F8253006F013F808BDD0030020F6
:1054FC0010B5124B5B781BB1012B114B1BD111E07A
:10550C00104A01209178104A1468104A1070104A01
:10551C0011700133E21812F8011C0D4A082B995432
:10552C00F7D10AE009221A710622DA7158329A71FF
:10553C0002225A7101E003221A7010BD5803002098
:10554C00AC040020BC04002030000020C00300206C
:10555C00C4030020044B5A6840F2D2439A4202D151
:10556C00024B01221A707047580300207409002066
:10557C0010B51C4A1C4B116801EA03031B498B42F2
:10558C002ED152681A4B9A422AD102F077F9194B54
:10559C001B78012B10D103F0D1FF05F035F904462F
:1055AC0001E002F09FF905F02FF9001B0028B8BFAD
:1055BC004042B0F57A7FF4DB04F0D4F909F078FFBF
:1055CC00002009F0FDFB00210B480AF09DFD0A4864
:1055DC000AF0FAFC09480BF0A1FA002004F0CCF90F
:1055EC0010BD00BF5803002000FFFF000081920097
:1055FC00D6C5B4A3140000200800024000240140CA
:10560C0010B5164B9A78012A08D003D3022A144CF1
:10561C000FD109E0587802F0A1F902E0587802F0B5
:10562C001FFA0F4B586006E0587802F0A7F960603B
:10563C0001E0042323700B4B1B786BB1084B0A4918
:10564C005A680A4B0A601AB91A6842F0080202E05A
:10565C001A6822F008021A6010BD00BF580300201F
:10566C00AC04002090040020BC0300206003002048
:10567C0008B5104B9A78012A02D0022A16D10CE0F8
:10568C005A7842B9586810B904F06EF911E0104616
:10569C0004F06EF90DE0032209E05A68587812B94B
:1056AC0002F04CF905E002F051F902E00422024B41
:1056BC001A7008BD58030020AC04002008B50B4B31
:1056CC009A78022A0ED15B78372B09D89B000849AF
:1056DC0003F5E260C9180A30023204F083F904E0E1
:1056EC00032200E00422034B1A7008BD580300206B
:1056FC00E8040020AC040020144A00231360144A70
:10570C0010B51360134A1360134A1360134A1370D5
:10571C00134A002199500433B3F5806FF8D1114B23
:10572C001B7E63B940F21A740F49204609190422F2
:10573C0004F058F9043440F2FA739C42F4D1094A4B
:10574C000A4B527D02B101221A7010BD5804002080
:10575C00BC030020E404002060030020540300205C
:10576C00E8040020BC040020CEFDFF1F980400209C
:10577C0008B5124B9A7812B1022A1AD10AE05B785A
:10578C004E2B14D10E4B18680E4B0730D97904F000
:10579C004DFB11E05B78372B09D89B000A4903F5C8
:1057AC00E260C9180A30042204F09EFA04E00322D5
:1057BC0000E00422054B1A7008BD00BF58030020FE
:1057CC0098010020BC040020E8040020AC04002058
:1057DC0008B5604B9A781AB1022A40F0A68099E07D
:1057EC005B78502B69D01FD8462B51D00ED8422B4A
:1057FC0043D005D8402B37D0412B40F089803AE07C
:10580C00442B40D0544B554A40D83AE04B2B48D00F
:10581C0004D8472B3FD0492B7AD13FE04D2B46D0B3
:10582C0042D34E2B74D145E0812B5AD00ED8532B3A
:10583C004CD004D8512B43D0522B69D143E05A2B76
:10584C004AD0802B4BD0552B62D142E0842B53D0C5
:10585C0004D8822B4CD0832B5AD14BE0FE2B4ED04C
:10586C0050D8F02B54D14AE03D4B186804F008F99D
:10587C00394B58605CE0394B42E0384B5A78364B28
:10588C004FE012794DE0354BDA69F8E7527948E090
:10589C00324BDA68F3E7314B9A68F0E72F4BDA7D3D
:1058AC0032E02E4BDA78EAE72C4B9A78E7E72B4B71
:1058BC005A7DE4E7294BDA79E1E7284B9A7DDEE75C
:1058CC00264B1A7DDBE7254B1A6AD8E7234B1A695E
:1058DC00D5E7224B1A7ED2E7204B5A6ACFE7214BF1
:1058EC000EE0204B1A78042A14BF00220122C6E7CE
:1058FC001D4B02E01D4B00E01D4B1A68BFE71D4B12
:10590C001A78BCE71C4B1A78003A18BF0122B6E78C
:10591C0003220BE05A78104B372A04D8174951F858
:10592C0022205A6004E0032201E004220A4B1A7080
:10593C00134B1B786BB1084B12495A68124B0A6017
:10594C001AB91A6842F0080202E01A6822F008023A
:10595C001A6008BD58030020AC040020BC040020D1
:10596C000C00002098040020580400207C09002022
:10597C0078090020A404002088040020E8040020FA
:10598C0090040020BC0300206003002010B58A4B5B
:10599C009A781AB1022A40F0238104E15A784C2AF1
:1059AC0000F09E801ED8442A60D00CD8412A44D0E6
:1059BC0003D8402A40F012813BE0422A46D0432AC9
:1059CC0040F00C814AE0472A68D005D8452A55D0CA
:1059DC00462A40F0038159E0492A67D04B2A40F00F
:1059EC00FD8070E0532A00F0B38010D8502A00F0EC
:1059FC008B8005D84D2A7BD04E2A40F0EF807FE07B
:105A0C00512A00F08980522A40F0E88098E0832ADD
:105A1C0000F0BD8006D8552A00F0A2805A2A40F02A
:105A2C00DD80A9E0842A00F0B680FF2A40F0D68001
:105A3C00B6E01979614B186805E0614A1B7910686A
:105A4C00604A1946137004F0F1F9CCE05C4A1B79FA
:105A5C0010685C4A013019465370F4E7584A1B79B8
:105A6C001068584A043019461371ECE7544A5B68C5
:105A7C00106854491C3041F81C3F84E0504A1B7993
:105A8C001068504A053019465371DCE74C4A5B6884
:105A9C0010684C490C3041F80C3F74E0484A5B6884
:105AAC0010684849083041F8083F6CE01A79454BBA
:105ABC0012B1454901224A60DA75414B1868414BD5
:105ACC001730D97DBFE73E4A1B7910683D4C033037
:105ADC001946E37004F0AAF9E07803F0DBF882E0F1
:105AEC00374A1B791068374A023019469370AAE777
:105AFC00334A1B791068334A153019465375A2E79F
:105B0C001A79304BDA716EE02D4A1B7910682D4AE8
:105B1C0016301946937596E72A4A127D12F0010F3A
:105B2C0005D01B7913F0010F01D104F03BF8244A86
:105B3C00214B10681B79234A14301946137582E7E0
:105B4C001F4A5B6810681F49203041F8203F1AE05B
:105B5C001B4A5B6810681B49103041F8103F12E07B
:105B6C005A68012A3CD8164A1B7910681549183016
:105B7C0001F8183F012207E0114A5B6810681149CF
:105B8C00243041F8243F042204F0AEF82BE00E4BF5
:105B9C005A680E4B02E00C4B5A680D4B1A6022E00F
:105BAC001A790C4B1EE05A78372A17D859680A4BC9
:105BBC0043F8221017E000BF580300200C0000200F
:105BCC0098010020BC040020AC0400207C090020BB
:105BDC007809002088040020E8040020032200E05B
:105BEC000422014B1A7010BDAC04002008B5034B05
:105BFC00987808B9FEF7C6FE08BD00BF5803002010
:105C0C0008B5034B9A7812B95868FEF7BBFE08BD6D
:105C1C005803002008B5044B9A781AB958684042CA
:105C2C00FEF7B0FE08BD00BF5803002008B5AD4B11
:105C3C009A78002A41F07E805A78AC2A00F0EA84E7
:105C4C006BD81E2A00F0AE8230D8092A00F09E8153
:105C5C0013D8032A00F00A8105D8012A00F0DB8052
:105C6C0000F2E780C9E0062A00F02B81072A00F039
:105C7C006181042A41F05C80FEE0192A00F00F8259
:105C8C0008D80B2A00F0D981C0F0AB810D2A41F065
:105C9C004F80FEE11B2A00F04982C0F023821C2AAF
:105CAC0000F04A821D2A41F0438059E29B2A00F001
:105CBC002A8317D8922A00F0E58209D8852A00F0A9
:105CCC008B82862A00F0B3821F2A41F031807CE25D
:105CDC00972A00F00C83982A00F00F83962A41F043
:105CEC002780FEE2A22A00F0948309D89F2A00F0B4
:105CFC002983A12A00F058839C2A41F019801BE3C8
:105D0C00A42A00F00284C0F0CB83A52A00F02A84D8
:105D1C00A62A41F00D8000F053BCD32A00F0D185A7
:105D2C0031D8C22A00F0648515D8BE2A00F0288527
:105D3C000AD8B12A00F0BD84B22A00F0F884AD2A4A
:105D4C0040F0F68700F08DBCC02A00F0358500F2DB
:105D5C00418500F023BDC62A00F0828506D8C42AEE
:105D6C0000F0628500F26E8500F050BDC82A00F08C
:105D7C009385C0F08385C92A00F09585D22A40F01E
:105D8C00D78700F097BDF12A00F0478619D8E52A8D
:105D9C0000F0B4850AD8E22A00F0A285E42A00F0CB
:105DAC00A685D42A40F0C48700F092BDEA2A00F000
:105DBC00D485EB2A00F00986E62A40F0B98700F07A
:105DCC00A4BDFA2A00F0CD860AD8F52A00F07A860E
:105DDC00F92A00F09D86F42A40F0AA8700F048BE0C
:105DEC00FC2A00F02A87C0F0E686FD2A00F04E87D8
:105DFC00FE2A40F09D8700F072BF052805D1394B73
:105E0C005868FEF7F5FC00F0ACBF062840F0A987F7
:105E1C00FEF706FB26E0052805D1324B5868FEF745
:105E2C008DFD00F09EBF062840F09B87FEF706FB19
:105E3C0018E0052811D12B4B2B4A586800F542333A
:105E4C0003F5A863934203D8FEF79CFD00F089BFCD
:105E5C00264B04221A7000F084BF062840F081877C
:105E6C00FEF7F2FA214B586000F069BF062840F0AB
:105E7C007887FEF7EFFAF5E705280AD1194B1C498C
:105E8C005B688B4295BF1B4A184B13601A7000F06D
:105E9C0068BF062802D1174B1A686AE2072806D198
:105EAC00154B1449186803F01FFF00F05ABF08285F
:105EBC0040F05787104B0F49186803F093FD00F022
:105ECC0050BF05281AD1074B43F698225B689342C2
:105EDC0003D8084A536000F044BF044B04221A70E4
:105EEC0000F03FBF58030020801A0600AC040020CD
:105EFC00400D0300D003002004000020062802D12E
:105F0C009B4B5A6835E2072808D19A4B0422186833
:105F1C009949801803F0E8FE00F023BF082840F0F0
:105F2C002087944B042218689349801803F05AFD7B
:105F3C0000F017BF05280DD1904B914A5B68934236
:105F4C0003D88B4A936000F00CBF8E4B04221A705E
:105F5C0000F007BF062802D1854B9A6809E2072892
:105F6C0008D1844B884918680422083003F0BCFE21
:105F7C0000F0F7BE082840F0F4867E4B8249186882
:105F8C000422083003F02EFD00F0EBBE05280CD1E6
:105F9C005B687B4A934203D8754A136100F0E1BEFB
:105FAC00784B04221A7000F0DCBE062802D1704B2C
:105FBC001A69DEE1072808D16E4B7449186804226F
:105FCC00103003F091FE00F0CCBE082840F0C986DA
:105FDC00684B6E4918680422103003F003FD00F082
:105FEC00C0BE05280DD1654B694A5B68934203D846
:105FFC005F4AD36000F0B5BE624B04221A7000F009
:10600C00B0BE062802D15A4BDA68B2E1072808D193
:10601C00584B6049186804220C3003F065FE00F000
:10602C00A0BE082840F09D86524B5A49186804229D
:10603C000C3003F0D7FC00F094BE05280DD14F4B6B
:10604C00534A5B68934203D8494A536100F089BEB6
:10605C004C4B04221A7000F084BE062802D1444B2B
:10606C005A6986E1072808D1424B4B49186804222B
:10607C00143003F039FE00F074BE082840F071862D
:10608C003C4B454918680422143003F0ABFC00F07B
:10609C0068BE062840F06586FEF7C8F9E2E60528DA
:1060AC0004D15A68324B9A6500F05BBE062802D1C7
:1060BC002F4B9A6D5DE1072808D12E4B3749186894
:1060CC000422583003F010FE00F04BBE082840F0BC
:1060DC004886284B314918680422583003F082FC5A
:1060EC0000F03FBE052805D1244B5A68204B5A6559
:1060FC0000F037BE062802D11D4B5A6D39E1072836
:10610C0008D11C4B264918680422543003F0ECFDCE
:10611C0000F027BE082840F02486164B204918684A
:10612C000422543003F05EFC00F01BBE062840F045
:10613C00188604F0BBFF95E6052805D10F4B58686F
:10614C0004F0C0FF00F00DBE062802D104F0B4FF2D
:10615C0088E6072840F0058604F0BAFF00F001BE7F
:10616C00052840F0EA85FEF7F1F900F0FABD00BF12
:10617C00D003002004000020D4030020580300208A
:10618C00400D0300AC040020D8030020E0030020E5
:10619C00A0860100DC030020E4030020280400207A
:1061AC0024040020052804D1586804F0BBFF00F03B
:1061BC00D8BD062802D104F0AFFF53E6072840F003
:1061CC00D08504F0B5FF00F0CCBD052840F0B585B6
:1061DC00FEF7B2FC00F0C5BD05280CD1A14B5B68E5
:1061EC000A2B03D8A04A936100F0BBBD9F4B04223D
:1061FC001A7000F0B6BD062802D19B4B9A69B8E024
:10620C00072808D19A4B9B4918680422183003F0D0
:10621C006BFD00F0A6BD082840F0A385944B954972
:10622C0018680422183003F0DDFB00F09ABD052835
:10623C000CD18C4B5B680A2B03D88B4AD36100F0D2
:10624C0090BD8A4B04221A7000F08BBD062802D137
:10625C00854BDA698DE0072808D1854B864918688B
:10626C0004221C3003F040FD00F07BBD082840F0F8
:10627C0078857F4B8049186804221C3003F0B2FBF0
:10628C0000F06FBD05280ED15B68012B06D8754B4D
:10629C001A79754B83F8202000F063BD734B0422F0
:1062AC001A7000F05EBD062804D16F4B93F82020C5
:1062BC0000F025BD072808D16D4B704918680122E4
:1062CC00203003F011FD00F04CBD082840F049854A
:1062DC00674B6A4918680122203003F083FB00F0F9
:1062EC0040BD062840F03D85FEF7BAF8BAE5062811
:1062FC0040F03785FEF782F8B4E5062840F031858A
:10630C00FEF782F8AEE5052810D1586847F23052F6
:10631C0000F56A531833934203D8FEF753FA00F092
:10632C0020BD524B04221A7000F01BBD062840F011
:10633C001885FEF76FF895E5062840F0128503F0F6
:10634C00FBFA8FE505280FD1464B5B689A1F022A92
:10635C0000D923B9444A82F8213000F002BD434BE6
:10636C0004221A7000F0FDBC062806D13E4B93F8AF
:10637C0021203E4B5A6000F0E2BC072808D13C4B70
:10638C003F4918680122213003F0AEFC00F0E9BC53
:10639C00082840F0E684364B394918680122213030
:1063AC0003F020FB00F0DDBC052813D12D4A2E4B49
:1063BC0052683AB193F8512042F0010283F851200F
:1063CC0000F0CFBC93F8512022F0010283F8512049
:1063DC0000F0C7BC062805D1234B93F8512002F0DE
:1063EC000102C6E7072808D1214B2649186801226B
:1063FC00513003F079FC00F0B4BC082840F0B184B3
:10640C001B4B204918680122513003F0EBFA00F0C5
:10641C00A8BC052812D15A68134B3AB193F85120F5
:10642C0042F0020283F8512000F09BBC93F85120FB
:10643C0022F0020283F8512000F093BC062805D10B
:10644C00094B93F85120C2F3400292E707281BD165
:10645C00074B0C4918680122513003F045FC00F041
:10646C0080BC00BF58030020D0030020AC040020E7
:10647C0004000020E8030020EC030020F0030020BF
:10648C00F103002021040020082840F06A84934B7B
:10649C00934918680122513003F0A4FA00F061BC52
:1064AC00052813D18F4A904B52683AB193F851207A
:1064BC0042F0040283F8512000F053BC93F85120B1
:1064CC0022F0040283F8512000F04BBC062805D1C1
:1064DC00854B93F85120C2F380024AE7072808D174
:1064EC007E4B7F4918680122513003F0FDFB00F010
:1064FC0038BC082840F03584784B7949186801225B
:10650C00513003F06FFA00F02CBC05280ED1754BFE
:10651C005A68032A05D81A79734B83F8222000F0A5
:10652C0020BC724B04221A7000F01BBC062803D14D
:10653C006D4B93F822201CE7072808D1674B6C4958
:10654C0018680122223003F0CFFB00F00ABC0828A7
:10655C0040F00784614B664918680122223003F031
:10656C0041FAFEE3052810D15E4B5B68B3F5803F22
:10657C0007D25D4A9BB21846A2F8403005F020F8CD
:10658C00EFE35A4B04221A70EBE3062803D1564B67
:10659C00B3F84020EDE6072807D1504B5549186851
:1065AC000222403003F0A0FBDBE3082840F0D98343
:1065BC004A4B504918680222403003F013FAD0E3DA
:1065CC0005280CD1474B5A68032A04D81A79464B34
:1065DC0083F82320C5E3454B04221A70C1E3062837
:1065EC0003D1414B93F82320C3E6072807D13B4B3B
:1065FC00414918680122233003F076FBB1E30828E7
:10660C0040F0AF83354B3C4918680122233003F02E
:10661C00E9F9A6E305280AD15B68B3F5803F02D2FD
:10662C00314A13639DE3314B04221A7099E3062817
:10663C0002D12D4B1A6B9CE6072807D1274B2F490B
:10664C0018680422303003F04FFB8AE3082840F02E
:10665C008883224B294918680422303003F0C2F990
:10666C007FE305280BD11F4B5B68B3F5803F02D24B
:10667C001D4A536375E31D4B04221A7071E30628FF
:10668C0002D1194B5A6B74E6072807D1134B1C49DE
:10669C0018680422343003F027FB62E3082840F02A
:1066AC0060830E4B164918680422343003F09AF9B3
:1066BC0057E305280CD10B4B43F698225B689342A9
:1066CC0002D8094A93634CE3084B04221A7048E33E
:1066DC00062817D1044B9A6B4BE600BF0400002030
:1066EC002104002058030020D0030020AC0400201B
:1066FC00F203002010040020F3030020000400200B
:10670C0004040020072807D1A24BA34918680422CF
:10671C00383003F0E9FA24E3082840F022839D4B3B
:10672C009D4918680422383003F05CF919E30528F8
:10673C000BD19A4B5B68012B03D8994A82F86130D4
:10674C000FE3984B04221A700BE3062803D1944BE9
:10675C0093F861200DE6072807D18E4B92491868F3
:10676C000122613003F0C0FAFBE2082840F0F98204
:10677C00884B8D4918680122613003F033F9F0E23F
:10678C00052804D1874B586802F09EFFE9E20628E1
:10679C0040F0E78202F05CFFFFF764BB052804D1F0
:1067AC00804B586802F096FFDBE2062840F0D98255
:1067BC0002F054FFFFF756BB052804D1794B5868FB
:1067CC0002F08EFFCDE2062840F0CB8202F04CFFA7
:1067DC00FFF748BB052804D1724B586802F086FFBE
:1067EC00BFE2062840F0BD8202F044FFFFF73ABB3F
:1067FC00052804D16B4B586802F07EFFB1E20628E5
:10680C0040F0AF8202F03CFFFFF72CBB052804D10F
:10681C00644B586802F076FFA3E2062840F0A18290
:10682C0002F034FFFFF71EBB052804D15D4B5868FE
:10683C0002F06EFF95E2062840F0938202F02CFFE6
:10684C00FFF710BB052804D1564B586802F066FFC1
:10685C0087E2062840F0858202F024FFFFF702BB96
:10686C00052804D14F4B586802F05EFF79E20628E8
:10687C0040F0778202F01CFFFFF7F4BA052804D130
:10688C00484B586802F056FF6BE2062840F06982CC
:10689C0002F014FFFFF7E6BA062840F06282FDF71B
:1068AC0029FEFFF7DFBA062840F05B82FDF728FED1
:1068BC00FFF7D8BA062840F05482FDF73DFEFFF7EB
:1068CC00D1BA062840F04D82FDF732FEFFF7CABA66
:1068DC00062840F0468201F08BFD00B2FFF7C2BAE9
:1068EC00062840F03E82FDF7F3FDFFF7BBBA062801
:1068FC0040F03782FDF7F2FDFFF7B4BA062840F0FE
:10690C003082FDF7F1FDFFF7ADBA05280BD1234B13
:10691C005B68B3F5803F02D2214A536421E2214BDC
:10692C0004221A701DE2062802D11D4B5A6C20E578
:10693C00072807D1174B1D4918680422443003F06F
:10694C00D3F90EE2082840F00C82124B1749186854
:10695C000422443003F046F803E205280BD10F4B18
:10696C005B68B3F5803F02D20D4A9364F9E10D4B9D
:10697C0004221A70F5E1062802D1094B9A6CF8E44E
:10698C00072817D1034B0A4918680422483003F032
:10699C00ABF9E6E1040000200804002058030020B5
:1069AC00D0030020AC04002031040020140400208B
:1069BC0018040020082840F0D4818D4B8D491868AC
:1069CC000422483003F00EF8CBE105280BD18A4B9A
:1069DC005B68B3F5803F02D2884AD364C1E1884B2F
:1069EC0004221A70BDE1062802D1844BDA6CC0E493
:1069FC00072807D17E4B8349186804224C3003F0DA
:106A0C0073F9AEE1082840F0AC81794B7D491868E8
:106A1C0004224C3002F0E6FFA3E105280ED15A689F
:106A2C00794902F5423303F5A8638B4202D8734BC4
:106A3C00DA6596E1724B04221A7092E1062802D1B3
:106A4C006E4BDA6D95E4072807D1694B6F491868CE
:106A5C0004225C3003F048F983E1082840F081817E
:106A6C00634B6A49186804225C3002F0BBFF78E182
:106A7C0005280CD1604B42F210725B68934202D82D
:106A8C005E4AD3846DE15E4B04221A7069E10628DC
:106A9C0003D15A4BB3F926206BE4072807D1544B8A
:106AAC005B4918680222263003F01EF959E10828C8
:106ABC0040F057814E4B564918680222263002F09E
:106ACC0091FF4EE1052808D14B4B5A684B4B003ACD
:106ADC0018BF012283F82B2043E1062803D1474B32
:106AEC0093F82B200BE1072807D1414B4949186833
:106AFC0001222B3003F0F8F833E1082840F0318103
:106B0C003B4B4449186801222B3002F06BFF28E103
:106B1C0005280BD1384B5B68022B03D8374A82F817
:106B2C002A301EE1364B04221A701AE1062803D1D2
:106B3C00324B93F82A201CE4072807D12C4B3649FA
:106B4C00186801222A3003F0CFF80AE1082840F037
:106B5C000881274B3049186801222A3002F042FF85
:106B6C00FFE005280CD15B68B3F5803F04D2234AC3
:106B7C00D363FDF7E1FFF4E0214B04221A70F0E03F
:106B8C00062803D11D4BDA6BFFF7F3BB072807D19F
:106B9C00174B2249186804223C3003F0A5F8E0E0BA
:106BAC00082840F0DE80124B1C49186804223C3047
:106BBC0002F018FFD5E005280AD10F4B5A680F4B8D
:106BCC00003A18BF012283F82C20FDF7B5FFC8E06E
:106BDC00062803D1094B93F82C2090E0072821D1EB
:106BEC00034B0F49186801222C3003F07DF8B8E0F4
:106BFC00040000201804002058030020D0030020BB
:106C0C00AC0400201C040020801A06002C04002078
:106C1C00F6030020FB030020FA0300200C040020E4
:106C2C00FC030020082840F09C804E4B4E4918680D
:106C3C0001222C3002F0D6FE93E005280BD14B4BF1
:106C4C005B68012B03D84A4A82F82D3089E0494B06
:106C5C0004221A7085E0062804D1454B93F82D20A8
:106C6C00FFF787BB072807D13E4B43491868012221
:106C7C002D3003F039F874E0082872D1394B3E49B5
:106C8C00186801222D3002F0ADFE6AE005280BD108
:106C9C00364B5868831EFC2B02D8FEF71BFC60E0B9
:106CAC00344B04221A705CE0062804D1304B93F864
:106CBC002520FFF75EBB072807D12A4B2F49186800
:106CCC000122253003F010F84BE0082849D1254B60
:106CDC002A4918680122253002F084FE41E005287B
:106CEC0008D1224B5A68224B003A18BF012283F874
:106CFC00242036E0062807D11D4B93F82420003AB7
:106D0C0018BF0122FFF735BB072807D1154B1C49CB
:106D1C0018680122243002F0E7FF22E0082820D175
:106D2C00104B174918680122243002F05BFE18E062
:106D3C00032200E004220F4B1A70062811D1114BCC
:106D4C001B7873B10B4B10495A68104B0A6022B96F
:106D5C001A6842F008021A6003E01A6822F008026E
:106D6C001A6008BD04000020FC030020580300201A
:106D7C00D0030020AC040020FD030020F50300200C
:106D8C00F403002090040020BC03002060030020CA
:106D9C0010B5274B997821B15B78032B01D0042BCC
:106DAC0041D1234B5B780A2B3BD8DFE803F0060973
:106DBC000C0F141A1D282D30350002F035FD2DE076
:106DCC0002F02EFD2AE002F033FD27E0184B586844
:106DDC0002F030FD22E0164B0846596802F0B0FC78
:106DEC0024E002F0C5FC21E002F0CAFC044602F0EB
:106DFC00CDFC104B40EA0404E4B25C6016E00C4B92
:106E0C00586802F027FD11E002F036FD06E0084B51
:106E1C00586802F037FD09E002F03AFD054B586066
:106E2C0004E0032200E00422024B1A7010BD00BFE4
:106E3C0058030020AC04002008B50B4B9A7872B9AB
:106E4C005A7812B1012A08D103E05868FDF7D0FC3A
:106E5C0008E05868FDF7FCFC04E0032200E0042283
:106E6C00024B1A7008BD00BF58030020AC04002070
:106E7C0010B5A94AA94B107851686422232859608F
:106E8C001A70587000F0F68053D8132800F0CB809D
:106E9C0028D8082811D8052880F0B080022800F0E6
:106EAC00A48003D8012840F049819BE0032800F01E
:106EBC009F80042840F042819DE00B2800F0A780C1
:106ECC0006D8092800F09D800A2840F037819BE005
:106EDC000E2800F0A2800F2800F0A2800C2840F0B1
:106EEC002D8197E01B2800F0B08011D8162800F0F7
:106EFC00A38006D8142800F09980152840F01E8134
:106F0C0097E0172800F09B80182840F0178199E033
:106F1C001F2800F0A38006D81C2800F099801E289A
:106F2C0040F00C8197E0212800F09E8000F29F80B9
:106F3C0097E0822800F0C58029D8432800F0AC8067
:106F4C0011D8402800F09F8006D8242800F09580A6
:106F5C00272840F0F38093E0412800F097804228E6
:106F6C0040F0EC8095E0462800F09F8006D844283D
:106F7C0000F09580452840F0E18093E0802800F0F7
:106F8C009A8000F29B80472840F0D88090E08828B7
:106F9C0000F0B68011D8852800F0A48006D883288C
:106FAC0000F09280842840F0C98090E0862800F0A0
:106FBC00A180872840F0C280A5E08D2800F0B28027
:106FCC0006D8892800F0A2808C2840F0B780A0E079
:106FDC00F22800F0AD80FF2800F0AD808E2840F044
:106FEC00AD80A2E0FEF70CFEABE0FEF713FEA8E0CE
:106FFC00FEF7FCFDA5E0FFF71FFFA2E0FEF716FE73
:10700C009FE0FEF7C3FC9CE0FEF7E2FB99E0FEF785
:10701C00AFFB96E0FEF752FB93E0FEF729FB90E006
:10702C00FEF7EEFA8DE003F065F88AE003F040F924
:10703C0087E003F0CBF984E003F0BEF981E003F0C4
:10704C001FFA7EE003F034FA7BE003F0ABFA78E051
:10705C0003F040FA75E003F043FA72E003F058FADB
:10706C006FE003F085FA6CE003F098F869E003F048
:10707C00BDFB66E003F0AEFB63E003F0EDF860E00F
:10708C0002F092FF5DE000F059FB5AE000F058FB73
:10709C0057E000F057FB54E000F056FB51E000F0D5
:1070AC0055FB4EE000F054FB4BE000F053FB48E086
:1070BC0000F052FB45E002F0C7FF42E002F08EFF09
:1070CC003FE002F09DFF3CE002F0A0FF39E000F051
:1070DC00D5FB134B1C7D02F02FFC0146204603F020
:1070EC0013F92EE003F02CF900F0C0FB0020FDF7A3
:1070FC0069FB26E00A4B197D987803F009FB20E028
:10710C00FEF7F6F91DE003F021F91AE003F046FB57
:10711C0017E003F0D1FA14E058030020AC0400206F
:10712C00BC04002002F096FF0BE0FFF731FE08E0F4
:10713C00FEF71EFA05E0FEF70DFA02E0014B022203
:10714C001A7010BDAC0400202DE9F04F764B8BB0BB
:10715C001B78044663B1754B1B78062B08D00A2BA1
:10716C0006D00F2B04D01F2B02D0714B00221A70AB
:10717C00704B1B78012B48D16D4B1A78511EC9B23C
:10718C00012942D858786C496C4BCD681B78012A80
:10719C000CBF4FF0070C4FF0080C002201958DF836
:1071AC0000C08DF801008DF80220D3B9644A8E68B6
:1071BC001578117992F801E092F807C0907952791C
:1071CC008DF808608DF809508DF80AE08DF80BC029
:1071DC008DF80C008DF80D208DF80E108DF80F30F9
:1071EC000DE0012B09D1574B0132D15C0AA8831851
:1071FC00082A03F8211CF6D101E0022B05D06846C1
:10720C0004F072FD002800F039824F4B1B78012BE3
:10721C004CD1474A1278032A20D1484B1B7893B99A
:10722C00454E474DB07877782A786B78C719BF18D8
:10723C00EA79FF18AB79BF186A79FF182B79BF1858
:10724C00FF18FFB218E0012B30D100253D4BE85C54
:10725C00013501F02FFD092DF8D127E0042A25D1A5
:10726C00354E374DB27877781046D7190137002252
:10727C002B706A60FFB26A7001F01CFD707801F02F
:10728C0019FD287801F016FD687801F013FDE879F6
:10729C0001F010FDA87901F00DFD687901F00AFDEF
:1072AC00287901F007FD384601F004FD274B1B78C7
:1072BC00012B73D11E4A1278072A49D11F4B1B7818
:1072CC002BBB1D4A1E4B5578967893F800E093F82B
:1072DC0001C0AF19D8797744997967445A79C7199D
:1072EC001B79CF19D719DF198DF818708DF810602C
:1072FC008DF811508DF812E08DF813C08DF8140034
:10730C008DF815108DF816208DF8173009E0012B2B
:10731C0007D1013B0B4A995C04AAD1540133092BC8
:10732C00F8D104A8092137E0880400205803002074
:10733C000C0200204D000020BC040020C0030020E3
:10734C00AC040020C40300204A00002014000020DC
:10735C00082A23D19849994A91F801C091F802E082
:10736C0000250EEB0C06013604A8092155608DF89A
:10737C0012308DF813502F468DF814508DF815508F
:10738C008DF816508DF817508DF8186055701370D5
:10739C008DF810E08DF811C001F0BAFF884B8949C7
:1073AC001A7800230B7088490B7012B1012002F07F
:1073BC00E3FA864B1D78012D3CD1684604F014FC91
:1073CC00002837D09DF80010814B9DF808A09DF83F
:1073DC0009809DF80A709DF80B609DF80CC09DF813
:1073EC000D009DF80E90784A9DF801B0072983F89E
:1073FC00049083F800A083F801809F70DE7183F8FD
:10740C0006C0587182F801B001D1157001E0022359
:10741C001370704B1B785A1ED2B2012A05D9052B5A
:10742C0003D06D4B01251D7005E06B4B00221A70CB
:10743C00012500E00025694B1B78012B59D10DF17A
:10744C00270001F011FC002853D001F029FC10B1E9
:10745C005D4B00229A705C4B9DF8270099784A1C72
:10746C00D2B2C918092A08719A7041D1524A1879B6
:10747C005178002288429A703AD11346524D291DF8
:10748C00895C01325B18082ADBB2F7D12A7B9A425D
:10749C002CD14F4B697AAA7AEE7A6F7995F806E07F
:1074AC0095F807C0287A1E7199715A711F7083F86C
:1074BC0001E083F802C0D87103F0A6F9454B484EA1
:1074CC001B783060591E47480022C9B2AA7002705E
:1074DC00033201292A7005D9052B03D03E4B012517
:1074EC001D7006E03C4B00221A7001E004232B7047
:1074FC0001253D4B1B78012B43D107A801F0F0FE71
:10750C0000283ED00022134607A9C95C013352184B
:10751C00082BD2B2F8D19DF824102B4C91422ED1CD
:10752C002B4B9DF821109DF822209DF81D609DF895
:10753C001EE09DF81FC09DF820009DF82350997106
:10754C005A711E701D7183F801E083F802C0D87166
:10755C0003F05AF91F4B22491B7808605A1E214927
:10756C000020D2B208700721012A217003D9052B03
:10757C0001D0012200E00022174B1A7039E0237071
:10758C0037E0002D35D113490B78013BDBB2012BD1
:10759C002FD8012C2DD1154B1A68B2F5006F27D8B6
:1075AC00104601321A600A4902F048FB064B0922C8
:1075BC001A70094B1C701CE0BC040020AC040020A9
:1075CC0074090020C00300200C0200204D00002094
:1075DC005803002098040020900400204A0000204A
:1075EC00A8040020B404002014000020580400203B
:1075FC000D70244B1B78042B04D1234B93F90030D2
:10760C00002B2EDA214B1B783BB1042B05D0082B19
:10761C0003D0062B01D0FFF72BFC1C4B1B78092B3E
:10762C0005D1184A1178022901D103311170184A79
:10763C0012681AB3092B21D1124B1B78012B1DD1C7
:10764C001449013B096809E0134850F82300013341
:10765C00814203D10B4B05221A700FE09342F3D3F6
:10766C000CE0FDF7FFF8094B1B783BB1042B05D060
:10767C00082B03D0062B01D002F0F4FF0BB0BDE8B1
:10768C00F08F00BF98040020580300200C0200204B
:10769C009C040020580400205C04002073B5204B8F
:1076AC00024640781F4D1870907800265870D0789C
:1076BC00EC46987010790C46D8715079987192F804
:1076CC0006E095E8030083F805E0D2798CE8030026
:1076DC001A71154B1E70FFF7CBFB144B1B7873B94B
:1076EC00637023702B78A3706B78E370EB79237144
:1076FC00AB7963716B79A3712B79E37108E0012B82
:10770C0006D10B4B9B195B78A3550136082EF8D18B
:10771C00044B6A4692E8030083E803007CBD00BF7B
:10772C0058030020AC04002090040020C00300206B
:10773C00C4030020704700BF704700BF704700BFF4
:10774C00704700BF704700BF704700BF704700BF55
:10775C00704700BF704700BF704700BF0E4B10B59D
:10776C000022012002214FF4FA744FF0080C5C62E5
:10777C0083F805C09860D9601A621A7058709970B5
:10778C00DA701A719A711A611A755A759A75DA75D6
:10779C001A76DA6110BD00BFBC0400202B4B4FF4ED
:1077AC00FA6CC3F814C04FF0020CC3F81CC00CF1F7
:1077BC00040CF0B583F821C00CF1020C83F825C041
:1077CC000CF1C00CC3F85CC040F2DC5CC3F838C0F0
:1077DC00DFF87CC04FF47A66002101204FF4FA7474
:1077EC004FF496750527DE63C3F854C01E605E60C7
:1077FC0043F2903C4FF47A761F61A3F840105D641D
:10780C00DC6483F85000C3F858C09C60DF6098615A
:10781C0083F8200083F8221083F8231083F82410B7
:10782C00DE84198583F82A0083F82B0083F82C104A
:10783C001D635D6383F842109C6483F8511083F8D8
:10784C00601083F82D1083F86110F0BDD003002078
:10785C0000390300014B10225A61704700080140A7
:10786C00014B10221A61704700080140024B4FF483
:10787C0000421A61704700BF00100140024B4FF4E8
:10788C0000425A61704700BF00100140024B9868DB
:10789C0000F40040704700BF00100140024B4FF451
:1078AC0080521A61704700BF00100140024B4FF428
:1078BC0080525A61704700BF00100140704700BFF2
:1078CC00704700BF704700BF704700BF704700BFD4
:1078DC00704700BF704700BF704700BF704700BFC4
:1078EC00704700BF704700BF014B04221A617047FC
:1078FC0000080140014B04225A6170470008014006
:10790C00054B9A6812F0040F02D004225A6101E070
:10791C0004221A61704700BF00080140024B4FF46B
:10792C0000721A61704700BF000C0140024B4FF40B
:10793C0000725A61704700BF000C014010B9024B35
:10794C0020225A61704700BF0010014010B9024B51
:10795C0020221A61704700BF0010014018B10128A5
:10796C0003D0002005E0034B00E0034B9868C0F304
:10797C008000704700140140000C014008B1002049
:10798C0003E0024B9868C0F34010704700100140B0
:10799C00064B1B78012B04D1054B4FF480521A6116
:1079AC0002E0044B01221A70704700BF1400002043
:1079BC00000C01401C020020064B1B78012B04D14B
:1079CC00054B4FF480525A6102E0044B00221A70AE
:1079DC00704700BF14000020000C01401C02002066
:1079EC00054B1B78012B03D1044B0020DB6801E015
:1079FC00034B1878704700BF14000020000C0140A6
:107A0C001C020020704700BF38B5084B40F2FF74D1
:107A1C00074D5868214600F0E5F96868214600F0EA
:107A2C00E1F9A868214600F0DDF938BD1C02002000
:107A3C0014000020094B10B59C68C4F382140CB1DF
:107A4C00072C05D1012803D11F3001F055FF02E0AE
:107A5C00202001F059FF204610BD00BF000C014052
:107A6C0008B5062805D8DFE800F006090C0E11143D
:107A7C001700002014E00B4BD8680FE0094B186975
:107A8C000CE0094B00E0074B586807E0054B986881
:107A9C0004E0044B586901E0024B986900F09AF934
:107AAC0008BD00BF140000201C02002037B501AD3A
:107ABC00002429464FF01F030848ADF804308DF818
:107ACC00074008F0AFF84FF00303294604488DF83F
:107ADC000740ADF8043008F0A5F83EBD0010014099
:107AEC00000C01402DE9F347584E01AD0420012153
:107AFC00032407F04BFC102730464FF0BE032946F9
:107B0C00ADF804308DF806408DF8077008F08AF84F
:107B1C00AE234FF00408DFF83CA13046376129460C
:107B2C0073614FF04103ADF804308DF806408DF8C9
:107B3C00078008F077F80820012107F027FC41F2B4
:107B4C00386350462946ADF804304FF020098DF8C3
:107B5C0006408DF8077008F065F841F2182350467E
:107B6C002946CAF81090CAF8143040F6C71306F527
:107B7C000066ADF804308DF806408DF8078008F0EB
:107B8C0051F83846012107F001FC30464FF22043F2
:107B9C002946ADF804308DF807708DF8064008F0D2
:107BAC0041F84FF4E043336103F5A1533046736160
:107BBC0029464FF43C63ADF804308DF806408DF83F
:107BCC00078008F02FF84FF01F0330462946002697
:107BDC00ADF804308DF806408DF8076008F022F8F7
:107BEC004846012107F0D2FB4FF40040314608F023
:107BFC00A9F84823164829468DF80730ADF80480BB
:107C0C008DF8064008F00EF83046334611494FF413
:107C1C0080644C610A468968013611F4006F4FF498
:107C2C0080611161926808BF013312F4006F18BFB4
:107C3C0001300A2EEAD10A2B01D0002003E00A28D9
:107C4C0014BF00200120BDE8FC8700BF00080140E4
:107C5C0000140140000C0140704700BFFEE700BF5C
:107C6C00FEE700BFFEE700BFFEE700BF704700BFA6
:107C7C00704700BF704700BF704700BF704700BF20
:107C8C00704700BF704700BF704700BF704700BF10
:107C9C00704700BF704700BF704700BF704700BF00
:107CAC00704700BF704700BF704700BF704700BFF0
:107CBC00704700BF704700BF704700BF704700BFE0
:107CCC0008B5024B1B68984708BD00BF6403002031
:107CDC0008B5024B1B68984708BD00BFB8040020CC
:107CEC00684620F00701044B8D4601B51B68984788
:107CFC00BDE80140854670478C04002008B5024B56
:107D0C001B68984708BD00BF94040020704700BF53
:107D1C00704700BF704700BF704700BF704700BF7F
:107D2C00704700BF704700BF704700BF704700BF6F
:107D3C00704700BF704700BF704700BF704700BF5F
:107D4C00704700BF704700BF704700BF704700BF4F
:107D5C00704700BF704700BF704700BF704700BF3F
:107D6C00704700BF704700BF704700BF704700BF2F
:107D7C00704700BF704700BF704700BF704700BF1F
:107D8C00704700BF684620F007018D4601B50023FF
:107D9C0003E00B495958995004330A4A0A49981878
:107DAC008842F6D3094B02E0002243F8042B084A20
:107DBC009342F9D3FCF72AFABDE801408546704797
:107DCC00781701080000002098010020980100207D
:107DDC00B02C0020024B33F8100080B2704700BF6B
:107DEC0030020020024B03EB40031982704700BFA6
:107DFC0030020020024B03EB4003188A704700BF8F
:107E0C003002002010B50A4C24781CB9002914BF8C
:107E1C000A461A4650214843064B424302991878A9
:107E2C00039B002808BF0B4692FBF3F010BD00BF6C
:107E3C008009002082090020A5234343044AA3F5AE
:107E4C00A52310684FF48052584390FBF2F0704712
:107E5C0054000020014B1870704700BF82090020AD
:107E6C00014B1870704700BF80090020074B10B5FC
:107E7C001B68074C34F8130080B2FFF7DDFF20229B
:107E8C000146206A04F0F2FD206210BD1C000020A7
:107E9C0030020020F8B5114B114E1B68044636F821
:107EAC00130080B2FFF7C8FF0E4B05461B6836F86F
:107EBC00130080B2FFF7C0FF064605FB05F006FB7A
:107ECC00060077197F4207FB070004F035FDA680FA
:107EDC00A060678025802046F8BD00BF20020020EE
:107EEC00300200201C000020F8B5114B114E1B680D
:107EFC00044636F8130080B2FFF79EFF0E4B054682
:107F0C001B6836F8130080B2FFF796FF064605FB98
:107F1C0005F006FB060077197F4207FB070004F00B
:107F2C000BFDA780A060668025802046F8BD00BFB1
:107F3C0020020020300200201800002038B5104C20
:107F4C00257885B1012D1AD10E4B5B6A002BB8BF79
:107F5C005B42B3F5E16F12DDFFF7A8FC0023237041
:107F6C00094B1D700BE0074B5B6AC733B3F5C77F3A
:107F7C0005D8FFF793FC044A01231370237038BD16
:107F8C008209002030020020810900202DE9F74FE2
:107F9C00534C0025074665625248884692469946DE
:107FAC00DDF834B006F052FDC8F5E168404501D368
:107FBC0007241EE04C4B626A1B68002A34F813003D
:107FCC0004EB43010B8A80B2B8BF5242C01A80EA5C
:107FDC00E073A3EBE07393420E9BC8BF6062514603
:107FEC000193CDF800B04A460C9BFFF70BFF06241B
:107FFC0005463C4806F02EFD404501D3002621E005
:10800C003A4A374B1268596A33F8120003EB4206AE
:10801C00328A80B2801A81EAE172A2EBE17280EAC4
:10802C00E071A1EBE0719142C8BF58620E9BCDF894
:10803C0000B0019351464A460C9BFFF7E3FE24F037
:10804C0002040646274806F009FD404502D34FF0CE
:10805C00000822E0264A224B1268596A33F81200B3
:10806C0003EB420CBCF8102080B2801A81EAE1725A
:10807C00A2EBE17280EAE071A1EBE0719142C8BF22
:10808C0058620E9BCDF800B0019351464A460C9BAA
:10809C00FFF7B8FE24F004048046022C07D0042C11
:1080AC0009D0012C0BD108EB06056D4207E008EB5B
:1080BC000506764203E006EB0508C8F1000805FB4F
:1080CC0005F006FB060008FB080004F035FCA7F8D9
:1080DC000480B8607E803D803846BDE8FE8F00BFCE
:1080EC0030020020002C014020020020180000204B
:1080FC001C00002070B590B0FFF7D8FC01200146A1
:10810C0007F036F901214FF4007007F03FF94148B0
:10811C0007F05AFF404B00240093404B0726019375
:10812C0080230593DB18069303F540730793A3F59F
:10813C00787338486946089303F5FF530993029402
:10814C00039604940A9407F0AFFF0121314807F01D
:10815C00DBFF01254FF4602331480BA90D930B94E1
:10816C008DF830508DF831400E948DF83C6008F04D
:10817C0033FB2C4B2A4819782A46032308F0AEFB14
:10818C00294B022219782648032308F0A7FB274B1A
:10819C00032219782248134608F0A0FB244B042232
:1081AC0019781F48032308F099FB224B05221978F4
:1081BC001B48032308F092FB1F4B06221978184822
:1081CC00032308F08BFB1D4B32461978144803230C
:1081DC0008F084FB224612484FF4FC6108F040FB87
:1081EC000F48294608F032FB0D48294608F024FBBD
:1081FC000B4808F03FFB0A4808F042FB0028FAD174
:10820C00074808F041FB064808F044FB0028FAD167
:10821C0010B070BD080002404C2401403002002018
:10822C0000240140340000203500002036000020DE
:10823C003700002038000020390000203A000020D0
:10824C00F0B54469856903466543881A4FF47A7C16
:10825C00002895FBFCF6B8BF4042B042B8BF0CFBFF
:10826C0000F5104E4FF47A7C30682D1895FBFCF01D
:10827C000CFB105737600CB9114611E0914205DA2E
:10828C001B6841189942A8BF194609E008DD064A47
:10829C001B6895FBF2F569185B429942B8BF194609
:1082AC000846F0BD5802002018FCFFFF2DE9F047EE
:1082BC00044690F821000D46062816469846DDF82F
:1082CC0020A0276800D0F0B92868014608F026FEE7
:1082DC003D4908F023FE814694F82500400808F03B
:1082EC00C9FD0146484608F019FE636981467820AD
:1082FC00584308F0BFFD0146484608F0C3FE08F09D
:10830C00D3FF034611E0072801D000230DE00868D5
:10831C00014608F003FE2D4908F0B4FE08F0C4FF36
:10832C00E36B6269434393FBF2F3C245C8EB0A0863
:10833C00B8BF7F42B8F1000FB8BFC8F100084FF4C6
:10834C0080409845D8BF002701F0E6FA012803D1F8
:10835C00304608F08FFD31E0384608F08BFD2E6872
:10836C0080464146304608F077FF70B1A0696369DA
:10837C0037B90B225043584308F078FD144917E0E5
:10838C00584308F073FD134912E04146304608F09B
:10839C0081FFA0B1A069636937B90B2250435843E0
:1083AC0008F064FD0C4903E0584308F05FFD0B49ED
:1083BC0008F068FE0146304608F0A8FC28602868E2
:1083CC0008F072FFBDE8F0870000C0400000F042EA
:1083DC0000401C4600007A4400401CC600007AC4D1
:1083EC00024B00229A601A605A6070475C020020AF
:1083FC00014BB3F90C0070475C02002070B5466865
:10840C00044615460846324671421E4604F00EFBE1
:10841C00236B00B2B3607368616B451BE818F160A5
:10842C003560706011B1104B93FBF1F10A46494273
:10843C0004F0FCFA0346F068B168326858434A43CA
:10844C004FF4803190FBF1F0A1F57F4192FBF1F2FA
:10845C00801830617360A1F5014147F6FF7204F09A
:10846C00E5FA00B270BD00BF0000FF7F2DE9F04FB0
:10847C0089B0A44DBDF84840BDF84AC02C82A5F87F
:10848C0012C0044628699B46DDF854808946019247
:10849C00169EDDF860A003F05DFBC0F30F43ADF852
:1084AC001A30ADF81800069BB8F800706B6194F8A0
:1084BC002130072B25D0082B00F06282062B40F0D0
:1084CC00DA8202F0F7FE94F82D3085B2012B0AD136
:1084DC0094F825101A984908E26902F0C5FE02F0DA
:1084EC007FFE4519ADB294F82430012B03D105F56C
:1084FC00FE45FF35ADB22DB2284602F0A9FE002094
:10850C00FAE103F02DF8012840F011824FF480605D
:10851C0001F002FA012813D04FF4007001F0FCF9BD
:10852C00012801D1199B5BB94FF4006001F0F4F9FB
:10853C00012840F0F981D8F80030002B00F0F481CC
:10854C0094F82A00012800F0788104D302286D4B9E
:10855C0040F0D78173E06B4B42F210715A680132D4
:10856C008A425A6025D8A56BB4F862305543B3F5EE
:10857C00007FB5FBF1F5ADB202D0B3F5806F02D13F
:10858C002BB2C8F80030002002F062FE002002F08E
:10859C00FBFF00215C4803F081FA04A9C0F30F43F0
:1085AC00ADF8100004223046ADF8123008F0E0FAB5
:1085BC0074E2564A002012785860012A12D1A58F15
:1085CC0003F028F8281A80B2254625F8400F02F04F
:1085DC00F7FF4F4B29461B680222ED18281B01F0B0
:1085EC0083FB14E002F0C4FF94F82A302BB994F802
:1085FC00423043F0010384F8423094F82A30022BC5
:10860C0005D194F8423043F0020384F842303D4BDC
:10861C004FF0000159831983584600F01FFB484660
:10862C0000F01CFB179A002300201360CAF80030DE
:10863C0002F090FF4FF4004001F05EF919E21B6864
:10864C00032B00F21682DFE813F004004800D00080
:10865C00D0002E4A2B4B1278012A00F0C4805A68A5
:10866C0042F210718A422BD8A56B013255435A60E5
:10867C000020B5FBF1F5009302F0EAFD002002F0BA
:10868C0083FF009B002103F1140003F007FA04227E
:10869C00C0F30F43ADF8100004A93046ADF812300A
:1086AC0008F066FAB4F86230ADB2B3F5007F03D0CF
:1086BC00B3F5806F40F0F2812BB2C8F80030EDE1D9
:1086CC000020009302F054FF94F8422042F0020282
:1086DC0084F84220009B012285E00C4A094B127859
:1086EC00012A17D1B4F84000009302F069FF02F0A0
:1086FC00A3FF00F50040009B013000B202221A607B
:10870C009860B6E15C020020700200202E0200206E
:10871C00040000209D6894F8252085EAE570520835
:10872C00A0EBE570C2EB024188425BDAE16DE769D0
:10873C00C1EBC1314F435743B4F86220B148B2F595
:10874C00007F97FBF0F702D0B2F5806F10D1DAF80A
:10875C0000A00021504608F09DFD08B1ED1B05E07E
:10876C005046002108F078FD70B17D19A64B0AE047
:10877C00B2F5006F08D1D8F80020002A01DDED1BFE
:10878C0001E001D07D199D609F4F0020258F02F0E4
:10879C005FFDB86802F0F8FEB7F9081007F1140095
:1087AC0003F07CF90422C0F30F43ADF8100004A9C8
:1087BC003046ADF8123008F0DBF9B4F86230B3F59E
:1087CC00007F02D0B3F5806F02D12BB2C8F8003015
:1087DC0094F8427017F0020740F060818A4B022235
:1087EC001A605CE103221A6043E1874D4FF00002EE
:1087FC002A836A83584600F031FA484600F02EFA74
:10880C002A6817990023022A0B60CAF8003005D198
:10881C00002002F09FFE4FF4004000E080207A4DD3
:10882C0001F06AF8002002F013FDA86802F0ACFE1B
:10883C00B5F9081005F1140020E1FFF7FBF8724DB3
:10884C0001468046287F02F0D1FC85F81C801FFA77
:10885C0080F802F02FFD94F8243005B2012B04BFF0
:10886C0005F5FE45FF35284602F0F2FC18F4004FE2
:10887C0003D005F5D445AA3511E0B8F1000F00F08E
:10888C00358105F5144505F5AA7508E000F5FE409F
:10889C00FF3080B200F5FE45FF35ADB227E05B4BF3
:1088AC00E06B1A7894F82530012A0BD000B24543BE
:1088BC005B0895FBF3F04FF6FF7390FBF3F080B27F
:1088CC0002F09AFE02F0B8FE4F4B4FF000025A83B2
:1088DC001A830546584600F0C1F9484600F0BEF927
:1088EC00002002F037FE4FF4004001F005F805F5CA
:1088FC00004501352DB2284602F046FE2946444873
:10890C0030E003F11400002103F0C8F80027C0F395
:10891C000F43ADF8100004A930460422ADF8123014
:10892C003D4608F025F9BAE000213948A6E002F0EE
:10893C0083FE94F82A3000F500400130012B85B2FB
:10894C0003D102F0B7FC00B200E000200FFA85F86A
:10895C0002F07EFC404602F017FE2B4B414603F121
:10896C0014009D8103F09AF804A9C0F30F43ADF8ED
:10897C00100004223046ADF8123008F0F9F878E017
:10898C00E26994F825304FEA0238DAF8000003FB6C
:10899C0008F808F089FC0028B8BF404200FB08F832
:1089AC002B6A40F2DC5298FBF2F89844642398FB53
:1089BC00F3F203FB1283DAF800A02B62002150467D
:1089CC004FF0000508F066FC08B14FF00105EDB260
:1089DC0025B10D4B6FF063019A8907E050460021D9
:1089EC0008F03AFC38B1084B64219A8998FBF1F8ED
:1089FC009044A3F80C80044BB3F80C8055B108F5E7
:108A0C0080480EE0C02709005C0200202E020020E6
:108A1C00700200205046002108F01EFC18B1A8F589
:108A2C0080481FFA88F80FFA88F1354803F036F8B9
:108A3C000422C0F30F43ADF8100004A93046ADF882
:108A4C00123008F095F802F035FC94F8243080B21E
:108A5C00012B03D100F5FE40FF3080B200B202F0D2
:108A6C00F7FB02F0E9FD00F50040013000B202F026
:108A7C008BFD002513E005F11400002103F00EF826
:108A8C000025C0F30F43ADF8100004A930460422B2
:108A9C00ADF812302F4608F06BF800E0002739B221
:108AAC004B46B6F900202046FFF7A8FC154F019B5A
:108ABC00388329B2B6F902202046FFF79FFC788351
:108ACC0007F1180002F046FF07F1180002F068FFEA
:108ADC00C0F30F43ADF80800ADF80A30029B1846FE
:108AEC007B6201F0F3FE09B0BDE8F08F02F0E2FB0F
:108AFC0094F8243080B2012B7FF4CCAEC6E600BFD4
:108B0C00700200205C0200202DE9F041066804464A
:108B1C0015460846324671421E4603F087FFD4F8CC
:108B2C004880431BC6F80880E56C1E493360074635
:108B3C00F56018464FF6FF7203F078FF0346706835
:108B4C00F16818183360706019B16168090491FB01
:108B5C00F5F10A46494203F069FF3268034605FB0A
:108B6C0000F002FB08F84FF4803290FBF2F0A2F513
:108B7C007F4298FBF2F840443061736094F82130E6
:108B8C00082B08D1002F01DDA06B09E016BFA06BEC
:108B9C003846404204E061680A46494203F046FF09
:108BAC00BDE8F0810100FFFF70B5466C1D46044620
:108BBC009E60881A0023EB6028600A494FF6FF720A
:108BCC0003F034FF0346A8684FF48072584390FBBF
:108BDC00F2F028612B6021680A46494203F026FF17
:108BEC0070BD00BF0100FFFFF8B546680C46054696
:108BFC007142104632461F4603F018FF2E6B636815
:108C0C00A660696BC71BF8180425E16091FBF5F5AC
:108C1C002760606011B10F4991FBF5F10A4649429A
:108C2C0003F004FF23680822454396FBF2F65E43EB
:108C3C004FF4803395FBF3F5A3F57C4396FBF3F6E9
:108C4C00AD19606025612846034940F60F6203F0B8
:108C5C00EDFEF8BD00000F0EF1F1FFFF00230361E4
:108C6C0003604360704700BF094B19685A68914212
:108C7C0001D100200BE01A68D118097A0132017079
:108C8C001A601A68202A01D100221A60012070474C
:108C9C0084020020014B9862704700BF84020020C0
:108CAC00034B1A78104612B100221A70012070473B
:108CBC008409002038B50B4B8446DC6A1A6B0134EE
:108CCC00202C08BF002494420BD0DD6A064AED1814
:108CDC00106885F834C040F227710122DC6205F07F
:108CEC00EFF838BD840200205C00002038B5054642
:108CFC00002401E0FFF7DEFF2B5D01341846002B4A
:108D0C00F8D138BD70B5294C238813F0200F1AD038
:108D1C00FEF766FE08B1A38815E0254B5A68196862
:108D2C000132202A08BF00228A4205D05968A08847
:108D3C00C918C0B208725A601E4B0A221A601C4B2A
:108D4C009A6A1D4B1A60194E338813F0800F1BD092
:108D5C00194B1C68C4B9164DEA6A2B6B9A420DD09C
:108D6C00FEF716FE2B6B5A1992F834200133B280A1
:108D7C002B632B6B202B07D12C6305E0304622464E
:108D8C0040F2277105F09CF80848038813F0400F57
:108D9C000AD040F2266105F08BF9054B1A6BDB6AA1
:108DAC009A4201D1FEF708FE70BD00BF004800409A
:108DBC0084020020880900208C09002070B5294C01
:108DCC00238813F0200F1AD0FEF70AFE08B1A388EF
:108DDC0015E0254B5A6819680132202A08BF002279
:108DEC008A4205D05968A088C918C0B208725A6066
:108DFC001E4B0A221A601C4B9A6A1D4B1A60194EA4
:108E0C00338813F0800F1BD0194B1C68C4B9164D56
:108E1C00EA6A2B6B9A420DD0FEF7BAFD2B6B5A19EE
:108E2C0092F834200133B2802B632B6B202B07D1AB
:108E3C002C6305E03046224640F2277105F040F8DD
:108E4C000848038813F0400F0AD040F2266105F061
:108E5C002FF9054B1A6BDB6A9A4201D1FEF7ACFD78
:108E6C0070BD00BF0044004084020020880900202F
:108E7C008C09002070B57B4B86B01C780546012C04
:108E8C002AD1794805F064F921464FF4003006F0F8
:108E9C008BFA2146042006F079FA0420002106F012
:108EAC0091FA0820002106F04DFF06AC4FF00403A8
:108EBC0024F8043D032321466C488DF816301533F5
:108ECC008DF8173006F0AEFE48238DF8173021468A
:108EDC0066484FF008032DE0654B1C78012C2DD112
:108EEC00644805F035F921464FF4802006F05CFA11
:108EFC002146082006F04AFA0820002106F062FA02
:108F0C005D48002106F01EFF06AC4FF4806324F888
:108F1C00043D0323594821468DF8163015338DF83E
:108F2C00173006F07FFE042354488DF81730214685
:108F3C004FF40063ADF8143006F074FE684604F08C
:108F4C0089FF0B2D25D8DFE805F02406090C0F123C
:108F5C0015181B1E20224FF461531CE04FF496434E
:108F6C0019E04FF4E14316E04FF4164313E04FF4CD
:108F7C00614310E04FF496330DE04FF4E1330AE017
:108F8C004FF4613307E03E4B05E03E4B03E03E4BB4
:108F9C0001E04FF4165300933C4B1A683C4B9A4239
:108FAC0002D1009B5B0800932E4B1B78012B04D144
:108FBC00384B2D4A1A60262307E02D4B1B78012BCA
:108FCC0005D1344B2B4A1A6027238DF81030314CC5
:108FDC006946206805F074F800250723012604A8CB
:108FEC008DF811308DF812508DF8136006F09CFA44
:108FFC00206840F2FF3105F037F8206828212A4616
:10900C0004F05EFF2068324640F2277104F058FFEE
:10901C002068324640F2266104F052FF2068324646
:10902C0040F2255104F04CFF20682A4640F22441BE
:10903C0004F046FF20682A4640F6460104F040FF43
:10904C0020682A4640F66A1104F03AFF2068602135
:10905C002A4604F035FF2068314604F023FF06B0A1
:10906C0070BD00BF290200200044004000080140F0
:10907C004B0000200048004010001400000C014080
:10908C0090D0030020A1070040420F0058000020A0
:10909C000024F4005C000020014B03221A6070478E
:1090AC00D8020020044A054B927A0AB1052200E04E
:1090BC0001221A60704700BFA0090020D8020020CE
:1090CC00704700BF014B00225A607047D802002045
:1090DC0008B5074B1A6892B242F008021A601A6877
:1090EC0092B242F004021A60FFF7D6FF08BD00BF2F
:1090FC00405C004010B5064C4FF6FB73226802EA48
:10910C0003032360FFF7CEFF4FF40643236010BD2B
:10911C00405C0040072818BF1F4B10B51E4C18BFF1
:10912C0018702378052B33D8DFE803F003060A0EFA
:10913C001621FFF7DFFF2BE0FFF7DCFF042328E00D
:10914C0002236370013324E06378013BDBB263706C
:10915C006378FBB9042218E0104B1A6892B242F003
:10916C0010021A6005232370DB18637012E0637819
:10917C00013BDBB26370637863B9084A4FF6EF7357
:10918C00116801EA030313600622034B1A7001E015
:10919C000623237010BD00BF040A0020405C004071
:1091AC00034B9B7A13B1034B05221A60704700BF27
:1091BC00A0090020D8020020014B04221A6070473D
:1091CC00D8020020034B1A7A202A01D100221A72ED
:1091DC00704700BFD8020020704700BF212808B597
:1091EC0008D1124B1B681B7803F07F03212B1AD17B
:1091FC000F4B0EE0202816D10C4B0E4A1B681B7827
:10920C0010720D4A03F07F03212B0CBF1346002371
:10921C004BB1064A4FF00001126800205182936155
:10922C009847002000E0022008BD00BF000A002083
:10923C007D920008D802002099920008074B1B6809
:10924C001B7803F07F03212B05D1022801D02228A3
:10925C0001D1002000E00220704700BF000A00206E
:10926C0019B9012801D8084600E00220704700BF58
:10927C0028B9044B4FF008021B681A8200E0024820
:10928C00704700BF000A00206000002028B9044B82
:10929C004FF008021B681A8200E00248704700BFBA
:1092AC00000A0020600000200B4B10B5DA6882B178
:1092BC001B68052B01D000220BE0002303E00749BB
:1092CC00595CC15401330449CC68A342F7D3002341
:1092DC00CB60104610BD00BFD80200200C0A002045
:1092EC00084BDB68082B01D800200AE00023064A53
:1092FC009A5CC2540133092BF9D1024B0022DA607B
:10930C0001207047D80200200C0A0020704700BFD3
:10931C0010B5074C0B468AB2C021636004F004F808
:10932C000120A18803F02CFE012003F0F7FC10BDF6
:10933C00D802002008B5064B1B68DB78042B01D93A
:10934C00002004E0034901EBC30104F04DFA08BD11
:10935C00000A00206800002008B5024904F044FA15
:10936C0008BD00BF8800002008B5024904F03CFA93
:10937C0008BD00BF90000020334B10B51B686FF088
:10938C003F0200245A72DC729C72204603F03EFCB1
:10939C0020464FF4007103F057FC1021204603F0D7
:1093AC0069FC4021204603F0BFFD8021204603F0DC
:1093BC00ABFD204603F0E8FC244B204693F86410E8
:1093CC0003F000FE204603F0B7FC0120214603F019
:1093DC003BFC0120C02103F097FD0120202103F06C
:1093EC0049FC0120214603F05DFC02204FF4C061D2
:1093FC0003F02AFC02204FF4807103F085FD02205B
:10940C00214603F04FFC0220202103F033FC032003
:10941C00214603F019FC03204FF4887103F084FDFE
:10942C000320402103F0CEFD03204FF4405103F004
:10943C0039FC2146032003F01DFC204604F0E2F920
:10944C00034B01221A6010BD000A002060000020AE
:10945C00D802002008B5174B174A196889B2118039
:10946C0016491288098801EA020212F4806F05D0AD
:10947C004FF6FF321A60124BDB6B98470E4B1A8873
:10948C000E4B1B8803EA020212F4007F08D0094934
:10949C000C4A4FF6FF500860117C0131C9B21174AF
:1094AC00054A1288134013F4004F01D003F0A8FFB3
:1094BC0008BD00BF445C0040920900204C0A00200B
:1094CC0060000020D802002010B5032003F0AAFD94
:1094DC00064C034602464FF488710548E36003F0DE
:1094EC003BFF032003F028FC10BD00BFD802002076
:1094FC000C0A002008B5064A064B20B110681988E2
:10950C0006F0F8FB03E01068198806F0F1FB08BDC3
:10951C009C0900209809002038B5064D01232B60CA
:10952C00054B002420461C60FFF7E4FF03232B604F
:10953C00204638BD405C0040445C004008B5FFF755
:10954C00EBFF08BD08B50120FFF7D4FF064B012146
:10955C00196006494FF4E0520A8005490020186052
:10956C0008601A6008BD00BF405C00404C0A002037
:10957C00445C0040084B10B51B6800249C72FFF73C
:10958C00E1FF064A4FF406431460043A1360044AA0
:10959C001460044A138010BD000A0020445C004093
:1095AC00D80200204C0A002007B5142200238DF8A5
:1095BC00042001A801228DF806308DF807208DF8C3
:1095CC00053005F0B1FF0EBD002008B505F054FEC6
:1095DC004FF40000012105F0E7FE08BDF7B5184C6B
:1095EC00184E194F194D9DF820C031602A803860F3
:1095FC000999302204F17E0084F8723084F873C02B
:10960C0007F0B6FA0A99182204F1B20007F0B0FA82
:10961C00FFF7DAFFFFF7C8FF03F0B6FF3868012148
:10962C0005F0B4FE03232D888DF8063030680D3319
:10963C0001A9ADF804508DF8073006F0F3FAFEBD21
:10964C00600000209C090020080A002098090020D6
:10965C00014B1868704700BFB4290020014B1868F3
:10966C00704700BFAC290020014B1868704700BF41
:10967C00A8290020014B1868704700BFA0290020C2
:10968C00014B1868704700BFB0290020014B1868C7
:10969C00704700BF94290020014B1868704700BF29
:1096AC009C290020014B1868704700BF98290020A6
:1096BC00014B1868704700BFA4290020014B1868A3
:1096CC00704700BF500A0020014B1860704700BF64
:1096DC00B4290020014B1860704700BFAC29002052
:1096EC00014B1860704700BFA8290020014B18607F
:1096FC00704700BFA0290020014B1860704700BFC5
:10970C00B0290020014B1860704700BF942900203D
:10971C00014B1860704700BF9C290020014B18605A
:10972C00704700BF98290020014B1860704700BF9C
:10973C00A4290020014B1860704700BF500A00207C
:10974C00094B03F5FA5C00221A605A609A60DA60E1
:10975C0010336345F7D1054B59600121DA6018705D
:10976C0059721A72704700BF540A0020EC02002094
:10977C00024B0022DA605A721A727047EC02002017
:10978C00014B187A704700BFEC020020014B587A4D
:10979C00704700BFEC020020014BD868704700BF37
:1097AC00EC02002008B5064B0021DA681961013281
:1097BC00B2F5FA7FDA6001D1FFF7DAFF08BD00BF1E
:1097CC00EC020020F0B585B0EC468CE80F00114B94
:1097DC0011491A690E680132B2421A610399029852
:1097EC00019C009D13DB1A7A8AB1DB68B3F5FA7F12
:1097FC000DDA0A4A4FEA031C02EB03170CEB0206C4
:10980C004CF802507C60B860F160FFF7CBFF05B0FC
:10981C00F0BD00BFEC02002090010020540A002093
:10982C004FF4FA70704700BF4FF4FA50704700BF06
:10983C0004207047B0F5FA7F07DA032905D8044BEA
:10984C0001EB800053F8200000E00020704700BFBF
:10985C00540A0020074B032809D8DFE800F008025F
:10986C000406012204E0022202E0032200E00022AE
:10987C005A617047EC020020014B5869704700BFD9
:10988C00EC020020014B1860704700BF90010020D3
:10989C00014B1868704700BF9001002010B5154BA4
:1098AC0093F800C0BCF1060F1DD8DFE80CF00406DD
:1098BC00090C0F121600012214E05B689A420AE0B0
:1098CC005B689A420BE05B68994204E05B689942E2
:1098DC0005E05B68984206DA02E05B68984202DDBC
:1098EC00044B01221A72034B1A7A012A01D1013A54
:1098FC005A7210BDEC020020024B1A6840EA0202B8
:10990C001A60704704030020024B1A6822EA000216
:10991C001A60704704030020034B1B6818420CBFED
:10992C0000200120704700BF0403002008B56D2003
:10993C00FFF7EAFF08BD00BF034B10B51C68FFF72B
:10994C00F5FF204610BD00BF04030020034B10B5EB
:10995C001C68FFF7EBFF04F06F0010BD0403002040
:10996C0062B6704772B6704708B5FDF787FF08BD41
:10997C0008B5FDF77BFF08BD08B510B105F072FE08
:10998C0001E005F077FE08BD07B5104B1B78E3B17D
:10999C00FDF7A8FFFDF7A8FFFDF7C8FF002301E0C6
:1099AC00019B01330193019A094B9A42F8D9FDF7B7
:1099BC00A1FFFDF7B3FF002301E0019B01330193ED
:1099CC00019A034B9A42E3D8F7E70EBDC10300207E
:1099DC003F0D030008B5FEF785F8014B187008BD64
:1099EC00C10300202DE9F341234B05461B78884623
:1099FC00012B16461DD1002418E001AF4FEA152C9F
:109A0C0039460222A6231D488DF804C08DF8055056
:109A1C0002F0BAFDA62339461848022202F02AFEAB
:109A2C009DF80430013508F804300134B442E4D315
:109A3C001FE000200321024602F0C8FB0020C5F302
:109A4C000721024602F0C2FB0020E9B2024602F0F6
:109A5C00BDFB002408E0944214BF0022012202F056
:109A6C00B5FB08F8040001340020721EB442014614
:109A7C00F1D3BDE8FC8100BF2D020020005800404E
:109A8C0073B5174B050A1B780446012B13D101AE95
:109A9C0031460222A53313488DF804508DF8054049
:109AAC0002F072FD31460F480222A62302F0E2FDBD
:109ABC009DF8040013E000200321024602F086FB0F
:109ACC000020E9B2024602F081FB0020E1B202461E
:109ADC0002F07CFB00200146012202F077FB7CBDEA
:109AEC002D0200200058004037B52D4B0C461B783A
:109AFC00012B4CD00725454300200321024602F0E0
:109B0C0065FB05F500650020C5F30721024602F050
:109B1C005DFB0020E9B2024602F058FB0020014632
:109B2C00024602F053FB8DF800000020014602466D
:109B3C0002F04CFB8DF8010000200146024602F0B9
:109B4C0045FB8DF8020000200146024602F03EFB68
:109B5C008DF8040000200146024602F037FB8DF818
:109B6C00050000200146024602F030FB8DF806008D
:109B7C0000200122014602F029FB2368009A23F001
:109B8C007F4322F07F429A428DF8070001D00020DB
:109B9C0005E063680198984214BF002001203EBD87
:109BAC002D02002038B5234B1B78012B41D0224BC2
:109BBC001C683BE000200621012202F007FB00207C
:109BCC000521024602F002FB00200122014602F0B0
:109BDC00FDFA10F0020FF2D000200221024602F032
:109BEC00F5FA0020C4F30721024602F0EFFA002038
:109BFC00E1B2024602F0EAFA002500203F2D14BF24
:109C0C00002201220146013502F0E0FA402DF4D188
:109C1C0000200521024602F0D9FA0020012201465B
:109C2C0002F0D4FA10F0010FF2D14034B4F5804FA9
:109C3C00C0D338BD2D0200201000002038B5224BB7
:109C4C000C461B78012B3DD00725454300200321F2
:109C5C00024602F0BBFA05F500650020C5F30721AA
:109C6C00024602F0B3FA0020E9B2024602F0AEFA64
:109C7C0000200146024602F0A9FA2070002001469D
:109C8C00024602F0A3FA607000200146024602F080
:109C9C009DFAA07000200146024602F097FA20714E
:109CAC0000200146024602F091FA60710020014644
:109CBC00024602F08BFAA07100200146012202F04C
:109CCC0085FAE07138BD00BF2D02002010B500F000
:109CDC009BFD044600F098FD001B0028B8BF4042D5
:109CEC000628F7DD10BD00BF2DE9F3414D4B0646AC
:109CFC001B780F46012B14461AD100250DE017F8DE
:109D0C0005E08DF804C08DF806E08DF8056002F0D2
:109D1C003BFCFFF7DBFF01360135A5424FEA162C61
:109D2C0001A94FF003024FF0A6033F48E7D376E0BA
:109D3C0000200621012202F049FA002005210246EA
:109D4C0002F044FA00200122014602F03FFA10F022
:109D5C00020FF2D000200221024602F037FA002056
:109D6C00C6F30721024602F031FA0020F1B2024696
:109D7C0002F02CFA002543E0013616F03F08795D1D
:109D8C0001D1012204E0621E954214BF002201227F
:109D9C00002002F01BFAB8F1000F30D1631E9D4277
:109DAC002DD200200521024602F010FA00200122DB
:109DBC00014602F00BFA10F00100F2D1062101224B
:109DCC0002F004FA00200521024602F0FFF90020FF
:109DDC000122014602F0FAF910F0020FF2D0002035
:109DEC000221024602F0F2F90020C6F307210246D6
:109DFC0002F0ECF90020F1B2024602F0E7F901356D
:109E0C00A542B9D300200521024602F0DFF900205B
:109E1C000122014602F0DAF910F0010FF2D1BDE88F
:109E2C00FC8100BF2D0200200058004037B5264BA6
:109E3C0004461B780D46012B10D14FEA102C01A9BA
:109E4C000322A53321488DF804C08DF805408DF808
:109E5C00065002F099FBFFF739FF33E00020062192
:109E6C00012202F0B3F900200521024602F0AEF9FE
:109E7C0000200122014602F0A9F910F0020FF2D0E5
:109E8C0000200221024602F0A1F90020C4F30721B0
:109E9C00024602F09BF90020E1B2024602F096F96C
:109EAC0029460020012202F091F9002005210246EA
:109EBC0002F08CF900200122014602F087F910F023
:109ECC00010FF2D13EBD00BF2D0200200058004012
:109EDC0038B5154B0C461B78012B24D00725454370
:109EEC0005F50065284609780135FFF79FFF2846E0
:109EFC0061780135FFF79AFF2846A1780135FFF705
:109F0C0095FF284621790135FFF790FF28466179A6
:109F1C000135FFF78BFF2846A179FFF787FF681CF7
:109F2C00E179FFF783FF38BD2D020020194B70B586
:109F3C00054618680C46FFF7A3FD174B1B788342A8
:109F4C0002D1164B1B78BBB1124E00213068FFF7C3
:109F5C006DFFFFF727FE124B294618682822FFF7E2
:109F6C00C3FE104B214618686822FFF7BDFE0A4B52
:109F7C0030681978FFF75AFF094B294618682822D0
:109F8C00FFF730FD074B214618686822FFF72AFDC2
:109F9C0070BD00BF0C00002000000020C103002099
:109FAC009801002004000020084B9A7852B95B7885
:109FBC00142B05D8064A1168064A42F8231004E00F
:109FCC00032200E00422044B1A707047580300204F
:109FDC00BC03002068030020AC040020054B0120CA
:109FEC005A7805498242087002D15A68034B1A60AC
:109FFC00704700BF5803002098040020580400202C
:10A00C00014B02221A70704798040020074A002363
:10A01C001360074A1370074A1360074A1360074A14
:10A02C001370074A1360074A1360704760030020DF
:10A03C009804002058040020A004002054030020A1
:10A04C00BC030020E4040020014B00221A7070476E
:10A05C009804002030B5234B5B78032B3ED8DFE807
:10A06C0003F008022F39204B18681E4B5C68002344
:10A07C0022E01D4A1368092B07D81A491B484C6863
:10A08C00591C40F8234011602BE0092227E052F8BC
:10A09C002350591CA5420ED102EB810204E052F868
:10A0AC00041C013342F8081C411E04328B42F6D3C7
:10A0BC000D4B196015E00B4683420C4AE7D310E0B8
:10A0CC00094A00231360094A002199500433282BB4
:10A0DC00F9D106E0064B0A225A6002E00322044B37
:10A0EC001A7030BD580300209C0400205C04002032
:10A0FC00AC040020264A274B5278092A3BD8DFE8CB
:10A10C0002F0050A0F141A22282E343720491A6837
:10A11C0049688A182EE01E4A196852688A1A29E082
:10A12C001B4A196852684A4324E0194A1968526854
:10A13C0091FBF2F21EE0164A1968526891FBF2F09C
:10A14C0002FB101216E012491A68496801EA020271
:10A15C0010E00F491A68496841EA02020AE00C490A
:10A16C001A68496881EA020204E01A68D24301E0E5
:10A17C00074A52681A60074A074B12681AB91A68DC
:10A18C0042F0080202E01A6822F008021A607047D6
:10A19C0058030020BC030020600300202A4A2B4BEC
:10A1AC0052780A2A43D8DFE802F0060B11161C2459
:10A1BC002A30363A3D0026491A6809688A1803E0A5
:10A1CC00234A196812688A1A1A6030E0204A196802
:10A1DC0012684A43F8E71E4A1968126891FBF2F2BA
:10A1EC00F2E71B4A1968126891FBF2F002FB10129D
:10A1FC00EAE717491A68096801EA0202E4E7144918
:10A20C001A68096841EA0202DEE711491A6809680E
:10A21C0081EA0202D8E70E4B1A68D243D4E71A68D7
:10A22C000B4BD1E70A4A1868116810601960074A8D
:10A23C00084B12681AB91A6842F0080202E01A6850
:10A24C0022F008021A60704758030020BC0300205B
:10A25C00E404002060030020134B5B78052B22D80C
:10A26C00DFE803F003080D12171C104B1A6802F0FC
:10A27C000F0217E00D4B1A6822F0100212E00B4B84
:10A28C001A6822F020020DE0084B1A6822F04002F6
:10A29C0008E0064B1A6822F0800203E0034B1A68B0
:10A2AC0022F480721A60704758030020600300206B
:10A2BC00124B1A68124B5B689A4206DD114B1968F7
:10A2CC0041F0040121F003010CE00E4B05D119689B
:10A2DC0021F0060141F0010104E0196821F00701A9
:10A2EC0041F002011960074B1AB91A6842F00802D2
:10A2FC0002E01A6822F008021A607047BC030020C2
:10A30C00580300206003002010F0020F0CD111F054
:10A31C00100F07D0064B04215A68064B1970064BD8
:10A32C001A6004E00A2200E00822044B1A707047FD
:10A33C00580300209804002050030020AC04002097
:10A34C00014B00221A707047980400200F4B5B7869
:10A35C00032B1AD8DFE803F0020413150C4B00E0B2
:10A36C000C4B1A680C4B110A93F800C00B4B187865
:10A37C000B4B1A7183F807C09871597105E0094BA2
:10A38C0000E0094B1A68064B5A60704758030020CE
:10A39C00500300205804002098040020540300208F
:10A3AC00AC040020BC030020E4040020014B02227A
:10A3BC001A707047C0030020024B5A68024B1A6097
:10A3CC00704700BF5803002058040020294B5B78CD
:10A3DC000C2B4ED8DFE803F0070C11161C21262B92
:10A3EC0030353A3F4400244B1B6813F0080F3BE018
:10A3FC00214B1B6813F0080F08E01F4B1B6813F070
:10A40C00010F31E01C4B1B6813F0010F31D12CE014
:10A41C00194B1B6813F0040F26E0174B1B6813F045
:10A42C00050F21E0144B1B6813F0020F1CE0124BBC
:10A43C001B6813F0030F17E00F4B1B6813F0100F82
:10A44C0012E00D4B1B6813F0200F0DE00A4B1B683C
:10A45C0013F0400F08E0084B1B6813F0800F03E06B
:10A46C00054B1B6813F4807F03D0024B5A68034BD7
:10A47C001A60704758030020600300205804002025
:10A48C00074970B50B68072B09D8064A06481668A9
:10A49C004068064D5C1C45F823600C60106070BD74
:10A4AC00A004002058040020580300203804002089
:10A4BC00054B1A6832B10549013A51F822101A605D
:10A4CC00034B1960704700BFA00400203804002023
:10A4DC0058040020014B00221A7070479804002089
:10A4EC00084B9A784AB95A78142A04D85968064BFA
:10A4FC0043F8221004E0032200E00422034B1A70FC
:10A50C00704700BF5803002068030020AC040020F3
:10A51C00114B9A7852B95A78104B142A04D8104916
:10A52C0051F822205A6004E0032201E00B4B042274
:10A53C001A700C4B1B786BB1084B0B495A680B4BC0
:10A54C000A601AB91A6842F0080202E01A6822F08E
:10A55C0008021A60704700BF58030020AC040020AA
:10A56C006803002090040020BC030020600300203E
:10A57C0010B5094B9A7852B95C78142C05D8F9F7B8
:10A58C005DFF064B43F8240004E0032200E00422A4
:10A59C00034B1A7010BD00BF580300206803002045
:10A5AC00AC04002038B5284B1B788BB9274A284BB4
:10A5BC005268B2F1FF3F04BF264A12680A214A438F
:10A5CC001A6000F021F9244B012218601E4B1A70FE
:10A5DC001E4B5C7814B1012C35D10EE000F014F94F
:10A5EC001D4B1A681A4B821A002A1B68B8BF5242BC
:10A5FC009A4224D9144B1C7025E0FFF79DF910F4F6
:10A60C00804507D0154B10491A68002022F0100223
:10A61C00087017E00E4C23688BB100F0F5F80E4A69
:10A62C0023681268821A002AB8BF52429A4206D98D
:10A63C000A4B05491A680D7042F0100202E0084BF3
:10A64C001A68013A1A6038BD5403002058030020E0
:10A65C00E8080020BC0300208404002060030020D4
:10A66C005804002070B5104D104E2868104C3278EC
:10A67C007368B0F5006F627063600FD83146FFF7F6
:10A68C0027FC31462868FFF72FFA20B12B680133DD
:10A69C002B60652300E00723237004E0072323705D
:10A6AC00044B00221A7070BD500300205803002088
:10A6BC00AC0400209804002037B5124C657815B115
:10A6CC00012D1AD10FE0104B042201A91868FFF7D5
:10A6DC0089F96168019A0D4B914202D101225A60AD
:10A6EC000EE05D600CE0A3782A2B06D1064B211DF1
:10A6FC0018680422FFF7F8FA02E0044B03221A70E0
:10A70C003EBD00BF5803002008000020AC04002010
:10A71C002DE9F3411E4B1F4C5B681F4A0125B3F515
:10A72C00006F1570207027DC11EA050624D118463D
:10A73C006946FFF783FA9DF800809DF801709DF83B
:10A74C0002C09DF807009DF806109DF805209DF8A5
:10A75C000430267284F80180A77084F803C020713D
:10A76C006171A271E3710B4BE95C1A7A01358A189D
:10A77C00082D1A72F7D108E00123064A00219954DA
:10A78C000133082BF9D113781372BDE8FC8100BF9B
:10A79C0058030020C4030020C003002008B50A4B56
:10A7AC000A491A6802EA010169B95A6840F2D243AF
:10A7BC009A4208D1064B1868FFF738FBFFF7F2F9FD
:10A7CC000120FFF7D9F808BD5803002000FFFF0057
:10A7DC000C00002008B5034B1A68034B5A60FBF7BA
:10A7EC00D5F808BDBC0300205803002008B5044B65
:10A7FC0005201A68034B5A60FBF718FA08BD00BF16
:10A80C00BC03002058030020014B1868704700BFA0
:10A81C000803002008B50C4B1B78012B01D1F9F76C
:10A82C00F1FC042004F0A0FA48F6A04004F0ACFAC5
:10A83C00012004F0AFFA05480321002204F042FF86
:10A84C00012004F0BDFA08BD2C0200209AC30200BE
:10A85C0008B5174B1A79CAB11968164A0131196033
:10A86C00154B11681B780131012B116005D1134B6D
:10A87C001A6812B11A68013A1A60114B1B78012B35
:10A88C0001D1F9F7C1FC0022094B00E001221A7139
:10A89C00094B1A78012A09D10A4B196831B1196888
:10A8AC00013919601B680BB9074B1A7008BD00BF42
:10A8BC0008030020780900204A0000208C090020A1
:10A8CC002C020020880900208409002043F2B601E4
:10A8DC0002B24A43494903144B434FF0020C9918F6
:10A8EC0091FBFCF19A1A82B0002992FBFCF20190C8
:10A8FC0004DA002A2ADB002B6CDC04E0002A56DA8E
:10A90C00002B47DC34E003F5E150801A4FF4802132
:10A91C0090FBF1F000F5617080B200EB6242A1F5A2
:10A92C00003193FBF1F192B2511A89B2344BB3F866
:10A93C0020C02CF4005C4FEA0C4C4FEA1C4CA3F8E2
:10A94C0020C098861A87998702B0704701F5E150AC
:10A95C00801A4FF4802390FBF3F000F56170A3F59F
:10A96C00003380B292FBF3F291FBF3F182182EE0EC
:10A97C00C3F5E150401880144FF4003200F56170BB
:10A98C0091FBF2F180B2411A93FBF2F289B28A1870
:10A99C0092B2CBE703F5E150801A801400F5617098
:10A9AC004FF4003180B292FBF1F28218B9E701F555
:10A9BC00E150801A4FF4802390FBF3F000F56170A6
:10A9CC00A3F5003380B291FBF3F100EB6242411A24
:10A9DC0092B2AAE7C3F5E15040184FF4802290FBE5
:10A9EC00F2F000F56170A2F5003291FBF2F180B249
:10A9FC00411A89B201EB63439AB297E7E0E3FFFF98
:10AA0C00002C0140064B00F5617001F5617102F5F7
:10AA1C00617280B289B292B2988619879A87704710
:10AA2C00002C0140014B1878704700BFB929002059
:10AA3C00014B1878704700BFB8290020013808B5C1
:10AA4C00052874D8DFE800F0034D0328284D0021B9
:10AA5C000A46374803F010FF00210A46344803F039
:10AA6C0019FF33480421002203F006FF304804216B
:10AA7C00002203F00FFF2E480821402203F018FF9C
:10AA8C002B480821012203F0F7FE04222848082154
:10AA9C0003F000FF022248E000210A46244803F09C
:10AAAC00EBFE00210A46224803F0F4FE2048042164
:10AABC00402203F0FDFE1E480421012203F0DCFEBF
:10AACC0004210A461A4803F0E5FE19480821002221
:10AADC0003F0D2FE00221648082103F0DBFE01220F
:10AAEC0023E013480021402203F0E2FE104800212D
:10AAFC00012203F0C1FE0E480021042203F0CAFE1D
:10AB0C000B480421002203F0B7FE0948042100225F
:10AB1C0003F0C0FE06480821002203F0ADFE00221F
:10AB2C000348082103F0B6FE0022024B1A7008BD40
:10AB3C00002C0140B8290020013808B5052800F286
:10AB4C001481DFE810F03300E40006008D00600093
:10AB5C00B70000210A46854803F08EFE00210A4604
:10AB6C00824803F097FE81480421602203F0A0FE86
:10AB7C007E480421012203F07FFE7C480421002240
:10AB8C0003F088FE79480821402203F091FE7748B3
:10AB9C000821012203F070FE04227448082103F0FE
:10ABAC0079FE734B01221A709218DCE06F48002179
:10ABBC00602203F07DFE6D480021012203F05CFE53
:10ABCC0000210A46694803F065FE6848042100220A
:10ABDC0003F052FE65480421002203F05BFE63483B
:10ABEC000821402203F064FE60480821012203F092
:10ABFC0043FE04225D48082103F04CFE5C4B00220E
:10AC0C001A700232AFE059480021602203F050FE66
:10AC1C0056480021012203F02FFE00210A4653481A
:10AC2C0003F038FE51480421402203F041FE4F4806
:10AC3C000421012203F020FE04210A464B4803F0B4
:10AC4C0029FE4A480821002203F016FE002247483C
:10AC5C00082103F01FFE464B00221A70013282E0DD
:10AC6C0000210A46414803F007FE00210A463F48EE
:10AC7C0003F010FE3D480421402203F019FE3B482E
:10AC8C000421012203F0F8FD04210A46374803F0A1
:10AC9C0001FE36480821602203F00AFE33480821E1
:10ACAC00012203F0E9FD00223048082103F0F2FDF7
:10ACBC00022255E02D480021402203F0F9FD2B48DB
:10ACCC000021012203F0D8FD28480021042203F0C2
:10ACDC00E1FD26480421002203F0CEFD2348042187
:10ACEC00002203F0D7FD21480821602203F0E0FD8B
:10ACFC001E480821012203F0BFFD00221B48082139
:10AD0C0003F0C8FD1A4B02221A7000222BE01748E0
:10AD1C000021402203F0CCFD14480021012203F055
:10AD2C00ABFD12480021042203F0B4FD0F480421AE
:10AD3C00602203F0BDFD0D480421012203F09CFDAF
:10AD4C000A480421002203F0A5FD0848082100222E
:10AD5C0003F092FD00220548082103F09BFD01221F
:10AD6C00034B1A70013A034B1A7008BD002C0140BA
:10AD7C00B9290020B829002008B5034608460AB9AD
:10AD8C0081F0070013B9FFF759FE01E0FFF7D4FE7D
:10AD9C0008BD00BF37B501AD1A23002428468DF835
:10ADAC0004308DF8074004F0BFFB284619238DF8BA
:10ADBC0004308DF8074004F0B7FB024803F072FF33
:10ADCC003EBD00BF002C0140F0B58F4B8FB01C78FE
:10ADDC000546012C07D12146402004F0D7FA214624
:10ADEC004FF4006002E040F60C00012104F0CEFAB2
:10ADFC00864803F057FF08A803F04AFB4FF0000207
:10AE0C00ADF8202045B940F60F63ADF82250ADF8EF
:10AE1C002430ADF826500BE04FF06002ADF8222044
:10AE2C004FF4E1634FF48072ADF82430ADF8262076
:10AE3C007648002308A98DF8283003F0D1F968462C
:10AE4C0003F030FB25B9ADF80050ADF8065007E023
:10AE5C004FF0700340F20552ADF80030ADF806200B
:10AE6C004FF00103ADF80230694B4FF004021B7830
:10AE7C00ADF80420012B0CD125B9ADF80850ADF874
:10AE8C000A500EE04FF00203ADF808304FF0080204
:10AE9C0005E04FF00003ADF808304FF00202ADF8BA
:10AEAC000A204FF480734FF4007258486946ADF88D
:10AEBC000C30ADF80E2003F0B5F95448694603F098
:10AECC00F9F90DAC6946514803F044FA204604F0F8
:10AEDC00F3FE4D4B1978012916D14E4804F032FF80
:10AEEC0018238DF83730032321468DF836304A4825
:10AEFC004FF47C53ADF8343004F094FE46484FF4D4
:10AF0C00285104F001FF15E01823444821468DF820
:10AF1C0037304FF4E06203238DF83630ADF834202F
:10AF2C0004F080FE4EF2000321463D48ADF834306B
:10AF3C0004F078FE354C0021204603F0E3FB20465C
:10AF4C00002103F0E9FB2046002103F0EFFB354B19
:10AF5C004FF400621B884FF00006ADF816304FF42A
:10AF6C00806304A92046ADF81020ADF812304FF4E0
:10AF7C0000524FF48043ADF81C30ADF81A20ADF8F8
:10AF8C001460ADF8186003F06BFA2046012103F051
:10AF9C00C5FC01210A46204603F0C0FA01212046D7
:10AFAC0003F0A2FB4FF4A06004F0B4FA01271A23BB
:10AFBC000BA88DF82C308DF82D708DF82E608DF837
:10AFCC002F7004F0B1FA19230CA88DF830308DF8DD
:10AFDC0032608DF833708DF8317004F0A5FA1DB91C
:10AFEC00A5862587A58704E04FF46172A286228787
:10AFFC00A2870121054803F073FA0448012103F0EC
:10B00C007DFA0FB0F0BD00BF24020020002C0140DF
:10B01C004E000020C000160000180140000801403E
:10B02C00000C014050000020024B1A6801321A60DB
:10B03C00704700BFC02900200028B8BF40424043E1
:10B04C008B6DC9694FF0140C48430CFB03FC154B7A
:10B05C0070B51A6844F620655C6890FBF5F5BCFB8E
:10B06C00F1F064210132B0FBF1F02D1982421A602B
:10B07C005D6016DB9A680C4C501C90FBF1FC01FBDC
:10B08C001C01DE6854F822004FF47A7CB5FBFCF509
:10B09C00361A76190020586044F82250DE60996008
:10B0AC00186070BD10030020C4290020014BD86823
:10B0BC00704700BF10030020014B1868704700BF99
:10B0CC00C0290020014B1860704700BFC029002028
:10B0DC0008B5054B1B7C012B05D1044B04491868A2
:10B0EC000422FEF701FE08BD10030020BC2900203D
:10B0FC00C029002008B5054B042218600449FEF74E
:10B10C0071FC044B01221A7408BD00BFBC2900203D
:10B11C00C029002010030020014B1868704700BFA5
:10B12C005C2B0020014B1860704700BF5C2B00208B
:10B13C0008B5074B1B78012B09D1064B064918683B
:10B14C000422FEF7D1FDFFF75FFB044B186008BD2E
:10B15C0024030020582B00205C2B0020542B0020B3
:10B16C0038B50F4B1B78012B18D1FFF74DFB0D4C4D
:10B17C004EF65F222368C31A002BB8BF5B42934282
:10B18C000CDD094B094A1D6810680135194604226B
:10B19C001D60FEF7A9FDFFF737FB206038BD00BF2F
:10B1AC0024030020542B00205C2B0020582B002063
:10B1BC0008B5074B042218600649FEF713FCFFF78D
:10B1CC0023FB054B01221860044B1A7008BD00BF0D
:10B1DC00582B00205C2B0020542B00202403002033
:10B1EC00014BB3F90000704728030020884203D0BC
:10B1FC00164B4FF000021A800138052822D8DFE8E0
:10B20C0000F00717030F0B13012916D0022912E0C7
:10B21C00052912D003290EE004290ED001290AE0D9
:10B22C0006290AD0052906E0022906D0042902E0E5
:10B23C00032902D0062905D101E0012003E04FF6D5
:10B24C00FF7000E0002000B2704700BF2803002010
:10B25C00014B5860704700BF28030020014B586811
:10B26C00704700BF2803002000F13B03762B10B57C
:10B27C000D4B0BD951430D4AB3F800C0800392FB20
:10B28C00F1F190FBF1F06044188002E04FF0000205
:10B29C001A80054C0649B4F9000042F6AA2201F0C6
:10B2AC00C5FB208010BD00BF28030020206CFBFFD5
:10B2BC0056D5FFFF012008B5FCF7BCFB0138C0B226
:10B2CC00052801D9002002E0024B33F8100000B22F
:10B2DC0008BD00BFB813010810B50B4C0022206844
:10B2EC00022103F01BF920684FF4487303850021F9
:10B2FC0003F060FB2068012103F0F2F820680221C2
:10B30C00012203F00BF910BD3C0000200C4B07B5DB
:10B31C001B78012B01D11B3304E00A4B1B78012B4A
:10B32C0002D11D338DF80430002301A88DF80730AD
:10B33C0004F0FAF8044B186803F0B4FC0EBD00BF1F
:10B34C0025020020400000203C000020F0B5694B95
:10B35C0089B01C780546012C16D12046214604F0F4
:10B36C0023F82146042006AC04F010F8204604F023
:10B37C00A3FC03238DF81A3001338DF81B302146C2
:10B38C005D484FF0070335E05C4B1E78012E35D13C
:10B39C000420314604F008F8594B06AC1F78012FF5
:10B3AC001AD13946202003F0F1FF204604F084FC2A
:10B3BC0003238DF81A30013321468DF81B30514888
:10B3CC004FF4E043ADF8183004F02CFC39464FF440
:10B3DC00805004F0B7FC11E03146082003F0D6FF92
:10B3EC00204604F069FC482347488DF81B30214661
:10B3FC004FF4E073ADF8183004F014FC434C03AE7A
:10B40C00206803F04FFC304603F042F84FF0FF3356
:10B41C0031462068ADF810304FF00003ADF8123013
:10B42C0002F0DEFE684603F047F84FF00003ADF87B
:10B43C0000304FF00203ADF802304FF00B036946B9
:10B44C002068ADF808304FF00303ADF8043003F07A
:10B45C00C5FB01224FF44871206803F0ADF8206859
:10B46C0003F07AF80121206803F066FA4021206885
:10B47C0003F0B0F80421206803F084FA012120685D
:10B48C0003F04CFA012D6E4628D11A4B1B78012B78
:10B49C0001D11B3304E0194B1B78012B02D11D3356
:10B4AC008DF81C30194C01250023022607A88DF8B5
:10B4BC001E308DF81D608DF81F5004F035F8206893
:10B4CC0041F65F6103F0E0FA314620682A4603F04A
:10B4DC0025F8294620682A4603F020F80B4C002159
:10B4EC00206803F067FA2068012102F0F9FF09B027
:10B4FC00F0BD00BF250200200008014040000020E4
:10B50C002402002000140140000C01403C000020EB
:10B51C00014B1880704700BF642B0020014B186052
:10B52C00704700BF602B002010B504460846FFF79B
:10B53C00EFFF2046FFF7F2FF10BD00BF014B18785C
:10B54C00704700BF30030020014B00221A70704777
:10B55C0030030020014B1870704700BF940100208D
:10B56C00014B1878704700BF94010020704700BF52
:10B57C00034B1B781BB9034B80B21B689884704734
:10B58C002E02002044000020014B5860704700BF81
:10B59C0030030020014B5868704700BF3003002077
:10B5AC000549064B4A8909891B688A18B2FBF3F1D5
:10B5BC0003FB112398B2704730030020602B00204E
:10B5CC00014B1881704700BF3003002008B50520DF
:10B5DC000021012200F0BAFD054B80111B7B1BB131
:10B5EC00044B1B68013B181A014B588108BD00BF66
:10B5FC0030030020602B002008B5044B01461B785B
:10B60C001BB9034B186803F0D5F908BD2E020020B6
:10B61C004400002008B5054B1B7823B9044B18686F
:10B62C0003F024FA01E0034B588908BD2E020020D8
:10B63C00440000203003002008B50E4B1B7823B9C2
:10B64C000D4B186803F012FA09E00C4B5A89188953
:10B65C000B4B80181B68B0FBF3F203FB1200084B7A
:10B66C00C0EB00401A68074BB0FBF2F01B88584344
:10B67C0080B208BD2E0200204400002030030020C0
:10B68C00602B0020642B002007B5184B1B78012B76
:10B69C002AD0174B1B78012B04D107338DF80430BB
:10B6AC00143310E0134B1B78012B04D116338DF897
:10B6BC000430063307E0104B1B78012B14D11633E2
:10B6CC008DF8043007338DF8003001A800238DF875
:10B6DC0003308DF8073003F027FF684603F024FF92
:10B6EC00064B186803F0DEFA0EBD00BF2E020020D8
:10B6FC0026020020480000202702002044000020E1
:10B70C00F0B58A4B8A4A1B788BB0012B0D4611730E
:10B71C00074600F00881874B1C78012C18D1204675
:10B72C00214603F041FE2146042008AC03F02EFE16
:10B73C00204604F0C1FA48238DF8233021464FF0FF
:10B74C0007037D48ADF8203004F06CFA1C233CE074
:10B75C007A4B1C78012C1CD10220214603F024FECC
:10B76C0008AE2146102003F011FE304604F0A4FA76
:10B77C004823314672488DF823304FF4E073ADF80E
:10B78C00203004F04FFA21466E4804F0DBFA1D23FA
:10B79C001BE06D4B1C78012C19D12146042003F0C1
:10B7AC0003FE2146082008AC03F0F0FD204604F00F
:10B7BC0083FA48238DF8233021464FF4E073634815
:10B7CC00ADF8203004F02EFA1E238DF8243002231D
:10B7DC00002409A88DF82530013B8DF827308DF811
:10B7EC00264003F0A1FE5A4B013F186803F05AFAA9
:10B7FC0003A802F04DFE012D18BFADF80E40ADF8B8
:10B80C000C40ADF81240524C08BF102303A920681D
:10B81C0008BFADF80E30ADF8107002F0E1FC012D50
:10B82C0001D1002200E0022203211346206802F01D
:10B83C00E5FE684602F040FE454B694618684FF03D
:10B84C000803ADF8083003F0C9F93A4B1B78012B0B
:10B85C0002D14FF004030CE0384B1B78012B02D1C2
:10B86C004FF0080305E0384B1B78012B03D14FF048
:10B87C000C03ADF80030364C6946206803F0AEF985
:10B88C000121206803F000F901210A46206802F02A
:10B89C0045FE20684FF000030121838402F020FE56
:10B8AC00244B1B78012B05D10020022104F078FADF
:10B8BC0004230EE0214B1B78012B01D1022003E065
:10B8CC00214B1878012805D1082104F069FA4FF4AE
:10B8DC0080730693002308248DF81C3006A80133CE
:10B8EC008DF81E308DF81D4004F002FB114B1B78B7
:10B8FC00012B02D18DF824400AE0104B1B78012B50
:10B90C0003D0114B1B78012B02D116338DF8243048
:10B91C000023012209A88DF826308DF827208DF8F8
:10B92C00253003F001FE0BB0F0BD00BF2E0200204D
:10B93C0030030020260200200008014048000020AF
:10B94C0000100140000C1A0027020020000C0140DE
:10B95C0044000020B0F90030B0F9022003FB03F1E1
:10B96C0002FB021110B50C4CA14214D94FEA116C18
:10B97C00ACF13A0C09495FFA8CFC31F81CC04FF45D
:10B98C00004102FB0CF203FB0CF392FBF1F293FB74
:10B99C00F1F14280018010BD0044FA3AC413010851
:10B9AC00124B37B5B3F902C0B3F90010B0F902204D
:10B9BC00B0F9000002FB0CF400FB01F500FB0CFCE1
:10B9CC004A434FF4004395FBF3F194FBF3F492FBE1
:10B9DC00F3F264189CFBF3F3D31A0020A2B262F3C7
:10B9EC000F009BB263F31F403EBD00BF400300201D
:10B9FC00A0F50040C0F3891000F44073B3F5807FCC
:10BA0C0082B037D001DC23B305E0B3F5007F05D05D
:10BA1C00B3F5407F0FD00023184639E0C0B21E4B5F
:10BA2C00420082F4FF7203EB4000D218B0F88C0095
:10BA3C00B2F88C302CE0184AC0B202EB4003400044
:10BA4C0080F4FF70B3F88C3082185B42B2F88C0033
:10BA5C000EE0114BC0B2420082F4FF7203EB4000C7
:10BA6C00D218B0F88C00B2F88C3040425B4280B2F5
:10BA7C009BB20DE0C0B2084B420082F4FF72D218A8
:10BA8C00B2F88C2003EB40035242B3F88C3090B2E6
:10BA9C0043EA004002B07047C413010830B50446B5
:10BAAC0085B00846FFF7A4FFC0F30F43ADF8023092
:10BABC00ADF80000134A00994FF400431160B4F93B
:10BACC000210B2F90200B4F900C0B2F9002001FB77
:10BADC0000F50CFB02F40CFB00F04A4394FBF3F46E
:10BAEC0095FBF3F192FBF3F2641A90FBF3F3D3188A
:10BAFC000020A2B262F30F009BB263F31F4005B0AB
:10BB0C0030BD00BF40030020032903D8DFE801F05B
:10BB1C0004081014002018E00D4B03EB400004E067
:10BB2C0040000B4B80F4FF70C018B0F88C000CE098
:10BB3C00074B03EB400004E04000054B80F4FF7022
:10BB4C00C018B0F88C00404280B200B2704700BF01
:10BB5C00C413010883B244F6E61100140FFA83FCF7
:10BB6C00484301FB0CF14FF4004291FBF2F190FBC6
:10BB7C00F2F290B24A42A2EB4002002063F30F00B3
:10BB8C0092B284B062F31F4004B0704730B585B0F8
:10BB9C006B4683E80300BDF90410BDF9020040F2C6
:10BBAC00C46202FB01F402FB00FCBDF900506FF013
:10BBBC00020290FBF2F003236D0091FBF2F10918E5
:10BBCC0095FBF3F540F6B8339CFBF3FC4A1994FB58
:10BBDC00F3F3CCEB030392B2002062F30F009BB2A1
:10BBEC0063F31F4005B030BD30B50C4B0C4C844694
:10BBFC0022681B689A4201D100200EE02368094A92
:10BC0C005D1C02EB03130FCB8CE80F00256023683F
:10BC1C00082B01D100232360012030BDF42B002020
:10BC2C00682B0020742B0020704700BF7FB52B4B76
:10BC3C002B4A19681268914204D10120002104F0AA
:10BC4C00B5FB48E01968274A02EB0111487850B15E
:10BC5C001B6802EB0312536804228DF80C2000229F
:10BC6C000192029307E01B68029002EB03125368E7
:10BC7C008DF80C000193194B1A681A4B03EB021345
:10BC8C009B781BB102238DF80D3001E08DF80D303F
:10BC9C00124B00221968134B0901CB5C8DF80E3046
:10BCAC000E4B0DF1180C18680CEB020102EB001C8A
:10BCBC000C4801326044007A082A01F8090CEFD1D3
:10BCCC001A6801321A601A68082A01D100221A6017
:10BCDC0001A804F079FB07B000BD00BF702B002059
:10BCEC006C2B0020F82B0020F0B5437887B006466B
:10BCFC00426833B104238DF80C3000230292019377
:10BD0C0003E0029301928DF80C30B37803B1022357
:10BD1C008DF80D30327800238DF80E20F21801A822
:10BD2C00117AC2180133082BD172F7D104F04CFBF5
:10BD3C00042818D10D4D0E4B2C681B680134082CAF
:10BD4C0008BF00249C4201D100200DE096E80F00B2
:10BD5C002F68084E06EB071C8CE80F0001200146EB
:10BD6C002C6004F023FB012007B0F0BD6C2B0020ED
:10BD7C00702B0020F82B002030B5294D294B2C6856
:10BD8C001B680134082C08BF00249C4287B043D0A8
:10BD9C0001A904F0F5FB9DF80C20234B042A09D1D2
:10BDAC002A68012103EB021251702A6803EB02137B
:10BDBC00029A08E02A68002103EB021251702A68EB
:10BDCC0003EB0213019A5A609DF80D30144A022BB2
:10BDDC00154B04D1126803EB0213012203E0126825
:10BDEC0003EB021300229A700D4B9DF80E101A688B
:10BDFC000D4B1201D1540023094A06A9C818116829
:10BE0C00094D03EB011110F8090C01334919082BEA
:10BE1C000872F1D1146001E004F096FB07B030BD5C
:10BE2C00F42B0020682B0020742B002008B5012077
:10BE3C00FFF7A2FF08BD00BF08B50020FFF79CFF6D
:10BE4C0008BD00BF2DE9F0470C238AB08DF81C30DB
:10BE5C0003238DF81D30013800238DF81B300C4660
:10BE6C00154607281AD8DFE800F01613100D0A192A
:10BE7C0007044FF0020313E04FF0040310E04FF0FF
:10BE8C0010030DE04FF014030AE04FF0280307E015
:10BE9C004FF0640304E04FF0C80301E04FF00803D7
:10BEAC00ADF81E3004F08CFC4FF00070012103F053
:10BEBC007BFA0120014603F069FA0420012103F00A
:10BECC0065FA0420002103F07DFA4FF4EA100021FA
:10BEDC0003F038FF0AAE4FF4805326F8043D0323D9
:10BEEC00314667488DF8263015338DF8273003F02E
:10BEFC0099FE0423314662488DF827304FF40063D5
:10BF0C0000260127ADF824301FFA84F803F08AFECE
:10BF1C0005A80DF1040A8DF81A608DF814608DF8DF
:10BF2C0015708DF816608DF817608DF818708DF8F7
:10BF3C00197004F039F94FEA4813ADF8083050463F
:10BF4C004FF0FF338DF804608DF805608DF80670A6
:10BF5C00ADF80A60ADF80C30ADF80E30ADF81060ED
:10BF6C008DF81270B14604F091F9BDB16B01ADF8CA
:10BF7C00083050464FF0FF338DF80560ADF80A607D
:10BF8C008DF812708DF804708DF80670ADF80C30C9
:10BF9C00ADF80E30ADF8107004F078F94FEAC80324
:10BFAC0043F004030DF10408002701260222641358
:10BFBC00ADF80A3040464FF0FF338DF80420ADF851
:10BFCC0008408DF805708DF80660ADF80C30ADF8B2
:10BFDC000E30ADF810708DF8126004F057F9BD42B8
:10BFEC001BDDEB0043F004036D130322ADF80A30A4
:10BFFC0040464FF0FF338DF804208DF80570ADF8F6
:10C00C0008508DF812608DF80660ADF80C30ADF864
:10C01C000E30ADF8106004F039F908AF0124072692
:10C02C000025142338468DF820308DF821608DF8CA
:10C03C0022508DF8234003F077FA152338468DF8FB
:10C04C0020308DF821608DF822508DF8234003F0BC
:10C05C006BFA132338468DF820308DF821608DF85B
:10C06C0022508DF8234003F05FFA0220214604F0A1
:10C07C009DF92146102004F099F90AB0BDE8F0872B
:10C08C000008014030B52E4B87B01B780546012BBC
:10C09C0003D1012801D12B4C00E02B4C2046002170
:10C0AC0002F0ECFE4FF00003ADF804304FF4827355
:10C0BC00ADF806304FF00003ADF808304FF0020336
:10C0CC00ADF80A304FF00103ADF80C304FF40073AB
:10C0DC00ADF80E304FF00003ADF81230ADF814305F
:10C0EC00052D1ED8DFE805F00306061D09104FF0DC
:10C0FC00100318E04FF0080315E04FF40063ADF89F
:10C10C0008304FF0100305E04FF40063ADF8083031
:10C11C004FF02803ADF810304FF00003ADF80A30A3
:10C12C0003E04FF01803ADF8103001A9204602F0DF
:10C13C0069FE2046012102F0A1FE07B030BD00BF10
:10C14C00280200200038004000300140F8B51D4D99
:10C15C0004462B780E468342174602D0FFF792FF17
:10C16C002C70042C05D0052C06D04CBBFBF772FBB5
:10C17C0004E0FBF7AFFB01E0FBF7B0FB1248022138
:10C18C0002F010FF0028F9D031460F4802F0AEFE45
:10C19C000D48012102F006FF0028F9D067B1042CEC
:10C1AC0005D0052C06D05CB9FBF75AFB04E0FBF775
:10C1BC0093FB01E0FBF794FB034802F099FE00E0CF
:10C1CC000020F8BD4403002000300140F8B52D4D8F
:10C1DC0004462B780E468342174602D0FFF752FFD7
:10C1EC002C70052C4CD8DFE804F00306090C0F1258
:10C1FC00FBF730FB0DE0FBF761FB0AE0FBF762FBA2
:10C20C0007E0FBF763FB04E0FBF764FB01E0FBF7E3
:10C21C0065FB1D4B1B78012B03D1012C01D11B4D50
:10C22C0000E01B4D2846022102F0BCFE0028F9D08C
:10C23C003146284602F05AFE2846012102F0B2FE91
:10C24C000028F9D0BFB1052C1AD8DFE804F003069A
:10C25C00090C0F12FBF704FB0DE0FBF731FB0AE0B6
:10C26C00FBF732FB07E0FBF733FB04E0FBF734FB97
:10C27C0001E0FBF735FB284602F03AFEC0B200E0C5
:10C28C000020F8BD440300202802002000380040A4
:10C29C00003001402DE9F041012186B04FF480506F
:10C2AC0003F074F80120014605AF03F06FF8182471
:10C2BC0003264FF0A00348483946ADF814308DF8EA
:10C2CC0016608DF8174003F0ADFC4FF04003424868
:10C2DC003946ADF814308DF816608DF8174003F020
:10C2EC00A1FC0120002103F02DFD4FF00003ADF85F
:10C2FC0000304FF48273ADF802304FF00003ADF80C
:10C30C0004304FF00203ADF806304FF00103ADF8E6
:10C31C0008304FF4007331486946ADF80A304FF0DD
:10C32C000003ADF80E30ADF81030ADF80C4002F053
:10C33C0069FD0121294802F0A1FD294BE8461D7831
:10C34C00012D42D14FF48040294603F02DF84AF2DA
:10C35C00000324483946ADF814308DF816608DF87A
:10C36C00174003F05FFC4FF4804339461D48ADF88D
:10C37C0014308DF816608DF8174003F053FC4FF015
:10C38C000003ADF800304FF48273ADF802304FF07B
:10C39C000003ADF804304FF00203ADF806304FF453
:10C3AC00007369461048ADF80A304FF00003ADF841
:10C3BC000C40ADF80850ADF80E30ADF8103002F06E
:10C3CC0021FD2946084802F059FD084B4FF0FF3279
:10C3DC001A7006B0BDE8F081000801400030014041
:10C3EC0028020020000C01400038004044030020CB
:10C3FC0082B000211C4A0191938A9BB20193019B4C
:10C40C0013F4806F06D0938A23F480631B041B0CF7
:10C41C0093820191019B13F4007F08D0124A938AF6
:10C42C0023F480631B041B0C938200230193019B58
:10C43C0013F4807F08D00C4A938A23F480731B0476
:10C44C001B0C938200230193019B13F4006F08D003
:10C45C00054A938A23F400631B041B0C938200236C
:10C46C00019302B0704700BF0054004082B000211D
:10C47C001C4A0191938A9BB20193019B13F4806F28
:10C48C0006D0938A23F480631B041B0C93820191C6
:10C49C00019B13F4007F08D0124A938A23F4806323
:10C4AC001B041B0C938200230193019B13F4807FCC
:10C4BC0008D00C4A938A23F480731B041B0C9382C0
:10C4CC0000230193019B13F4006F08D0054A938A53
:10C4DC0023F400631B041B0C93820023019302B012
:10C4EC00704700BF0058004038B50D461F4C194628
:10C4FC00E3B91033A3601E4B65609842E2600AD129
:10C50C0010331C48236003F0FFFD1A48214603F04A
:10C51C00CBFD184826E0184B1848236003F0F4FDB7
:10C52C001648214603F0C0FD14481BE0104B0021B7
:10C53C0098426560E260A1600AD110331048236014
:10C54C0003F0E2FD0E48214603F0AEFD0C4809E075
:10C55C00094B0C48236003F0D7FD0A48214603F031
:10C56C00A3FD0848012103F0CFFD38BD782C002035
:10C57C00005400406C00024010580040440002403F
:10C58C00800002405800024073B5002601960096C8
:10C59C00B0F804C004461FFA8CFC4CF4807CA0F864
:10C5AC0004C01D4633464FF6FF760096FFF79CFFFE
:10C5BC00A3889BB243F40063A38023889BB243F40B
:10C5CC008073238004E0009B5A1E0092002B46D0FF
:10C5DC00A38A13F0010FF6D0224B05F0FE054FF69F
:10C5EC00FF7200921D701B78238204E0009B5A1E80
:10C5FC000092002B33D0A38A13F0020FF6D0238BBA
:10C60C009BB20193184B9C420CD14FF4001003F0D9
:10C61C0093FD0028F9D01548002103F075FD4FF467
:10C62C0000100BE04FF4005003F086FD0028F9D009
:10C63C000F48002103F068FD4FF4005003F08CFD0F
:10C64C00A38A13F0040FFBD023889BB243F400732E
:10C65C002380238813F4007FFBD1012000E000200D
:10C66C007CBD00BFA42C0020005400406C00024094
:10C67C004400024037B5002401940094B0F804C083
:10C68C0004461FFA8CFC4CF4807C1D46A0F804C0B8
:10C69C000123FFF729FFA3889BB243F48053A380A7
:10C6AC00A3889BB243F40063A3804FF6FF730093FF
:10C6BC0023889BB243F48073238004E0009B5A1EB2
:10C6CC000092002B42D0A38A13F0010FF6D0204B1E
:10C6DC0045F001054FF6FF7200921D701B78238206
:10C6EC0004E0009B5A1E0092002B2FD0A38A13F05B
:10C6FC00020FF6D0238B9BB20193164B9C420CD1AC
:10C70C004FF0007003F018FD0028F9D012480021FA
:10C71C0003F0FAFC4FF000700BE04FF4003003F024
:10C72C000BFD0028F9D00D48002103F0EDFC4FF46F
:10C73C00003003F011FD23889BB243F40073238077
:10C74C00238813F4007FFBD1012000E000203EBDC4
:10C75C00A42C0020005400408000024058000240ED
:10C76C0070B5012186B00646082002F00FFE0120AC
:10C77C00014602F0FDFD644B05AC9E4204AD28D190
:10C78C004FF40010012102F00FFE03238DF8163038
:10C79C00193321465D488DF817304FF04003ADF842
:10C7AC00143003F03FFA4FF0800321465748ADF8A0
:10C7BC00143003F037FA4FF40010012102F010FE90
:10C7CC004FF40010002102F00BFE2846012320221A
:10C7DC0027E04FF48000012102F0E6FD03238DF8E1
:10C7EC0016301933494821468DF817304FF48063C1
:10C7FC00ADF8143003F016FA4FF4006321464348A9
:10C80C00ADF8143003F00EFA4FF48000012102F061
:10C81C00E7FD4FF48000002102F0E2FD28460123E1
:10C82C0022228DF8102006228DF813308DF812304C
:10C83C008DF8112002F078FE334B00259E4244F611
:10C84C00206303934BF6FF73ADF802304FF4806313
:10C85C00ADF806304FF48043ADF80050ADF8083019
:10C86C0069462B4C25D14FF028033046ADF80430E7
:10C87C0003F04CF9274803F0A7FB274B2146236014
:10C88C001023A3604FF6FF73E3608023636103F50D
:10C89C003E5320486362A56265602561A561E56130
:10C8AC00256203F001FC1D4803F08EFB21461B485A
:10C8BC0025E04FF0300369461948ADF8043003F019
:10C8CC0025F9184803F080FB174B214623601023F1
:10C8DC00A3604FF6FF73E3608023636103F53E535F
:10C8EC0010486362A56265602561A561E5612562FA
:10C8FC0003F0DAFB0D4803F067FB0C48214603F00C
:10C90C00D3FB06B070BD00BF00540040000C0140CA
:10C91C00782C00206C000240105400408000024033
:10C92C00005800404400024010580040580002409B
:10C93C0008B5FFF715FF08BD03464FF6FF7083429D
:10C94C0046DDB3F1807F23DBB3F1805F0FDBB3F106
:10C95C00804F07DB334A934263DC33491A168A5CF7
:10C96C0012020FE030499A158A5CD2010AE0B3F149
:10C97C00806F2D4A03DB1915525C920102E0991469
:10C98C00525C520193FBF2F101325218521019E031
:10C99C00B3F5801F0BDBB3F5800F234A03DB1914AF
:10C9AC00525C12010EE09913525CD2000AE0B3F50E
:10C9BC00802F1D4A03DB1913525C920002E099127E
:10C9CC00525C520093FBF2F1501C401840101BE0DB
:10C9DC00FF2B1FDDB3F5805F0ADBB3F5804F124AE6
:10C9EC0002DB1912505C0EE09911505C40080AE011
:10C9FC00B3F5806F0C4A03DB1911505C800802E020
:10CA0C009910505CC008013000FB00F29A4208DD1E
:10CA1C00013806E0002BA9BF034A4FF0FF30D05C71
:10CA2C00000970470080FE7F50160108904203DC1D
:10CA3C008142ACBF0A4602461046704770B50446A8
:10CA4C0010460E4604F016FA05462946204604F018
:10CA5C0021FC40B9304604F00DFA05462946204623
:10CA6C0004F0FAFB00B12C46204670BD70B514469C
:10CA7C000E4604F0FFF90546204604F0F7F904468B
:10CA8C002146284604F0FEFA0146284604F03CF9FB
:10CA9C000546304604F0EEF9214604F0F3FA01465F
:10CAAC00284604F033F904F0FFFB70BD70B51BB1E0
:10CABC002D2301F8013B40424B1CB0FBF2F402FB6E
:10CACC00140C5D1EBCF1090F8CBF0CF1570C0CF152
:10CADC00300C03F801CC1E4620460133002CECD15F
:10CAEC0034702B780A7805F8012901F8013BA9422A
:10CAFC00F7D3304670BD00BF0A2A08B584461346EA
:10CB0C008E4603D1002801DA012303E01A46604661
:10CB1C0071460023FFF7CAFF08BD00BF642303FB67
:10CB2C0000F292FBF1F29A420BDD47F612235943C5
:10CB3C006FF00303584391FBF0F000F574505C3038
:10CB4C0019E012F1640F0BDA47F6122359436FF018
:10CB5C000303584391FBF0F0A0F574505C380AE0E5
:10CB6C001C224B43424393FBF0F092FBF1F1024B3E
:10CB7C00401893FBF0F0704700410F00002908B5F6
:10CB8C0002DDFFF7CBFF14E006D1002811D0D4BF93
:10CB9C00084843F65C500CE0002805DBFFF7BEFFAD
:10CBAC0000F5F440B83004E0FFF7B8FFA0F5F4400E
:10CBBC00B83808BDA4C2FFFF014B1860704700BF16
:10CBCC00405C0040014B186880B27047405C0040EC
:10CBDC00014B1860704700BF445C0040014B186863
:10CBEC0080B27047445C0040014B186880B27047BB
:10CBFC00485C0040014B1860704700BF4C5C004023
:10CC0C00014B186880B270474C5C00404FF6F873CB
:10CC1C00024A00EA03031360704700BF505C0040F7
:10CC2C00014B186880B27047505C0040014B43F8D0
:10CC3C0020107047005C0040024B53F8200080B27B
:10CC4C00704700BF005C0040054B10B553F8204006
:10CC5C0048F68F1204EA02020A4343F8202010BD62
:10CC6C00005C0040024B53F8200000F4C060704799
:10CC7C00005C00400A4B10B553F8202048F6BF74F6
:10CC8C0002EA040411F0100F18BF84F0100411F024
:10CC9C00200F18BF84F0200443F8204010BD00BFC3
:10CCAC00005C00400A4B10B553F820204BF68F74F3
:10CCBC0002EA040411F4805F18BF84F4805411F468
:10CCCC00005F18BF84F4005443F8204010BD00BF2F
:10CCDC00005C004038B50D460446FFF7ADFF012D52
:10CCEC0002D120F4805003E0022D04D120F010007A
:10CCFC00014B43F8240038BD005C0040024B53F854
:10CD0C00200000F030007047005C0040024B53F8EC
:10CD1C00200000F440507047005C0040054B48F682
:10CD2C00BF7253F8201001EA020282F0300243F87D
:10CD3C0020207047005C0040054B4BF68F7253F877
:10CD4C00201001EA020282F4405243F8202070477E
:10CD5C00005C0040054B48F68F6253F8201001EA46
:10CD6C00020242F4807243F820207047005C0040BD
:10CD7C00044B48F68F6253F8201001EA020243F884
:10CD8C0020207047005C0040044B48F68F6253F83B
:10CD9C00201001EA020243F820207047005C00409A
:10CDAC00054B48F68F6253F8201001EA020242F458
:10CDBC00807243F820207047005C0040054B48F619
:10CDCC008F6253F8201001EA020242F4807243F899
:10CDDC0020207047005C0040044B48F68F6253F8EB
:10CDEC00201001EA020243F820207047005C00404A
:10CDFC00044B53F8200000F03000102814BF002022
:10CE0C0001207047005C0040054B53F8200000F4F3
:10CE1C004050B0F5805F14BF00200120704700BF68
:10CE2C00005C0040044B40F68F7253F8201001EA6E
:10CE3C00020243F820207047005C0040044B48F687
:10CE4C000F7253F8201001EA020243F820207047B9
:10CE5C00005C0040054B48F68F7253F8201001EA35
:10CE6C00020242F4804243F820207047005C0040EC
:10CE7C00054B48F68F7253F8201001EA020242F07B
:10CE8C00400243F820207047005C0040084B53F8E8
:10CE9C00202012F4804F09D053F8201048F68F72DE
:10CEAC0001EA020242F4804243F82020704700BF9E
:10CEBC00005C0040084B53F8202012F0400F09D0C2
:10CECC0053F8201048F68F7201EA020242F0400239
:10CEDC0043F82020704700BF005C0040054B10B5A4
:10CEEC0053F8204048F68F7204EA02020A4343F8D2
:10CEFC00202010BD005C0040024B53F8200000F0D5
:10CF0C000F007047005C0040064B49081B68490045
:10CF1C009BB203EBC00303F1005303F540535B00DA
:10CF2C0019607047505C0040054A064B126849086E
:10CF3C0092B202EBC002D3185B0049001960704733
:10CF4C00505C004004300020054B1B689BB203EB87
:10CF5C00C00303F1005303F540535B00188870477E
:10CF6C00505C0040044A054B126892B202EBC002BE
:10CF7C00D3185B0018887047505C004004300020C8
:10CF8C00044A054B126892B202EBC002D3185B0044
:10CF9C0019607047505C0040023000203E2909D9CE
:10CFAC004B0911F01F0F01D1013B9BB29B0243F4C3
:10CFBC00004305E04B0811F0010F18BF01339B0231
:10CFCC00036070470D4A0E4B126892B2D31803EBF4
:10CFDC00C0035B003E2909D94A0911F01F0F01D18A
:10CFEC00013A92B2920242F4004205E04A0811F072
:10CFFC00010F18BF013292021A607047505C00405A
:10D00C0006300020054A064B126892B202EBC002B1
:10D01C00D3185B0018688005800D7047505C004089
:10D02C0002300020054A064B126892B202EBC00295
:10D03C00D3185B0018688005800D7047505C004069
:10D04C00063000200C4B30B51D681C68C0001FFA60
:10D05C0085FC8444A4B2094B00190CF1005CC31884
:10D06C000CF5405C490852084FEA4C0049005B0043
:10D07C00520001601A6030BD505C0040043000204A
:10D08C00064B49081B6849009BB203EBC00303F134
:10D09C00005303F540535B0019607047505C00402F
:10D0AC00054A064B1268490892B202EBC002D3182B
:10D0BC005B00490019607047505C00400430002050
:10D0CC00054B1B689BB203EBC00303F1005303F544
:10D0DC0040535B0018887047505C0040044A054B75
:10D0EC00126892B202EBC002D3185B00188870472A
:10D0FC00505C004004300020012910B524D1254B90
:10D10C0025491B68C0009BB2591809184B003E2AD0
:10D11C0009D9510912F01F0F01D1013989B28902C5
:10D12C0041F4004105E0510812F0010F18BF013124
:10D13C00890219601749194B096889B2CB1818185C
:10D14C0040003E2A1ED913E0022922D1114BC00007
:10D15C001C681B68A4B21FFA83FC0F490F4B844454
:10D16C0000194118634449005B000A601A6010E022
:10D17C00530912F01F0F01D1013B9BB29B0243F4E8
:10D18C00004305E0530812F0010F18BF01339B0256
:10D19C00036010BD505C00400230002006300020BF
:10D1AC0001291BD11349144B096889B2CB1803EB25
:10D1BC00C00040003E2A09D9530912F01F0F01D1BB
:10D1CC00013B9BB29B0243F4004305E0530812F071
:10D1DC00010F18BF01339B0203600AE0022908D13A
:10D1EC000449054B096889B201EBC000C3185B0008
:10D1FC001A607047505C00400230002001291BD19E
:10D20C001349144B096889B2CB1803EBC0004000DA
:10D21C003E2A09D9530912F01F0F01D1013B9BB2D1
:10D22C009B0243F4004305E0530812F0010F18BFB2
:10D23C0001339B0203600AE0022908D10449054B23
:10D24C00096889B201EBC000C3185B001A60704713
:10D25C00505C004006300020054A064B126892B222
:10D26C0002EBC002D3185B0018688005800D704774
:10D27C00505C004002300020054A064B126892B206
:10D28C0002EBC002D3185B0018688005800D704754
:10D29C00505C0040063000200D4BC00019680D4A50
:10D2AC0089B241188A185200128812F47C4F01D0AE
:10D2BC0001200CE01A68084B92B28018C3185B006E
:10D2CC0018888005800D002814BF022000207047AC
:10D2DC00505C00400630002002300020012909D1AA
:10D2EC000B4A48F68F7352F8201001EA030343F0FF
:10D2FC0040030AE002290AD1054A48F68F7352F816
:10D30C00201001EA030343F4804342F820307047B5
:10D31C00005C004041EA0020704700BF030AC0B225
:10D32C0043EA0020704700BF01F10051013201F5C2
:10D33C00405110B549005208002308E010F803C012
:10D34C006478013A4CEA042C21F813C00233C41857
:10D35C00002AF3D110BD00BF01F10051013201F5DB
:10D36C00405110B549005208002304E031F8134035
:10D37C00013AC4520233002AF8D110BD08B529E095
:10D38C0047F6FF700860198801F00F018B0003F15C
:10D39C008043117003F5B843196889B211F4004F3A
:10D3AC0009D0186840F68F7100EA010119601278F3
:10D3BC000E4B013A0BE011F0800F0BD0186848F6B9
:10D3CC000F7100EA010119601278094B013A53F808
:10D3DC00223098470749084B0868084A80B21880E1
:10D3EC00188800B20028CBDB08BD00BF4801002024
:10D3FC002C010020445C0040920900209A09002076
:10D40C00F8B59AE047F6FF761E601688564F06F080
:10D41C000F06B30003F1804303F5B8433E70002EB2
:10D42C0064D127682668236807F4405C03EA00008F
:10D43C0080F400502060236806F0300003EA0101FC
:10D44C0081F0200121601388484A13F0100F1080DE
:10D45C00A5F800C004D023689BB213F0800F08D04D
:10D46C00226848F60F7302EA0303236000F0CEFA39
:10D47C0016E013F4006F08D0226840F68F7302EAAE
:10D48C000303236000F062FB0AE013F4004F54D056
:10D49C00226840F68F7302EA0303236000F0F8F968
:10D4AC0021682A884BF68F7301EA030312F4805F1C
:10D4BC0018BF83F4805312F4005F2D4A18BF83F415
:10D4CC0000531360294B11681A8848F6BF7301EAA0
:10D4DC00030312F0100F18BF83F0100312F0200F8B
:10D4EC00234A18BF83F0200313603BE01C68A4B2EE
:10D4FC0014F4004F0BD0196840F68F7201EA020247
:10D50C001A603A781B4B013A53F82230984714F0C2
:10D51C00800F12D0144948F60F720B789B0003F160
:10D52C00804303F5B843186800EA02021A600A78CF
:10D53C00114B013A53F822309847104B104A1D6892
:10D54C000B4C1FFA85FCA2F800C0B2F800C04BF6D9
:10D55C008F700FFA8CFCBCF1000F48F6BF71094DAF
:10D56C00FFF650AFF8BD00BF9A090020A82C002090
:10D57C00005C0040480100202C010020445C00406D
:10D58C0092090020A62C0020074A022108B5074862
:10D59C0011720749074B086007490A60074A136074
:10D5AC001B68984708BD00BFA00900206801002037
:10D5BC00BC09002098000020000A002094090020DB
:10D5CC0010B5074C20B922684FF00103138205E017
:10D5DC00044B1B681B68984720680A3010BD00BFBD
:10D5EC00000A0020BC09002010B50A4B0A4A1B682F
:10D5FC005178DA7891420AD3997841B99C8834B938
:10D60C009A72064B1B685B689847204600E0022024
:10D61C0010BD00BF000A002064010020BC090020DE
:10D62C0010B5074C20B922684FF00103138205E0B6
:10D63C00044B1B689B68984720680C3010BD00BFDA
:10D64C00000A0020BC09002038B50E4C0E4B226895
:10D65C001B68D1789B695079984723689A7A7AB17C
:10D66C0070B91A7962B99D7855B9084B1B68DB689B
:10D67C009847236828465979DA78D9721A7300E0EA
:10D68C00022038BD000A002094090020BC090020AB
:10D69C0008B50246244B20B91B684FF002011982D1
:10D6AC0040E0224A4FF000011B681180197811F0FC
:10D6BC007F0113D15B7A13F0200F03D0117841F066
:10D6CC000201117013F0400F184B15BF1A781A781D
:10D6DC0022F0010242F001021A701EE0012921D051
:10D6EC00022901D000221DE0597911F0800F01F0C0
:10D6FC000F0306D00E4951F8233003F03003102BE2
:10D70C0006E00B4951F8233003F44053B3F5805F26
:10D71C0003D1137843F001031370064B1B681B698C
:10D72C009847024A104608BD000A0020AC2C002085
:10D73C00005C0040BC09002010B51E4B19684A79EA
:10D74C0012F0800F22F0800305D01B4850F8230004
:10D75C0000F0300004E0184850F8230000F440506A
:10D76C00164C94F800C0634522D24C8804BBF8B127
:10D77C00897AE9B112F0800F09D00F4948F6BF72CF
:10D78C0051F8230000EA020282F0100208E00A4974
:10D79C004BF68F7251F8230000EA020282F4805299
:10D7AC0041F82320064B1B689B699847002000E03A
:10D7BC00022010BD000A0020005C00406401002023
:10D7CC00BC09002008B5064B1B685A7A42F02002AF
:10D7DC005A72044B1B68DB699847002008BD00BFD8
:10D7EC00000A0020BC090020054B1A68538A18B99E
:10D7FC008988CB1A138201E008681818704700BF9B
:10D80C00000A002030B50E4B1C78002310E05FFAA4
:10D81C0083FC4FEA8C0202F1804202F5B842156893
:10D82C0048F68F7105EA010141EA0C0111600133E0
:10D83C00A342ECD3034B40F08000186030BD00BF16
:10D84C00640100204C5C0040704700BF08B50C4BD5
:10D85C00002093F82C10FFF7B5FB0A4B1B68187AC5
:10D86C00082807D1084B4FF480521A80074B4FF011
:10D87C0010021A80092814BF0020012008BD00BF27
:10D88C0098000020000A0020A62C0020A82C0020C4
:10D89C0070B52D4B1C68237A032B01D0052B46D178
:10D8AC00A369228AABB1A2B1A58A954228BF1546BD
:10D8BC0028469847228A638A521BEB180646228216
:10D8CC0063820020FFF74EFB2A4601463046FFF7E5
:10D8DC0043FD238A5BB11D4B4FF4405200201A804C
:10D8EC000146FFF74DFB1A4B4FF030021A80A28A0B
:10D8FC00238A9A4203D8144B03221B6803E0124A72
:10D90C001BB1136805221A720DE012680621117200
:10D91C00104A1168104A89B28A18520013600C4BD5
:10D92C004FF030021A80084B1B681B7A06E0072B5D
:10D93C0003D10A4B1B68DB6898470823024A12681C
:10D94C001372FFF783FF70BD000A0020A62C002085
:10D95C00A82C0020505C00400230002094090020CC
:10D96C00F8B5244B1C68238A267ABBB9042E15D132
:10D97C00214822490278012A0BD1214C214A2468E2
:10D98C000370A0B28218520013604FF030020A806C
:10D99C002BE04FF010030B80072626E0A68AA26925
:10D9AC009E4234BF35461D462846B34294BF0426DA
:10D9BC000226904707460020FFF7C6FA2A46014682
:10D9CC003846FFF7B1FC29460020FFF7D9FA638AE5
:10D9DC00228AEB186382094B551B4FF030022582CB
:10D9EC001A80094B4FF440521A80024B1B681E726E
:10D9FC00F8BD00BF000A002045030020A82C002021
:10DA0C00505C004002300020A62C002008B5144BBE
:10DA1C001B681A7A022A01D0042A05D1FFF7A0FF4D
:10DA2C000F4B1B681B7A14E0062A11D15A78052A71
:10DA3C000AD11A7812F07F0F06D1D878FFF7E2FEE0
:10DA4C00084B1B681B6A9847074B1B689B689847D9
:10DA5C000823034A12681372FFF7F8FE08BD00BFD3
:10DA6C00000A0020BC0900209409002038B5324B74
:10DA7C001B68187810F07F0004D15A7A22F020022B
:10DA8C005A7258E0022855D15A88002A52D11A7974
:10DA9C00002A4FD15A7912F0800F22F0800405D061
:10DAAC00264951F8241001F0300104E0234951F8C3
:10DABC00241001F440512248007884423AD20029C3
:10DACC0038D09B7A002B35D012F0800F0FD01B4B27
:10DADC0053F8243003F03003102B25D1E4B2204648
:10DAEC00FFF7E8F920463021FFF7C4F81CE0134D8E
:10DAFC0055F8243003F44053B3F5805F14D134B996
:10DB0C00104B204693F82C10FFF75CFA02E02046ED
:10DB1C00FFF7BCF955F824204BF68F7302EA030388
:10DB2C0083F4405345F82430074B1B685B699847D6
:10DB3C00002000E0022038BD000A0020005C0040FC
:10DB4C006401002098000020BC090020F7B58D4B23
:10DB5C008D4E1A6835688D4B92B2D3182A7A5B00B9
:10DB6C00092A1B681BD09BB203F1005303F54053E9
:10DB7C005B001C4614F8012B03F10A072A705B7832
:10DB8C006B70B4F80300FFF7C9FB6880B4F80700AA
:10DB9C003468FFF7C3FBA08033687F88DF807A4C42
:10DBAC0001212368DA8819725D78002A62D11A780B
:10DBBC0012F07F022ED1092D02D1FFF715FD3BE0AB
:10DBCC00052D0DD193F90320002A4EDB9A78002AFB
:10DBDC004BD19A88002A48D19B7A002B37D044E04D
:10DBEC00032D0BD1DA78012A27D19A882ABB5B7ACC
:10DBFC0013F0200F21D0FFF7E5FD1DE0012D1CD106
:10DC0C00DA78012A19D19A88BAB95B7A13F0200F05
:10DC1C0013D00AE0012A04D10B2D0ED1FFF714FD0D
:10DC2C000AE0022A09D1012D02D1FFF71FFF03E000
:10DC3C00032D02D1FFF780FD48B1554B28461B68D8
:10DC4C005B699847032801D109230FE068B94D4A55
:10DC5C00504B12684FF0300192B2D3185B00002287
:10DC6C001A604D4B1980062300E00823464A1268BF
:10DC7C001372E3E0062D18D11A7812F07F0F40F0E2
:10DC8C0097809B78012B03D1414B1B68DB696EE0BD
:10DC9C00022B03D13E4B1B681B6A68E0032B40F040
:10DCAC0087803B4B1B685B6A61E0002D3CD1598837
:10DCBC0000297DD15A6822F47F42B2F5003F77D11A
:10DCCC001A7812F07F0203D19B88002B70D129E0C7
:10DCDC00012A0BD158792E4B1B689B699847002859
:10DCEC0066D123689B7A002B62D01BE0022A5FD19D
:10DCFC005B7913F0800F03F00F0205D0274951F820
:10DD0C00221001F0300104E0244951F8221001F4F2
:10DD1C0040512348007882424AD213F0700F47D109
:10DD2C00002945D01F4B23E0082D05D11B7813F09B
:10DD3C007F0F3DD11C4B1BE00A2D39D11A7802F014
:10DD4C007F02012A34D19A7A002A31D059880029CD
:10DD5C002ED15A6822F47F42B2F5803F28D15879EF
:10DD6C000B4B1B689B69984710BB104B00E0FBB139
:10DD7C00054A4FF0000112680020936151829847C8
:10DD8C00002020E0505C0040000A002004300020FD
:10DD9C009409002002300020A82C0020005C0040D8
:10DDAC00640100209DD60008CDD500082DD60008B2
:10DDBC00244C254B22681B6850781B699847032814
:10DDCC0001D1236806E01F4B4FF6FF711B681A8ABE
:10DDDC008A4201D1092203E0022800D012B908229C
:10DDEC001A722BE093F90010002921DAD9880191DD
:10DDFC000198824202D9019A1A8211E08A420FD20A
:10DE0C001149096891F82C108A4201D2002105E0D1
:10DE1C0092FBF1F001FB102212B901210B4A117097
:10DE2C00094A126892F82C209A82FFF799FD05E0B6
:10DE3C0003221A72064B4FF440521A80FFF706FD6C
:10DE4C00FEBD00BF000A00209409002045030020FD
:10DE5C00A62C0020002383814FF416528380C380AC
:10DE6C0003814FF00C030260438170470A8810B5A0
:10DE7C004C88B1F804C0038AC98844EA020242EA19
:10DE8C000C0223F470630A431B041B0C92B242EA8B
:10DE9C000303038210BD00BF0023C38003804380B3
:10DEAC008380704721B183899BB243F4005304E013
:10DEBC00838923F400531B041B0C8381704700BF20
:10DECC0001F01F034FF0010CC1F3421161450CFA34
:10DEDC0003F301D10C3004E0022901D1103000E031
:10DEEC0014301AB1026842EA030302E0026822EA23
:10DEFC0003030360704700BF1AB1838A9BB21943B6
:10DF0C0003E0838A9BB223EA01018182704700BF40
:10DF1C00038A23F00F031B041B0C0382038A9BB29E
:10DF2C0041EA030303827047838923F400631B04D3
:10DF3C001B0C838183899BB241EA03038381704765
:10DF4C0021B183899BB243F0020304E0838923F05F
:10DF5C0002031B041B0C8381704700BF038A23F050
:10DF6C0020031B041B0C0382038A9BB241EA0303AC
:10DF7C000382704721B1038A9BB243F4804304E0CF
:10DF8C00038A23F480431B041B0C0382704700BFDD
:10DF9C00C905C90D818070478088C005C00D7047C8
:10DFAC0083899BB243F0010383817047038BDBB2FF
:10DFBC000383038B9BB243EA01230383704700BFA7
:10DFCC00038B03F47F430383038B9BB241EA03036C
:10DFDC000383704721B1838A9BB243F0200304E092
:10DFEC00838A23F020031B041B0C8382704700BF21
:10DFFC0021B1838A9BB243F0100304E0838A23F09F
:10E00C0010031B041B0C8382704700BF21B1838A51
:10E01C009BB243F0080304E0838A23F008031B043B
:10E02C001B0C8382704700BF838A23F004031B04FC
:10E03C001B0C8382838A9BB241EA03038382704761
:10E04C0021B1838A9BB243F0020304E0838A23F05C
:10E05C0002031B041B0C8382704700BF0388194208
:10E06C000CBF002001207047C94389B20180704762
:10E07C004FF0010CC1F3421201F01F0362450CFA80
:10E08C0003F301D1828903E0022A0CBF028A828A3F
:10E09C0092B21340028892B20BB9184607E0090AF3
:10E0AC00012313FA01F111420CBF0020012070472B
:10E0BC00090A01238B40DB439BB20380704700BFEE
:10E0CC00038ACA8823F440531B041B0C134303829A
:10E0DC0083898A8830B5044608890D4623F4B053E9
:10E0EC00498940EA020223F00C030A431B041B0C6F
:10E0FC0092B242EA0303A381A38AAA8923F4407350
:10E10C001B041B0C134387B0A38201A801F0E8F891
:10E11C000E4B2A689C420CBF049B039B192159434C
:10E12C0092006423B1FBF2F1B1FBF3F2120110097E
:10E13C0003FB101109013231B1FBF3F303F00F03B0
:10E14C0043EA020292B2228107B030BD003801408E
:10E15C0008B5214B98422BD008D8A3F50063984200
:10E16C0016D003F58063984234D119E01B4B9842CA
:10E17C0026D003F5684398422CD101214FF48040FE
:10E18C0001F020F94FF48040002101F01BF921E04F
:10E19C004FF40030012101F023F94FF4003016E068
:10E1AC004FF48020012101F01BF94FF480200EE088
:10E1BC004FF40020012101F013F94FF4002006E088
:10E1CC004FF48010012101F00BF94FF48010002165
:10E1DC0001F006F908BD00BF004C004000500040A3
:10E1EC00038803F08F0303800388B1F806C04A88C4
:10E1FC009BB243EA0C0313439BB203808B88838549
:10E20C000B880385064B984203D003F500639842B4
:10E21C0001D10B7A03864FF001038382704700BF54
:10E22C00002C0140038C2DE9F04123F001031B0469
:10E23C001B0C0384038C0A894C8823F002031C4EAC
:10E24C0014431B048288B1F806C0058B1B0CA4B2C6
:10E25C00B04244EA030392B20C88ADB2A0F834C0C9
:10E26C0003D006F50066B04218D18E894F89B1F8FB
:10E27C000E804FF6F77C03EA0C0C4CEA070748EAD1
:10E28C0006064FF6FB73898847F6FF4C02EA0C0C26
:10E29C0007EA0303B2B20B4342EA0C024FF68F714A
:10E2AC0005EA01012143828001830384BDE8F081EA
:10E2BC00002C0140038C2DE9F04123F010031B04CA
:10E2CC001B0C0384028CB1F808C022F0200212044B
:10E2DC008488120C4B8842EA0C1242EA0313A2B255
:10E2EC001B4C068BB1F806C0A0420D88B6B29BB28F
:10E2FC00A0F838C003D004F50064A0421BD1B1F8DB
:10E30C000A804FF67F748F8903EA040447F2FF3CBE
:10E31C0002EA0C0C44EA0814CA894FF6BF738988C8
:10E32C0004EA03034CEA870C43EA01134CEA820229
:10E33C003C469BB292B248F6FF7106EA010141EAF3
:10E34C00052189B2828001830384BDE8F08100BF7E
:10E35C00002C0140038C2DE9F04123F480731B0445
:10E36C001B0C0384028CB1F808C022F40072120456
:10E37C008488120C4B8842EA0C2242EA0323A2B294
:10E38C001A4C868BB1F806C0A0420D88B6B29BB26F
:10E39C00A0F83CC003D004F50064A0421BD1B1F836
:10E3AC000A804FF2FF748F8903EA040444F6FF7C61
:10E3BC0002EA0C0C44EA0824CA894FF6FF33898818
:10E3CC0004EA03034CEA071C43EA01234CEA021259
:10E3DC003C469BB292B24FF68F7106EA010129437B
:10E3EC00828081830384BDE8F08100BF002C014052
:10E3FC00038CF0B523F480531B041B0C0384B1F87D
:10E40C0006C0078C0C8882880D89868B4B88A0F8F7
:10E41C0040C0DFF848C0BFB2604592B2B6B203D07C
:10E42C000CF5006C604505D192048989920C42EA86
:10E43C00811292B24DF6FF7C07EA0C0C48F6FF7184
:10E44C0006EA01014CEA053C41EA04214CEA03339B
:10E45C0089B29BB2828081830384F0BD002C014081
:10E46C00B1F802C00B888A884CEA0303B1F806C0E5
:10E47C0013430A8943EA0C03B1F80AC013438A898F
:10E48C0043EA0C0313439BB2A0F84430704700BF1F
:10E49C0000234FF0FF320372438082800380C380DD
:10E4AC00704700BF0023C381038043808380C380F7
:10E4BC00038143818381704700234FF00102038164
:10E4CC00038043808280C380704700BF0023838118
:10E4DC00038043808380C38003814381704700BFE6
:10E4EC0021B103889BB243F0010304E0038823F0BD
:10E4FC0001039B059B0D0380704700BF39B1B0F839
:10E50C0044306FEA43436FEA53439BB203E0B0F8E5
:10E51C0044305B045B0CA0F8443070471AB183891B
:10E52C009BB2194303E083899BB223EA01018181E9
:10E53C00704700BF818270470A43A0F8482070479B
:10E54C001AB183899BB2194303E083899BB223EAF6
:10E55C0001018181704700BF038923F007031B046D
:10E56C001B0C0381704700BFB0F808C05FFA8CFC2D
:10E57C0041EA0C0C42EA0C0C4CEA032C1FFA8CFC02
:10E58C00A0F808C0704700BF10B50446FFF7ECFFB9
:10E59C0023899BB243F48043238110BD10B50446FC
:10E5AC00FFF7E2FF238923F077031B041B0C43F0D6
:10E5BC007703238110BD00BF01858282704700BFA5
:10E5CC00038823F070039B059B0D41EA0303038032
:10E5DC00704700BF038923F070031B041B0C41EA36
:10E5EC0003030381704700BF10B50446FFF7F2FF29
:10E5FC0023899BB243F00703238110BD30B50489F6
:10E60C00B0F818C0058C2CF4407CADB22CF0030C87
:10E61C0024F007044FEA0C4C25F0220542EA0505CC
:10E62C0024044FEA1C4C45EA0315240C4CF4807C62
:10E63C0021434CF0010CADB20181A0F818C0058447
:10E64C0030BD00BF038B23F070031B041B0C41EA8D
:10E65C0003030383704700BF038B23F4E0431B04C5
:10E66C001B0C43EA01239BB203837047838B23F07B
:10E67C0070031B041B0C41EA03038383704700BF28
:10E68C00838B23F4E0431B041B0C43EA01239BB252
:10E69C008383704721B103889BB243F0800304E06D
:10E6AC00038823F080039B059B0D0380704700BFFC
:10E6BC0021B183889BB243F0040304E0838823F0E8
:10E6CC0004031B041B0C8380704700BF21B183889B
:10E6DC009BB243F0080304E0838823F008031B0477
:10E6EC001B0C8380704700BF21B183889BB243F021
:10E6FC00010304E0838823F001031B041B0C8380BB
:10E70C00704700BF038B23F008031B041B0C41EA6A
:10E71C0003030383704700BF038B23F400631B04C4
:10E72C001B0C43EA01239BB203837047838B23F0BA
:10E73C0008031B041B0C41EA03038383704700BFCF
:10E74C00838B23F400631B041B0C43EA01239BB251
:10E75C0083837047038B23F004031B041B0C41EAD7
:10E76C0003030383704700BF038B23F480631B04F4
:10E77C001B0C43EA01239BB203837047838B23F06A
:10E78C0004031B041B0C41EA03038383704700BF83
:10E79C00838B23F480631B041B0C43EA01239BB281
:10E7AC0083837047038B23F080031B041B0C41EA0B
:10E7BC0003030383704700BF038B5B045B0C43EACA
:10E7CC0001239BB203837047838B23F080031B04CC
:10E7DC001B0C41EA03038383704700BF838B5B04EC
:10E7EC005B0C43EA01239BB283837047038C23F0B9
:10E7FC0002031B041B0C41EA03030384704700BF94
:10E80C00038C23F008031B041B0C41EA0303038451
:10E81C00704700BF038C23F020031B041B0C43EA3E
:10E82C0001139BB203847047038C23F080031B04F9
:10E83C001B0C43EA01139BB203847047038C23F433
:10E84C0000731B041B0C43EA01239BB20384704727
:10E85C00038C23F400631B041B0C43EA01239BB2BF
:10E86C0003847047038C23F400531B041B0C43EAF2
:10E87C0001339BB20384704701238B408A40018C87
:10E88C0089B221EA03030384018C0A4392B2028405
:10E89C00704700BF04238B408A40018C89B221EA67
:10E8AC0003030384018C0A4392B20284704700BFB5
:10E8BC0001238B40B0F820C010B51FFA8CFC2CEA59
:10E8CC000303038409B1082909D1183049084458B5
:10E8DC004FF68F7304EA0303435043580CE004399A
:10E8EC001830C1F34E01445848F6FF7304EA030391
:10E8FC0043501202435892B243EA0202425010BDF6
:10E90C0021B103889BB243F0020304E0038823F097
:10E91C0002039B059B0D0380704700BF21B1038848
:10E92C009BB243F0040304E0038823F004039B052B
:10E93C009B0D0380704700BF21B183889BB243F0CD
:10E94C00800304E0838823F080031B041B0C83806A
:10E95C00704700BF038823F008039B059B0D0380C1
:10E96C0003889BB241EA030303807047838823F03A
:10E97C0070031B041B0C838083889BB241EA030346
:10E98C0083807047038923F007031B041B0C03814E
:10E99C0003899BB241EA030303817047038923F087
:10E9AC0080031B041B0C038103899BB241EA030304
:10E9BC0003817047818470478185704781867047D9
:10E9CC000187704781877047A0F84010704700BFDF
:10E9DC00038B23F00C031B041B0C0383038B9BB2D4
:10E9EC0041EA030303837047038B23F440631B0446
:10E9FC001B0C0383038B9BB243EA01239BB203835F
:10EA0C00704700BF838B23F00C031B041B0C838308
:10EA1C00838B9BB241EA030383837047838B23F47C
:10EA2C0040631B041B0C8383838B9BB243EA01233F
:10EA3C009BB28383704700BF0388DBB203800388DB
:10EA4C009BB241EA03030380704700BF808E80B203
:10EA5C00704700BF008F80B2704700BF808F80B2BC
:10EA6C00704700BFB0F8400080B27047808C80B215
:10EA7C00704700BF008D80B2704700BF038A1942F7
:10EA8C000CBF002001207047C94389B20182704736
:10EA9C00038A828911EA030092B203D011420CBF9F
:10EAAC0000200120704700BFC94389B20182704722
:10EABC00B0F820C010B52CF0010C4FEA0C4C4FEA0A
:10EACC001C4CA0F820C0048BB0F820C0A4B21FFAD4
:10EADC008CFC24F0F30442EA04042CF0020C44EA0B
:10EAEC0003144CF0010C4CEA010CA4B20483A0F802
:10EAFC0020C010BDB0F820C010B52CF0100C4FEA9F
:10EB0C000C4C4FEA1C4CA0F820C0B0F818C0048C78
:10EB1C002CF4407CA4B24FEA0C5C4FEA1C5C24F051
:10EB2C0020044CEA022C44F010044CEA033C44EA66
:10EB3C0001141FFA8CFCA4B2A0F818C0048410BDF8
:10EB4C0038B50D46602D1146044603D10122FFF75E
:10EB5C00D1FF02E00122FFF7ABFF29462046FFF769
:10EB6C0039FD23899BB243F00703238138BD00BFD5
:10EB7C00F8B50C46A2884988B4F800C005460029AF
:10EB8C000CBF02270027012A0CBF0226012623896D
:10EB9C00BCF1000F10D1FFF78BFF2846E188FFF77F
:10EBAC0017FF2846394632462389FFF7A3FF28462C
:10EBBC00E188FFF719FF0FE0FFF79CFF2846E1887B
:10EBCC00FFF712FF2846394632462389FFF770FFBC
:10EBDC002846E188FFF7FCFEF8BD00BF38B50B886E
:10EBEC000C4605464BB94988A2882389FFF760FF7C
:10EBFC002846E188FFF7ECFE53E0042B09D1498845
:10EC0C00A2882389FFF776FF2846E188FFF7ECFE00
:10EC1C0047E0082BB1F802C0B1F804E0098920D113
:10EC2C00028C22F480721204120C0284838B028CEC
:10EC3C009BB292B223F0F30322F4007243EA011167
:10EC4C0042EA0C2C89B21FFA8CFC41EA0E0E4CF4F1
:10EC5C00807CA0F81CE0A0F820C0E188FFF7D2FE71
:10EC6C001FE0028C22F480521204120C0284838B5B
:10EC7C00028C23F4407392B21B051B0D22F400523C
:10EC8C0043EA0E2342EA0C3C43EA01331FFA8CFCA4
:10EC9C009BB24CF4805C8383A0F820C0E188FFF722
:10ECAC00BDFE38BD08B52D4B984237D00BD8A3F517
:10ECBC000063984226D003F58063984228D0B0F1C7
:10ECCC00804F4AD118E0264B984233D004D8A3F594
:10ECDC008063984241D127E0224B984204D003F53F
:10ECEC000063984239D12EE04FF40060012100F00E
:10ECFC0069FB4FF400602DE00120014600F070FB31
:10ED0C0001201CE00220012100F06AFB022016E029
:10ED1C000420012100F064FB042010E008200121F4
:10ED2C0000F05EFB08200AE01020012100F058FBE7
:10ED3C00102004E02020012100F052FB20200021B3
:10ED4C0000F04EFB09E04FF40050012100F03AFBBB
:10ED5C004FF40050002100F035FB08BD000C0040C2
:10ED6C0000140040002C0140042804D1054B1A6803
:10ED7C0042F0040203E0034B1A6822F004021A600A
:10ED8C00704700BF10E000E0014B5860704700BFB7
:10ED9C0010E000E0012804D1084B1A6842F001028F
:10EDAC0006E010F1020F05D1044B1A6822F00102A3
:10EDBC001A6002E0014B00229A60704710E000E0FC
:10EDCC0020B1054B1A6842F0020203E0024B1A68AC
:10EDDC0022F002021A60704710E000E0014B9868C4
:10EDEC00704700BF10E000E0C308022B0BBF044BC0
:10EDFC00034B1B68DB6833FA00F000F0010070472E
:10EE0C0010E000E00B884A88B1F804C01A43CB88A4
:10EE1C0042EA0C02B1F808C01A434B8930B542EAF9
:10EE2C000C028D89B0F800C0CC891A432A432243C6
:10EE3C000CF4415313439BB20380838B23F4006384
:10EE4C001B041B0C83830B8A038230BD00234FF001
:10EE5C000702C3810282038043808380C3800381C5
:10EE6C0043818381704700BF00234381038043802B
:10EE7C008380C3804FF002030381704721B1038864
:10EE8C009BB243F0400304E0038823F040031B04CF
:10EE9C001B0C0380704700BF21B1838B9BB243F4E2
:10EEAC00806304E0838B23F480631B041B0C83833B
:10EEBC00704700BF0909012313FA01F189B21AB195
:10EECC0083889BB2194303E083889BB223EA010138
:10EEDC00818070471AB183889BB2194303E0838801
:10EEEC009BB223EA01018180704700BF818170478A
:10EEFC00808980B2704700BF4FF6FF63994205D0FE
:10EF0C0003889BB243F48073038002E003881940AA
:10EF1C000180704721B183889BB243F0040304E065
:10EF2C00838823F004031B041B0C8380704700BFF1
:10EF3C00038823F400631B041B0C038003889BB21F
:10EF4C0041EA03030380704703889BB243F4805368
:10EF5C000380704721B103889BB243F4005304E053
:10EF6C00038823F400531B041B0C0380704700BF61
:10EF7C00012914BF008B808A80B27047008A80B24E
:10EF8C00704700BFB1F5804F04D103889BB243F4A6
:10EF9C00804304E0038823F480431B041B0C038090
:10EFAC00704700BF038919420CBF00200120704735
:10EFBC00202906D1038903889BB243F040030380C8
:10EFCC0008E0402901D0082901D1038902E0C94396
:10EFDC0089B20181704700BF012301F00F0213FABF
:10EFEC0002F2B0F804C000891FFA8CFC80B2104009
:10EFFC0006D009098B401CEA030F0CBF002001202E
:10F00C00704700BF552906D1038903889BB243F092
:10F01C00400303800DE0562901D0532901D1038907
:10F02C0007E001F00F01012313FA01F1C94389B282
:10F03C0001817047838BF0B523F47A6323F01F03AF
:10F04C001B041B0C83834FF0020303840B89868BF8
:10F05C00022B87B004460D46B6B201D1002225E042
:10F06C0001A88F8800F03CF9EB88002F0CBF01271A
:10F07C000227B3F5007F2989019A06D1A3F5FB730A
:10F08C0053430902B3FBF1F305E00A2349015A4348
:10F09C004F43B2FBF7F305330A229BB2B3FBF2F3F7
:10F0AC0003F001021202C3F34F0392B2991E89B20C
:10F0BC00FE2928BF002228BF0223E98842EA030365
:10F0CC000B439BB223842B886A8846EA0303A988E6
:10F0DC0043F4006313436A890B4313439BB2A3832A
:10F0EC0007B0F0BD08B5154B98421BD003F574431F
:10F0FC00984204D0A3F5784398421DD10AE001212F
:10F10C004FF4805000F05EF94FF48050002100F075
:10F11C0059F911E04FF48040012100F061F94FF4EE
:10F12C00804006E04FF40040012100F059F94FF403
:10F13C000040002100F054F908BD00BF003C004025
:10F14C000D4B0E4A196841F001011960596801EA2A
:10F15C0002025A601A6822F0847222F480321A6019
:10F16C001A6822F480221A605A6822F4FE025A604D
:10F17C0000229A60704700BF001002400000FFF8A8
:10F18C000C4BB0F5803F1A6822F480321A601A6872
:10F19C0022F480221A6003D0B0F5802F08D103E04E
:10F1AC001A6842F4803202E01A6842F4A0221A6013
:10F1BC00704700BF00100240034B1A6822F0F8029F
:10F1CC0042EAC0021A60704700100240014B1860FE
:10F1DC00704700BF00004242044B5A6822F47C1274
:10F1EC0040EA02020A435A60704700BF0010024016
:10F1FC00014B1860704700BF60004242034B5A68D5
:10F20C0022F0030240EA02025A60704700100240EA
:10F21C00024B586800F00C00704700BF0010024011
:10F22C00034B5A6822F0F00240EA02025A6070471F
:10F23C0000100240034B5A6822F4E06240EA0202DA
:10F24C005A60704700100240034B5A6822F4605217
:10F25C0042EAC0025A6070470010024019B1054BD7
:10F26C001A78104303E0034B1A7822EA0000187056
:10F27C00704700BF09100240014B1860704700BF77
:10F28C00D8004242034B5A6822F4404240EA020240
:10F29C005A60704700100240064B002201281A7079
:10F2AC001A7002D0042804D101E0187001E0052284
:10F2BC001A70704720100240014B1860704700BF55
:10F2CC0080044242024B1A6A40EA02021A627047F8
:10F2DC0000100240014B1860704700BF3C044242D2
:10F2EC001F4B10B55A6802F00C02042A13D0082ADE
:10F2FC0011D15A685968C2F38342023211F4803F2B
:10F30C0003D05B6813F4003F01D0164B00E0164BA2
:10F31C005A43026001E0144B0360114A134B5168CD
:10F32C000468C1F30311595C34FA01F1416054686B
:10F33C00C4F3022C13F80C4031FA04F484605468C2
:10F34C00C4F3C22C13F80CC021FA0CF1C160526842
:10F35C00C2F381329B181B7CB1FBF3F1016110BD30
:10F36C000010024000093D0000127A0050170108FD
:10F37C0019B1054B5A69104303E0034B5A6922EA51
:10F38C0000005861704700BF0010024019B1054BD6
:10F39C009A69104303E0034B9A6922EA00009861D2
:10F3AC00704700BF0010024019B1054BDA691043D9
:10F3BC0003E0034BDA6922EA0000D861704700BF12
:10F3CC000010024019B1054BDA68104303E0034BFF
:10F3DC00DA6822EA0000D860704700BF00100240D3
:10F3EC0019B1054B1A69104303E0034B1A6922EA61
:10F3FC0000001861704700BF00100240014B1860FC
:10F40C00704700BF40044242014B1860704700BF78
:10F41C004C004242014B1870704700BF071002406D
:10F42C004309012B02D1084B1B6805E0022B0BBFD3
:10F43C00054B054B1B6A5B6A00F01F0033FA00F0AA
:10F44C0000F00100704700BF0010024008B53120E9
:10F45C00FFF7E6FF094B18705A6801325A601A78A8
:10F46C0022B95A6840F2FF139A42F0D13120FFF7CB
:10F47C00D7FF003818BF012008BD00BF480300208B
:10F48C00024B5A6A42F080725A6270470010024076
:10F49C00034B9B6818420CBF00200120704700BF33
:10F4AC0000100240014B1870704700BF0A10024058
:10F4BC000B4B4FF0FF316FF07042C3F88010C3F864
:10F4CC008420C3F88011C3F88421002303F1C00108
:10F4DC00034A013300200F2B42F82100F6D170476C
:10F4EC0000E100E0094B4FF0206058600848002212
:10F4FC004FF0FF319A60D8601A615A619A61DA61F3
:10F50C001A625A629962D9621963704700ED00E081
:10F51C000000FA0540F0BE60024B40F42020D86099
:10F52C00704700BF00ED00E030B5C27803787AB3C5
:10F53C001C4A4178D2684FF00F0CD243C2F302221E
:10F54C002CFA02FCC2F104029140807803F0030211
:10F55C000CEA000C4CEA010CD2004FEA0C1CFF2008
:10F56C0090400CFA02FC012403F01F02944099080D
:10F57C000D4AC03152F821500CEA000C25EA00006B
:10F58C004CEA00005B0942F8210042F8234008E0F5
:10F59C0003F01F02012191405B09034A203342F81A
:10F5AC00231030BD00ED00E000E100E00023C3704B
:10F5BC000370437083707047024B5868C0F3093076
:10F5CC00704700BF00ED00E0012200F01F0312FAAB
:10F5DC0003F34009044A403052F820001840984286
:10F5EC0014BF00200120704700E100E0014B1860BF
:10F5FC00704700BF00EF00E000F01F0301229A40AB
:10F60C004009024B603043F82020704700E100E0D5
:10F61C00024B58688005800D704700BF00ED00E07C
:10F62C00012200F01F0312FA03F34009044A803050
:10F63C0052F820001840984214BF00200120704757
:10F64C0000E100E0014B1868704700BF00ED00E0DE
:10F65C0021F0604121F07F01014B0143996070471B
:10F66C0000ED00E0014A024BDA6070470400FA0535
:10F67C0000ED00E0014A024BDA6070470100FA0528
:10F68C0000ED00E019B1054B1A69104303E0034B80
:10F69C001A6922EA00001861704700BF00ED00E013
:10F6AC0000F01F00012313FA00F019B1044B5A6A41
:10F6BC00104303E0024B5A6A22EA0000586270477A
:10F6CC0000ED00E0144B70B5DC684FF0FF0CE44328
:10F6DC00C4F302242CFA04F5C4F1040411FA04F462
:10F6EC00C0F30126F6000CFA06FC02EA050545EA11
:10F6FC000404240114FA06F6C0F38110063053F802
:10F70C00202022EA0C0243F8202053F82020164334
:10F71C0043F8206070BD00BF00ED00E0C0F3832013
:10F72C0001238340044A506A03EA0000984214BF44
:10F73C0000200120704700BF00ED00E000F01F002A
:10F74C0001228240024B59680A435A60704700BF3D
:10F75C0000ED00E000F01F020123013A13FA02F25F
:10F76C00024B59680A435A60704700BF00ED00E035
:10F77C00C0F3833001238340044A506A03EA00003B
:10F78C00984214BF00200120704700BF00ED00E03C
:10F79C00C0F3814313B90A4BD86A10E0012B0CD18A
:10F7AC00074AC0F30153906ADA00D040022B14BF11
:10F7BC0000F00F0000F0FF0001E0014B186B7047E8
:10F7CC0000ED00E010F4800F0BBF024B014B586BA7
:10F7DC00986B704700ED00E008B5F4F7C1FC08BD6C
:10F7EC0008B50001F4F7B9FC08BD00BF08B5F4F783
:10F7FC00B2FC08BD08B5F4F7ACFC08BD08B5F4F7CD
:10F80C00A6FC08BD08B5F4F7A0FC08BD002341F226
:10F81C008832C260C38003804BF6FF7283804FF442
:10F82C00804342800381704721B103889BB243F02F
:10F83C00010304E0038823F001031B041B0C038069
:10F84C00704700BF21B183889BB243F4006304E08E
:10F85C00838823F400631B041B0C8380704700BF58
:10F86C0021B183889BB243F4805304E0838823F452
:10F87C0080531B041B0C8380704700BF21B103888D
:10F88C009BB243F4807304E0038823F480731B045D
:10F89C001B0C0380704700BF21B103889BB243F45B
:10F8AC00007304E0038823F400731B041B0C038017
:10F8BC00704700BF21B103889BB243F4806304E01E
:10F8CC00038823F480631B041B0C0380704700BF68
:10F8DC00838901F0FE019BB223F0FE0341EA03038E
:10F8EC008381704721B183899BB243F0010304E00B
:10F8FC00838923F001031B041B0C8381704700BF19
:10F90C0021B103889BB243F0400304E0038823F049
:10F91C0040031B041B0C0380704700BF1AB1838883
:10F92C009BB2194303E083889BB223EA01018180D7
:10F93C00704700BF01827047008AC0B2704700BF99
:10F94C0012B141F0010101E001F0FE0101827047AA
:10F95C0082B0019B0190CB5A98B202B0704700BFA5
:10F96C0031B103886FEA43436FEA53439BB202E021
:10F97C0003885B045B0C0380704700BFB1F5005F2C
:10F98C0004D103889BB243F4005304E0038823F4AE
:10F99C0000531B041B0C0380704700BF21B103886C
:10F9AC009BB243F4805304E0038823F480531B047C
:10F9BC001B0C0380704700BFB1F5006F04D10388A6
:10F9CC009BB243F4006304E0038823F400631B043C
:10F9DC001B0C0380704700BF21B103889BB243F01E
:10F9EC00200304E0038823F020031B041B0C03807A
:10F9FC00704700BF008BC0F30720704721B103880C
:10FA0C009BB243F0100304E0038823F010031B04A3
:10FA1C001B0C0380704700BF21B903889BB243F0D5
:10FA2C00800304E0038823F080031B041B0C038079
:10FA3C00704700BFB1F5804F05D0838B23F4804312
:10FA4C001B041B0C03E0838B9BB243F48043838326
:10FA5C00704700BF828A038B90B240EA034020F0CB
:10FA6C007F407047828A038B90B240EA034020F0BB
:10FA7C007F40884214BF002001207047838A028B8C
:10FA8C009BB243EA02430B4023F07F40003818BF7F
:10FA9C00012070470B0F012B03D1C94389B281821E
:10FAAC000EE0022B01D1838A0AE0062B06D1838A51
:10FABC0003889BB243F00103038001E0838A038B2C
:10FACC00704700BF838A028B9BB243EA02430B4010
:10FADC0023F07F40003818BF012070470B0F012B1B
:10FAEC0003D1C94389B281820EE0022B01D1838AF2
:10FAFC000AE0062B06D1838A03889BB243F00103EC
:10FB0C00038001E0838A038B704700BF70B586B019
:10FB1C000446868801A80D46FFF7E2FB039930489E
:10FB2C0026F03F063604B1FBF0F0360C80B240EA0A
:10FB3C000606A6802288EB6822F001021204120C41
:10FB4C002280284A93420AD85B00B1FBF3F30130C0
:10FB5C009BB280B22084032B98BF042323E0B5F81A
:10FB6C0002C04BF6FF72944505D103225343B1FBFF
:10FB7C00F3F39BB206E019225343B1FBF3F39BB2B0
:10FB8C0043F480431A05120D0AB943F001034FF4F4
:10FB9C009672504302F52F7290FBF2F0013080B256
:10FBAC00208443F40043A38323889BB243F00103D6
:10FBBC0023802388E98823F480632A8823F00A03AE
:10FBCC001B0441EA02021B0C13439BB223802B89BA
:10FBDC00AA8842EA03039BB2238106B070BD00BF22
:10FBEC0040420F00A086010008B50D4B984204D08E
:10FBFC0003F58063984212D107E04FF40010012105
:10FC0C00FFF7EEFB4FF4001006E04FF480000121EB
:10FC1C00FFF7E6FB4FF480000021FFF7E1FB08BD86
:10FC2C0000540040CB78F0B513F0100F18BF8A7851
:10FC3C00098803F00F0C18BF4CEA020C11F0FF0FEF
:10FC4C001AD0046800220126964006EA0105B54246
:10FC5C000ED196000F27B7400CFA06F624EA0704DB
:10FC6C003443282B01D1456102E0482B08BF0561C4
:10FC7C000132082AE7D10460FF291CD9446800220C
:10FC8C0002F108050126AE4006EA0105B5420ED187
:10FC9C0096000F27B7400CFA06F624EA0704344303
:10FCAC00282B01D1456102E0482B08BF05610132C8
:10FCBC00082AE5D14460F0BD0423C370022383708D
:10FCCC004FF0FF3303807047836819420CBF00204C
:10FCDC0001207047806880B2704700BFC36819422A
:10FCEC000CBF002001207047C06880B2704700BF75
:10FCFC0001617047416170470AB1016100E04161E7
:10FD0C00704700BFC160704741F4803383618161EB
:10FD1C008361836983697047064A10B514684FF68E
:10FD2C00807341EA001104EA030341EA0303136000
:10FD3C0010BD00BF00000140014B1860704700BFB0
:10FD4C001C0020420304154A00F4401C1B0CBCF59B
:10FD5C00401F30B5546806D1556824F0706425F006
:10FD6C007065556011E010F4801F06D0C0F303429B
:10FD7C004FF0030C0CFA02F203E0420D120113FADD
:10FD8C0002F224EA020444F0706419B1400D00013F
:10FD9C0083401C43014B5C6030BD00BF0000014040
:10FDAC0001F003039B000F229A4010FA03F310B5E5
:10FDBC008908074C023154F8210020EA020244F869
:10FDCC00212054F82120134344F8213010BD00BFEA
:10FDDC00000001400120014608B5FFF7F3FA0120AD
:10FDEC000021FFF7EFFA08BD08B5264B98422BD03F
:10FDFC000CD8A3F5006398421AD003F5806398429F
:10FE0C001CD0A3F5006398423AD10BE01E4B9842EC
:10FE1C0026D003F58063984228D0A3F5006398425E
:10FE2C002ED117E004200121FFF7CCFA042024E0A6
:10FE3C0008200121FFF7C6FA08201EE0102001213E
:10FE4C00FFF7C0FA102018E020200121FFF7BAFAC2
:10FE5C00202012E040200121FFF7B4FA40200CE0F2
:10FE6C0080200121FFF7AEFA802006E04FF480706D
:10FE7C000121FFF7A7FA4FF480700021FFF7A2FAD7
:10FE8C0008BD00BF00140140001C0140044B1A685F
:10FE9C0002F038021A601A6840EA02021A607047CF
:10FEAC0000200240044B1A6822F008021A601A68FB
:10FEBC0040EA02021A60704700200240044B1A68A4
:10FECC0022F010021A601A6840EA02021A607047A7
:10FEDC0000200240044B00221A605A609A60DA60DB
:10FEEC00024A5A61704700BF00040140FFFF07003F
:10FEFC00837930B5016802794BB3184BCC431D683C
:10FF0C0090F805C004EA05051D605D682C405C6036
:10FF1C00D45844EA0101D15002689868D14301EAEF
:10FF2C0000009860D8680140BCF1100FD96007D16F
:10FF3C00996811439960D96841EA0202DA600BE0D2
:10FF4C005CF8031041EA02024CF8032004E0034B76
:10FF5C00D05820EA0101D15030BD00BF000401404F
:10FF6C0000230C228371427103600371704700BF40
:10FF7C00024B1A6940EA02021A6170470004014000
:10FF8C00034B5B6918420CBF00200120704700BF77
:10FF9C0000040140014B5861704700BF0004014050
:10FFAC00054B1A685B69034001D1184603E0104207
:10FFBC000CBF00200120704700040140014B586128
:10FFCC00704700BF000401400268002322F00102C8
:10FFDC000260036043608360C3602D4B984233D052
:10FFEC0011D83C3B984229D006D8283B984221D0C6
:04FFFC0014339842E0
:020000040801F1
:100000004BD11FE0264B984220D01433984244D164
:100010001EE0244B98422CD008D8A3F56773984271
:100020001DD003F56273984237D11DE01E4B9842F4
:1000300029D0143398422BD0283B98422DD11DE073
:100040001A4B12E0194B15E0184B18E0174B1BE048
:10005000164B1EE0154B5A6842F470021CE0134B1D
:100060005A6842F0706217E0114B5A6842F00F0272
:1000700012E00F4B5A6842F0F0020DE00C4B5A6848
:1000800042F4706208E00A4B5A6842F4704203E09E
:10009000074B5A6842F470225A6070476C00024065
:1000A000440002401C04024044040240000002409C
:1000B000000402408A6870B50C6A0B6944EA0202C7
:1000C0004C691A438B692243CC6905684E6A42EA3F
:1000D000030323438C6A334325F4FE4C23432CF063
:1000E000F00C43EA0C030360CB6843600B68836049
:1000F0004B68C36070BD00BF002383620360436030
:100100008360C360036143618361C36103624362CF
:10011000704700BF19B1036843F0010302E00368B0
:1001200023F001030360704712B10368194302E032
:10013000036823EA01010160704700BF406880B294
:10014000704700BF10F0805F14BF044B044B1B6866
:1001500003420CBF00200120704700BF0004024092
:100160000000024010F0805F14BF024B024B586049
:10017000704700BF000402400000024010F0805FA2
:1001800014BF044B044B1B6803420CBF002001202A
:10019000704700BF000402400000024010F0805F82
:1001A00014BF024B024B5860704700BF000402406E
:1001B00000000240374B01221A605A6812F0010217
:1001C00001D1104664E00278012A0BBF1A681A6850
:1001D00042F0800222F080021A604378012B04D1A1
:1001E0002C4B1A6842F0400203E02A4B1A6822F0B6
:1001F00040021A608378012B04D1264B1A6842F022
:10020000200203E0234B1A6822F020021A60C37810
:10021000012B04D11F4B1A6842F0100203E01D4B62
:100220001A6822F010021A600379012B04D1194BCD
:100230001A6842F0080203E0164B1A6822F008021E
:100240001A604379012B04D1124B1A6842F0040260
:1002500003E0104B1A6822F004021A608279C37915
:1002600090F808C0920742EA03624189437A42EA61
:100270000C4242EA03520139064B0A43DA611A681A
:1002800022F001021A60586880F0010000F00100BD
:10029000704700BF0064004090F800C0012202FADD
:1002A0000CF23B4B2DE9F045D3F8004292B244F0FA
:1002B0000104C3F80042D3F81C42D14301EA04040C
:1002C000C3F81C428478A4B90CF1480CD3F80C7222
:1002D000B0F80AA0C688B0F8088085884FEACC0438
:1002E00004F1804446EA0A4645EA084501EA070760
:1002F00015E0012C1AD10CF1480CD3F80C72B0F8AF
:1003000004A0C688B0F8088045894FEACC0404F1FF
:10031000804446EA0A4645EA084542EA070704F5EA
:10032000C844C3F80C7243F83C60656043782BB94D
:10033000174BD3F8044201EA040404E0144BD3F849
:10034000044242EA0404C3F80442838923B9104BEF
:10035000D3F81442214006E0012B06D10C4BD3F810
:10036000141242EA0101C3F81412837B012B05D158
:10037000074BD3F81C120A43C3F81C22044BD3F8D2
:10038000002222F00102C3F80022BDE8F08500BF80
:100390000064004003220272013A002342724FF0CF
:1003A0000102C3714281037043708370C370037193
:1003B00043718371704700BF19B1054B5A691043EF
:1003C00003E0034B5A6922EA00005861704700BFFE
:1003D00000640040364B70B59968024611F0806F9A
:1003E00001D000200CE0996811F0006F01D00120CD
:1003F00006E09B6813F0805F01D1042056E00220E4
:100400002B4B00F118010901CC5804F00104CC5029
:10041000157A92F809C035B9146864051460CD588E
:100420004CEA050C07E0546845EA0C0CE400546003
:10043000CE584CEA060C4CEA0404CC50947A00F1F5
:10044000180C4FEA0C1C04F00F040CF1804394725A
:1004500003F5C8435D68010125F00F055D605D6827
:1004600001F180412C435C60537B947BD57A1B0463
:1004700043EA0463147B2B4343EA042301F5C84198
:10048000C1F88831557C937CD47B2D0445EA036503
:10049000137C45EA040242EA0322054BC1F88C2191
:1004A0005CF8032042F001024CF8032070BD00BF4D
:1004B00000640040012810D002D302282CD11AE099
:1004C000164A91689368926801F0010103F00203F3
:1004D00043EA8103C2F380621AE0104A936891688C
:1004E00003F48073926801F400719B0943EA1123BD
:1004F000C2F3C0620CE0094A9368916803F4803348
:10050000926801F400319B0B43EA1143C2F300727D
:100510001343034AD05C70470023FAE700640040AD
:1005200064170108012808D002D302280FD109E07E
:10053000074B9A6842F0800208E0054B9A6842F443
:10054000004203E0024B9A6842F400029A6070474E
:100550000064004018B9044B2022DA6002E0024B2C
:1005600020221A61704700BF0064004010B9064B9A
:10057000D86805E0012801D0002003E0024B18698B
:1005800000F00300704700BF00640040254B00F1FD
:100590001B02120110B5D45804F004040C721CB9EB
:1005A000D3585B0D0B6002E0D358DB084B6000F1C1
:1005B0001B021C4B1201D35802F1804203F00203CC
:1005C0004B7202F5C8425468030104F00F0C81F825
:1005D0000AC0526803F18043120ACA7403F5C84383
:1005E000D3F8B821CA72D3F8B821120A0A73D3F823
:1005F000B821120C4A73D3F8B821120E8A73D3F8BB
:10060000BC21CA73D3F8BC21120A0A74D3F8BC21E6
:10061000120C4A74D3F8BC311B0E8B74FFF79AFF8F
:1006200010BD00BF00640040044B1A6842F0020293
:100630001A601868C0F34000704700BF00640040B3
:10064000054B1A6822F002021A60186880F0020056
:10065000C0F34000704700BF00640040034B9B693B
:1006600018420CBF00200120704700BF006400400A
:10067000024B9A6922EA00029A61704700640040C6
:10068000202831D00CD8062820D004D8042825D022
:10069000052844D118E007281DD008283FD11FE0C5
:1006A000B0F5007F2BD005D840281FD0B0F5807F53
:1006B00035D11FE0B0F5803F2CD0B0F5003F2BD0F6
:1006C000B0F5806F2BD11FE0012201E04FF4807262
:1006D000134B9A6023E04FF48032F9E7082200E0E0
:1006E00010220F4BDA601AE0082200E010220C4BB7
:1006F0001A6114E00A4B9A6922F0010208E0084BE3
:100700009A6922F0020203E0054B9A6922F0040282
:100710009A6104E0082200E01022014B5A60704701
:100720000064004001420CBF00200120704700BF60
:10073000202808B532D00CD8062821D004D80428A7
:1007400026D0052818D119E007281ED0082813D173
:1007500020E0B0F5007F29D005D8402820D0B0F5A2
:10076000807F09D120E0B0F5803F27D0B0F5003F71
:1007700022D0B0F5806F1BD0002024E0012101E0E1
:100780004FF48071104B98681BE04FF48031F9E70B
:10079000082100E010210C4BD86812E0082100E08D
:1007A0001021094B18690CE0012102E0022100E050
:1007B0000421054B986904E0102100E00821024B58
:1007C0005868FFF7AFFF08BD00640040012108B57D
:1007D0004FF00070FEF70AFE4FF000700021FEF7A8
:1007E00005FE08BD436830B523F470230C680A7910
:1007F00023F48073234343EA0223436082688D68B5
:10080000CC680A4B45EA040C02EA03034A794CEA35
:10081000030343EA420383600B7CC26A013B22F478
:100820007002DBB242EA0353C36230BDFDF7F1FF51
:10083000002301220274C36003600371437183606B
:10084000704700BF19B1836843F0010302E0836879
:1008500023F001038360704719B1836843F4807308
:1008600002E0836823F4807383607047C9B212B1D9
:100870004368194302E0436823EA0101416070477D
:10088000836843F008038360704700BF8068C0F34B
:10089000C0007047836843F004038360704700BF63
:1008A0008068C0F38000704719B1836843F4A003E7
:1008B00002E0836823F4A003836070478068C0F37C
:1008C000805070474368013923F4604343EA413361
:1008D0004360704719B1436843F4006302E0436822
:1008E00023F4006343607047092930B511D94FF0F4
:1008F000030C0CFB01FC0725ACF11E0C05FA0CF5F2
:1009000003FA0CFCC46824EA050343EA0C03C36041
:100910000EE04FF0030C0CFB01FC072505FA0CF56B
:1009200003FA0CFC046924EA050343EA0C0303619F
:10093000062A0DD80523013A5A434FF01F0C0CFA32
:1009400002FC9140436B23EA0C020A4342631CE021
:100950000C2A0DD805235A434FF01F0C233A0CFAEA
:1009600002FC9140036B23EA0C020A4302630CE091
:1009700005235A434FF01F0C413A0CFA02FC9140F8
:10098000C36A23EA0C020A43C26230BD19B183680C
:1009900043F4801302E0836823F48013836070477C
:1009A000C06C80B2704700BF014B1868704700BF31
:1009B0004C24014019B1436843F4806302E043686A
:1009C00023F480634360704719B1436843F4805354
:1009D00002E0436823F4805343607047836823F444
:1009E000E04341EA03038360704700BF19B18368A5
:1009F00043F4004302E0836823F4004383607047BC
:100A000019B1836843F4021302E0836823F40213EC
:100A1000836070478068C0F340507047092930B543
:100A200011D94FF0030C0CFB01FC0725ACF11E0C97
:100A300005FA0CF503FA0CFCC46824EA050343EA42
:100A40000C03C3600EE04FF0030C0CFB01FC072508
:100A500005FA0CF503FA0CFC046924EA050343EAE1
:100A60000C030361836BC3F3015CCCEB0202023223
:100A70004FF0050CD2B20CFB02F20CF11A0C0CFA7E
:100A800002FC914023EA0C030B43836330BD00BF9B
:100A9000836B013923F4401343EA015383637047A6
:100AA0000A5070472830405880B27047436823F49A
:100AB000400323F4007341EA03034360704700BF1F
:100AC00041628262704700BF436823F01F0341EA1E
:100AD00003034360704700BF20B1054B9A6842F49E
:100AE000000203E0024B9A6822F400029A60704709
:100AF00000240140036819420CBF00200120704708
:100B0000C9430160704700BF4368006810EA1120C4
:100B100004D0C9B219420CBF00200120704700BFA9
:100B20006FEA11210160704708B5134B98420FD04E
:100B300003F5A053984213D0A3F5C053984219D19E
:100B40004FF400700121FEF743FC4FF400700EE0FB
:100B50004FF480600121FEF73BFC4FF4806006E01B
:100B60004FF400400121FEF733FC4FF40040002118
:100B7000FEF72EFC08BD00BF00280140032A2DE926
:100B8000F0070BD83AB1002311F803C000F803C0F6
:100B900001339342F8D1BDE8F007704782180C4644
:100BA000034603E014F8011C03F8011C03F00306DC
:100BB0001946A44601330134002EF3D11CF003047E
:100BC000634608BFC1EB020C68D06542C4F1040A59
:100BD0000CEB050733464FEACA0A5CF805604FEA9A
:100BE000C408551A08E057F8044F264604FA0AF4D8
:100BF00049EA0404CC5004335C18032D26FA08F9A2
:100C0000A5F104050CEB0306EDDC002302E0F15C2A
:100C1000E154013319199142F9D3BCE753F8404C20
:100C200041F8404C53F83C4C41F83C4C53F8384C9C
:100C300041F8384C53F8344C41F8344C53F8304CAC
:100C400041F8304C53F82C4C41F82C4C53F8284CBC
:100C500041F8284C53F8244C41F8244C53F8204CCC
:100C600041F8204C53F81C4C41F81C4C53F8184CDC
:100C700041F8184C53F8144C41F8144C53F8104CEC
:100C800041F8104C53F80C4C41F80C4C53F8084CFC
:100C900041F8084C53F8044C41F8044C1C460D46EE
:100CA00040334031BCF13F0FACF1400CB6DC214683
:100CB0002B46541B0FE051F8105C43F8105C51F8C0
:100CC0000C5C43F80C5C51F8085C43F8085C51F884
:100CD000045C43F8045C0F2C0D469C4601F11001A6
:100CE00003F11003A4F11004E5DCCCEB02010023B6
:100CF00003E0EC584CF8034004335E19032903EB7E
:100D00000C04A1F10401F4DC7FE700BF80F0004097
:100D100002E000BF81F0004142001FBF5FEA4103D3
:100D200092EA030F7FEA226C7FEA236C6AD04FEAD3
:100D30001262D2EB1363C1BFD21841404840414018
:100D4000B8BF5B42192B88BF704710F0004F40F4CA
:100D5000000020F07F4018BF404211F0004F41F4E6
:100D6000000121F07F4118BF494292EA030F3FD0B2
:100D7000A2F1010241FA03FC10EB0C00C3F12003C5
:100D800001FA03F100F0004302D5494260EB400054
:100D9000B0F5000F13D3B0F1807F06D340084FEABF
:100DA000310102F10102FE2A51D2B1F1004F40EBB4
:100DB000C25008BF20F0010040EA0300704749001C
:100DC00040EB000010F4000FA2F10102EDD1B0FAE7
:100DD00080FCACF1080CB2EB0C0200FA0CF0AABFDC
:100DE00000EBC25052421843BCBFD040184370477A
:100DF00092F0000F81F4000106BF80F40000013280
:100E0000013BB5E74FEA41037FEA226C18BF7FEA56
:100E1000236C21D092EA030F04D092F0000F08BF98
:100E20000846704790EA010F1CBF0020704712F07F
:100E30007F4F04D1400028BF40F00040704712F1BE
:100E400000723CBF00F50000704700F0004343F023
:100E5000FE4040F4000070477FEA226216BF084659
:100E60007FEA23630146420206BF5FEA412390EA1C
:100E7000010F40F4800070474FF0000304E000BF12
:100E800010F0004348BF40425FEA000C08BF7047C3
:100E900043F0964301464FF000001CE050EA010287
:100EA00008BF70474FF000030AE000BF50EA01029C
:100EB00008BF704711F0004302D5404261EB410189
:100EC0005FEA010C02BF84460146002043F0B643AE
:100ED00008BFA3F18053A3F50003BCFA8CF2083AD3
:100EE000A3EBC25310DB01FA02FC634400FA02FCDC
:100EF000C2F12002BCF1004F20FA02F243EB0200E3
:100F000008BF20F00100704702F1200201FA02FC44
:100F1000C2F1200250EA4C0021FA02F243EB020037
:100F200008BF20EADC7070474FF0FF0C1CEAD0527B
:100F30001EBF1CEAD15392EA0C0F93EA0C0F6FD03C
:100F40001A4480EA010C400218BF5FEA41211ED01A
:100F50004FF0006343EA501043EA5111A0FB013106
:100F60000CF00040B1F5000F3EBF490041EAD371DB
:100F70005B0040EA010062F17F02FD2A1DD8B3F157
:100F8000004F40EBC25008BF20F00100704790F0C6
:100F9000000F0CF0004C08BF49024CEA502040EA18
:100FA00051207F3AC2BFD2F1FF0340EAC2507047DE
:100FB00040F400004FF00003013A5DDC12F1190F1C
:100FC000DCBF00F000407047C2F10002410021FA8E
:100FD00002F1C2F1200200FA02FC5FEA310040F1A6
:100FE000000053EA4C0308BF20EADC70704792F01F
:100FF000000F00F0004C02BF400010F4000F013A57
:10100000F9D040EA0C0093F0000F01F0004C02BF51
:10101000490011F4000F013BF9D041EA0C018FE7C0
:101020000CEAD15392EA0C0F18BF93EA0C0F0AD0C6
:1010300030F0004C18BF31F0004CD8D180EA0100EC
:1010400000F00040704790F0000F17BF90F0004F85
:10105000084691F0000F91F0004F14D092EA0C0F67
:1010600001D142020FD193EA0C0F03D14B0218BFFA
:10107000084608D180EA010000F0004040F0FE4040
:1010800040F40000704740F0FE4040F440007047DC
:101090004FF0FF0C1CEAD0521EBF1CEAD15392EA5B
:1010A0000C0F93EA0C0F69D0A2EB030280EA010C4B
:1010B00049024FEA402037D04FF0805343EA1111E4
:1010C00043EA10130CF000408B4238BF5B0042F142
:1010D0007D024FF4000C8B4224BF5B1A40EA0C00E7
:1010E000B3EB510F24BFA3EB510340EA5C00B3EB19
:1010F000910F24BFA3EB910340EA9C00B3EBD10F07
:1011000024BFA3EBD10340EADC001B0118BF5FEA58
:101110001C1CE0D1FD2A3FF650AF8B4240EBC25081
:1011200008BF20F0010070470CF0004C4CEA502042
:101130007F32C2BFD2F1FF0340EAC250704740F491
:1011400000004FF00003013A37E792F0000F00F083
:10115000004C02BF400010F4000F013AF9D040EA01
:101160000C0093F0000F01F0004C02BF490011F495
:10117000000F013BF9D041EA0C0195E70CEAD1538D
:1011800092EA0C0F08D142027FF47DAF93EA0C0F74
:101190007FF470AF084676E793EA0C0F04D14B0258
:1011A0003FF44CAF08466EE730F0004C18BF31F00A
:1011B000004CCAD130F000427FF45CAF31F0004304
:1011C0007FF43CAF5FE700BF4FF0FF3C06E000BF9D
:1011D0004FF0010C02E000BF4FF0010C4DF804CDC0
:1011E0004FEA40024FEA41037FEA226C18BF7FEAD0
:1011F000236C11D001B052EA530C18BF90EA010FD2
:1012000058BFB2EB030088BFC81738BF6FEAE17060
:1012100018BF40F0010070477FEA226C02D15FEAFC
:10122000402C05D17FEA236CE4D15FEA412CE1D068
:101230005DF8040B704700BF844608466146FFE72F
:101240000FB5FFF7C9FF002848BF10F1000F0FBD11
:101250004DF808EDFFF7F4FF0CBF012000205DF80A
:1012600008FB00BF4DF808EDFFF7EAFF34BF01208F
:1012700000205DF808FB00BF4DF808EDFFF7E0FF28
:1012800094BF012000205DF808FB00BF4DF808ED79
:10129000FFF7D2FF94BF012000205DF808FB00BFDC
:1012A0004DF808EDFFF7C8FF34BF012000205DF8BE
:1012B00008FB00BF4FEA4002B2F1FE4F0FD34FF0E0
:1012C0009E03B3EB12620DD94FEA002343F00043B3
:1012D00010F0004F23FA02F018BF404270474FF061
:1012E0000000704712F1610F01D1420205D110F0E8
:1012F000004008BF6FF0004070474FF0000070479B
:101300005400520049004E0041004D004900430086
:1013100020004D006F00740069006F006E00200017
:1013200043006F006E00740072006F006C002E00AE
:1013300054004D00430020004300440043002000BF
:101340004400450056002E0009024300020100C07F
:101350003209040000010202010005240010010509
:10136000240100010424020205240600010705826D
:10137000030800FF09040100020A0000000705033A
:101380000240000007058102400000000403090438
:1013900026035400720069006E0061006D00690050
:1013A00063004D006F00740069006F006E00200044
:1013B000430074006C0000005515AC6A004001C089
:1013C000ABEA57956B7FD87EB87DA07C8F7B857A02
:1013D000827985780878147726763D7559747B7301
:1013E000A172367264719670CC6F076F456EE66DB0
:1013F0002A6D726CBE6B0D6B5F6AB5696169BB6803
:1014000019687967DC664266AB656065CC643B64ED
:10141000AD63206396620F62CB614761C460446034
:10142000C65F495FCE5E925E1A5EA45D2F5DBD5CB5
:101430004B5CDC5BA55B385BCC5A625AF95992591C
:101440002C59F95895583358D15771571257B456EB
:101450000000C90092015B022403ED03B6047F057E
:1014600048061107D907A2086A09330AFB0AC40B08
:101470008C0C540D1C0EE30EAB0F72103A110112BE
:10148000C8128F1355141C15E215A8166E173318C1
:10149000F918BE19821A471B0B1CCF1C931D571E2F
:1014A0001A1FDD1F9F2061212322E522A623672426
:1014B0002825E825A82667272628E528A329612AC4
:1014C0001F2BDC2B992C552D112ECC2E872F413024
:1014D000FB30B5316E322633DF3396344D3504366A
:1014E000BA366F372438D9388C39403AF23AA53BAE
:1014F000563C073DB83D683E173FC53F734021410C
:10150000CE417A422543D0437A442445CD457546A1
:101510001C47C34769480F49B449584AFB4A9D4B89
:101520003F4CE04C814D204EBF4E5D4FFB4F9750DE
:101530003351CE51685202539B533254C9546055B3
:10154000F5558A561D57B0574258D3586459F35928
:10155000825A0F5B9C5B285CB35C3E5DC75D4F5E4F
:10156000D75E5D5FE35F6860EB606E61F061716242
:10157000F1627063EE636C64E8646365DD65566612
:10158000CF664667BC673268A66819698B69FD69D2
:101590006D6ADC6A4A6BB76B236C8E6CF86C616D9C
:1015A000C96D306E966EFB6E5E6FC16F2270837078
:1015B000E27040719D71F9715472AE7207735E737F
:1015C000B5730A745F74B27404755575A575F375B7
:1015D00041768D76D87622776B77B377FA773F7836
:1015E0008478C77809794A798979C879057A417AFE
:1015F0007C7AB67AEE7A267B5C7B917BC57BF87B26
:10160000297C597C887CB67CE37C0E7D397D627DAB
:10161000897DB07DD57DFA7D1D7E3E7E5F7E7E7E9E
:101620009C7EB97ED57EEF7E097F217F377F4D7FFF
:10163000617F747F867F977FA67FB47FC17FCD7FD8
:10164000D87FE17FE97FF07FF57FF97FFD7FFE7F27
:101650000010161B2023272A2D30323537393B3D09
:101660004041434547494B4C4E50515354565759AE
:101670005A5B5D5E60616263656667686A6B6C6D2C
:101680006E707172737475767778797A7B7C7D7EF3
:1016900080808182838485868788898A8B8C8D8EE1
:1016A0008F9090919293949596969798999A9B9BE8
:1016B0009C9D9E9FA0A0A1A2A3A3A4A5A6A7A7A806
:1016C000A9AAAAABACADADAEAFB0B0B1B2B2B3B433
:1016D000B5B5B6B7B7B8B9B9BABBBBBCBDBDBEBF6F
:1016E000C0C0C1C1C2C3C3C4C5C5C6C7C7C8C9C9B4
:1016F000CACBCBCCCCCDCECECFD0D0D1D1D2D3D300
:10170000D4D4D5D6D6D7D7D8D9D9DADADBDBDCDD55
:10171000DDDEDEDFE0E0E1E1E2E2E3E3E4E5E5E6B1
:10172000E6E7E7E8E8E9EAEAEBEBECECEDEDEEEE14
:10173000EFF0F0F1F1F2F2F3F3F4F4F5F5F6F6F779
:10174000F7F8F8F9F9FAFAFBFBFCFCFDFDFEFEFFE9
:101750000000000001020304010203040607080957
:101760000204060802000000000000013136333098
:08177000563230390000000080
:10177800D100000040000000FB070000FF07000048
:101788000008000001000000010000000200000045
:10179800050000000600000003000000040000002F
:1017A8006C1701080B0C0D0A0E0809000008004010
:1017B80001000000000400400101010101010100D5
:1017C80001000000A000000000127A00004800405C
:1017D80000C20100000008008C130108040000008A
:1017E8009013010826000000DC00002032000000F1
:1017F800100100201A0000004813010843000000EF
:10180800C800002012000000819500088593000898
:10181800D1910008E5910008E99100084992000873
:101828006D920008759300086593000841930008BD
:1018380000000000400000001201100102000040FA
:101848003C2A000002080102030100003203540090
:101858004D0043004D002D003000300030003000B6
:10186800200028007600690072007400750061008D
:101878006C00200043004F004D00290020000000AC
:101888001A0354004D0043004D0030003000300072
:10189800300000000000000000000000D1900008A7
:1018A80055D8000855D8000855D8000855D800085C
:1018B80055D8000855D8000855D8000855D800084C
:1018C800D594000855D8000855D8000855D8000800
:1018D80055D800080401000055D80008AD9100084B
:1018E80055D8000855D8000855D8000855D800081C
:1018F80055D8000855D80008C59100080100000017
:081908000100000001000000D5
:040000050800410CA2
:00000001FF
